:100000000C940D110C943E110C943E110C943E1165
:100010000C943E110C943E110C943E110C943E1124
:100020000C943E110C943E110C943E110C943E1114
:100030000C943E110C943E110C943E110C943E1104
:100040000C943E110C943E110C943E110C943E11F4
:100050000C943E110C943E110C943E110C9430857E
:100060000C943E110C94EC8D0C94C28D0C943E11AA
:100070000C943E110C943E110C943E110C943E11C4
:100080000C943E110C943E110C943E110C943E11B4
:100090000C94988D0C946E8D0C943E110C949125BB
:1000A0000C943E110C943E110C943E110C943E1194
:1000B0000C943E110C943E110C943E110C943E1184
:1000C0000C943E110C943E110C943E110C94448DF2
:1000D0000C941A8D0C943E110C94F08C0C94C68CDC
:1000E0000C943E1107634236B79BD8A71A3968565D
:1000F00018AEBAAB558C1D3CB7CC5763BD6DEDFD4A
:10010000753EF6177231BF000000803F0800000006
:10011000BE922449123EABAAAA2ABECDCCCC4C3EFC
:1001200000000080BEABAAAAAA3E00000000BF00EB
:100130000000803F0000000000084178D3BB4387E7
:10014000D1133D190E3CC3BD4282AD2B3E68EC82FB
:1001500076BED98FE1A93E4C80EFFFBE01C4FF7F80
:100160003F00000000000C943B590C9459630C9420
:100170009C5E0C9454330C94AB320C94C3140C94CA
:100180000B4D0C940D320C94C37F0C94D1460C94FF
:10019000C7360C9491240C94CFC00C9404320C9468
:1001A00099350C94236E0C9497150C94762B0C9423
:1001B000BA140C944D410C94D77F0C940E1C0C94E3
:1001C0001B4D0C942F590C9435220C9441410C94E6
:1001D00010330C94DF620C9487AC0C9422220C94A4
:1001E0004B350C94D03F0C942EAB0C94F1800C94B6
:1001F000FB4B0C9432AB0C94D5450C94E51D0C9440
:10020000E57F0C94EE4C0C9432AC0C94D4120C940C
:10021000C0150C94E3400C949C330C94C9C90C9405
:10022000D6630C94A8230C94B9120C94C9120C94A4
:100230009A5D0C9483350C948D1F0C945A110C9478
:1002400003140C94BB8F0C94B44C0C9466350C9432
:1002500031330C9478120C94FFAB0C9449150C9428
:100260003CAB0C947B120C9490620C947E520C94D8
:10027000812F0C94364D0C9463640C94BCC90C947F
:100280000EC50C9470110C94FE310C941A3A0C9417
:1002900018AC0C9407360C9456110C942AAB0C94A1
:1002A0003CAC0C94C7120C94603F0C94B1360C9487
:1002B000681C0C94681A0C94FC130C941E590C9432
:1002C000654D0C9462C20C9440AB0C94DA7B0C9498
:1002D0002C160C940B640C94D1400C94C6620C94B4
:1002E0008A150C94CA470C9488800C94D4580C94AA
:1002F000BD130C94D5820C94E7800C94911E0C9441
:10030000A1120C949B630C94C9320C9489180C9420
:1003100040110C94222F0C94EF690C9470140C94DF
:10032000AC120C94D8120C9421330C94581F0C94DA
:10033000E5130C94BA3E0C94EC320C943A460C94AF
:1003400045360C9422AC0C94DA400C94EC120C94CC
:100350009C2F0C9466640C9405BF0C9421590C944A
:1003600094760C942C590C94322F0C94B6C90C949E
:10037000CD800C940B7B0C94B5820C9400150C94DE
:10038000BFB00C94D28F0C94CA1C0C94EE800C94C9
:1003900035330C94E7450C9434810C94883F0C94CD
:1003A00069640C94EF330C94754E0C9424410C94B6
:1003B0001C320C94C4830C94DDD60C94FE400C9437
:1003C000A2140C94DC130C94996E0C9469120C9486
:1003D00039370C9479370C9452AB0C94DF150C948C
:1003E00037410C9449890C94B9B00C945C180C9466
:1003F0001C130C94BE140C94B8190C94042D0C947A
:1004000095AE0C947DAC0C943D170C94E4750C9453
:100410009E120C9420AB0C94C8240C94A9280C9424
:100420008FAE0C9450AC0C9423160C9440630C9437
:1004300002470C945BC20C9409160C94E8580C9477
:100440007B110C94F7800C945FAC0C9473AC0C94FF
:1004500069170C94AC140C94D2810C94BC910C943C
:100460006E7F0C94B5C80C9480350C94A93F0C9405
:1004700024AB0C9429820C9446AC0C94BCB00C9424
:1004800012590C942E5D0C9469AC0C947D360C942E
:100490006FCA0C9445130C94F8240C9446CA0C941F
:1004A000F2360C9404AC0C943B820C94C7B00C94C0
:1004B000FD470C9449180C9428360C94854C0C94E8
:1004C00091160C9423250C94B82F0C9446150C947B
:1004D00042820C9428370C9462AE0C9472180C94DF
:1004E000F4130C943D580C9430150C9460240C9427
:1004F00034370C9467810C94C0140C94B47F0C9422
:1005000012AB0C94EAC90C94D21D0C946D140C948B
:100510008D360C941AAB0C94D0370C94A6330C94F3
:10052000554D0C94BA190C9482140C947A580C946E
:1005300022170C9435160C942C3A0C94A6150C9496
:10054000B6190C9412360C9468900C9439130C94D0
:10055000B5120C9488470C940F300C9411410C94F4
:10056000D5C00C94122E0C94ED820C9455360C943C
:100570002C8A0C943E4C0C945B7F0C9434180C9495
:1005800020320C94584D0C9426240C946D7F0C94BE
:1005900051AB0C9403220C94B4690C94DD3B0C9485
:1005A0002AAC0C94B4190C948B170C94ED140C9485
:1005B0004A370C940CAB0C9461CA0C945A620C949C
:1005C000CC120C94285D0C940C370C9439330C9499
:1005D00038AB0C9451360C9416AB0C944B410C94E4
:1005E00013630C9486320C9468320C94BD120C94F4
:1005F0007C120C9420C40C949C1D0C94714E0C9491
:10060000A18F0C94F0810C949B130C9414130C94F4
:1006100070400C94C6450C94D91E0C94F3AF0C9406
:100620008CAE0C94BD630C940EAC0C9404170C941B
:100630003B800C941F5D0C9453310C944AAB0C948A
:10064000E8360C94B52E0C9437330C94FB580C946C
:1006500091AC0C944E2E0C942F900C9477120C9419
:10066000E93F0C94F7310C94C2B00C949D120C9499
:100670006F4E0C941D900C94DA140C9429460C9433
:100680009C3F0C9439830C94EC400C94B0370C9440
:100690008A640C94FF810C94602E0C944EAB0C94E5
:1006A000F7AB0C9449370C94362E0C9476370C9497
:1006B00080810C94F81D0C9446AB0C941A370C9462
:1006C000DC120C94ECAF0C94B28F0C94B4334E410A
:1006D0004E494E495459494E46CDCCCC3D0AD723BC
:1006E0003C17B7D13877CC2B329595E6241FB14F04
:1006F0000A000020410000C84200401C4620BCBE49
:100700004CCA1B0E5AAEC59D746364696E6F7073DC
:100710007578585B00556E6B6E6F776E20737566DB
:100720006669782000556E6B6E6F776E20636D641E
:100730002000636C724374723A2000454F46002FCC
:1007400000496E3A20003D00494E3A003D004C45BC
:100750004741435920494E3A00000020002300261B
:100760000029002C002F00320000010000030106C8
:100770000109012D3E00200023002D3E00200050E5
:10078000656E6465643A2023007261770076616C5F
:100790000074656D70007361740068756500666152
:1007A0006E0052474200485356006D6F6465005317
:1007B0006574436D643A0053746F726564204558E4
:1007C000543A00737566666978436F64653A002031
:1007D000666F7220286D73293A004354524C3A20B8
:1007E0005363686564756C6520636D642000206DDB
:1007F00073203A0041726D656420666F722000209C
:1008000044697361726D656400584F4E0048414CF5
:1008100054002074696D653A004354524C3A20529A
:1008200065733A002054533A0020543A003D00507A
:10083000696E3A004354524C3A20436F6D6D616EBD
:100840006420626C6F636B656420627920647269F6
:10085000766572206F72206368616E6E656C2066CB
:10086000726F7A656E004354524C3A204F4E3A41B3
:100870006C7265616479204163746976650A00432E
:1008800054524C3A2048414C543A416C7265616470
:100890007920496E6163746976650A004354524C4D
:1008A0003A20584F4E3A2044697361626C65640A7D
:1008B000004354524C3A20584F4E3A416C72656195
:1008C0006479204163746976650A004354524C3A56
:1008D00020584F464620736B69707065642E205017
:1008E00072657620636D643A004354524C3A20544A
:1008F00075726E6564206F66662066726F6D3A0071
:100900004354524C3A20526573746F72656420668A
:10091000726F6D3A004354524C3A2049676E6F72C1
:1009200065642C206368616E6E656C20636D643D48
:100930000020457865633A004354524C3A204163A5
:10094000746976653A004354524C3A2048414C54FD
:100950003A416C726561647920496E6163746976AD
:10096000650A004354524C3A20584F4E3A2044698D
:100970007361626C65640A004354524C3A20584FCC
:100980004E3A416C726561647920416374697665A1
:100990000A004354524C3A20584F464620736B6924
:1009A000707065642E205072657620636D643A0025
:1009B0004354524C3A205475726E6564206F6666DB
:1009C0002066726F6D3A004354524C3A2052657360
:1009D000746F7265642066726F6D3A004354524CB6
:1009E0003A204E6F7420656E6F756768206D656D77
:1009F0006F727920666F722067726F7570206F70EA
:100A000065726174696F6E00496E76616C6964200D
:100A100061726700496E76616C696420617267007B
:100A20004354524C3A20556E6B6E6F776E2073753F
:100A30006666697800536B697070656420686F6DD5
:100A40006965207374756666002000205375623DE9
:100A500000204974656D3D004354524C3A20524188
:100A60004D3D004354524C3A204F75744F664D65CE
:100A70006D6F72793A2000282D292000282B29201B
:100A8000002076616C7565206973200020756E6B9F
:100A90006E6F776E0A005D3D005B0020696E7661C7
:100AA0006C6964002000206F6B003A002066616969
:100AB0006C6564003A005265747279696E67204310
:100AC0004D440A004354524C2F706F6C6C3A204FC7
:100AD00075744F664D656D6F72793A2000207365AD
:100AE000632072656D61696E696E6700537461742D
:100AF00075732064656666657265640A00444D58C6
:100B0000000000000000444D585247425700004486
:100B10004D5852474200000050574D000000000061
:100B2000004D42555344494D0000544845524D4FE5
:100B300000000052454C41590000000047524F55FB
:100B40005000000000564354454D500000004D42F7
:100B50005553564300000041434841494552000067
:100B60005350494C45440000004D4F544F52000033
:100B700000005049440000000000004D4255530061
:100B80000000000055415254425244470052454C27
:100B9000415950574D00444D5852474257570056FF
:100BA000454E545300000000454C455641544F52A9
:100BB00000434F554E544552000048554D0000002B
:100BC0000000004D455243555259000020002D3E73
:100BD00000436F6E76657274696E6720002D3E006B
:100BE00057726F6E672041737369676E6D656E74BF
:100BF0002000524742783A200020764C6576656C9A
:100C00003A0020436F6E76563A0020436F6E76535B
:100C10003A0020486F743A00436F6C643A002043F6
:100C20006F6E76657274656420563A00436F6E7617
:100C3000657274656420533A002D3E0057726F6EE2
:100C4000672041737369676E6D656E7420002D3E79
:100C50000057726F6E672041737369676E6D656EC2
:100C600074200053617665643A0020537566663AD5
:100C7000002041543A00206973200044656C65747B
:100C8000696E6720636F6E662E2052414D2077613A
:100C9000733A0053746F70706564006E6F746869A6
:100CA0006E6720746F2073746F700053746F707070
:100CB000696E67206368616E6E656C73202E2E2EE0
:100CC000004E6F7420756E6C6F636B656420696E87
:100CD00020313073202D20636F6E74696E7565202E
:100CE0002E2E2E00556E6C6F636B696E6720636FDE
:100CF0006E666967202E2E2E00436F6E6669672030
:100D00006368616E676564206C6F63616C6C792CDD
:100D100020706F7274616C2064697361626C6564C9
:100D2000002F636F6E6669672E6A736F6E0072655F
:100D3000626F6F742000436D643A20002F636F6D03
:100D40006D616E642F002F72616D2F002F697465C5
:100D50006D2F002F6974656D2F004C6F636174698E
:100D60006F6E3A20687474703A2F2F6C617A7968CC
:100D70006F6D652E72752F707761003F6D61633DF9
:100D8000002669703D0026706F72743D00266E610A
:100D90006D653D002F002000436F6D706C657465BC
:100DA0002E2052656D6F766520746F706963200028
:100DB00024636F6D6D616E6400536B697070696E52
:100DC000672E2E00436C65616E55702072657461EC
:100DD000696E656420746F706963200022002200D0
:100DE0004F75744F664D656D6F727921005D2000FF
:100DF0003A5B000A005D00456D7074793A205B0033
:100E00000A003A004D41433A00554450205379734B
:100E10006C6F6720696E697469616C697A65642EAC
:100E20000A005379736C6F6720706172616D733A59
:100E3000002E6C6F63616C00536572766963652088
:100E40007265636F72643A20006D444E5320726580
:100E500073706F6E64657220737461727465642E52
:100E6000004572726F722073657474696E672075C5
:100E700070204D444E5320726573706F6E646572BE
:100E80002100476F74204950206164647265737358
:100E90003A00276970205B69705B2C646E735B2C71
:100EA00067775B2C7375626E65745D5D5D5D272091
:100EB0002D20736574207374617469632049500A2E
:100EC000004661696C656420746F20636F6E6669AB
:100ED000677572652045746865726E6574207573F8
:100EE000696E6720444843502E20596F7520636116
:100EF0006E20736574206970206D616E75616C6C15
:100F0000792100204D41534B3A002047573A0020A9
:100F1000444E533A004C6F616465642066726F6D95
:100F200020666C6173682049503A000A75736573D6
:100F300020444843500A005374617274696E6720FC
:100F40006C616E0043757272656E74204C414E2068
:100F5000636F6E6669672869702C646E732C67779F
:100F60002C7375626E6574293A000A557365207496
:100F70006865736520636F6D6D616E64733A2027D9
:100F800068656C7027202D207468697320746578FB
:100F9000740A276D61632064653A61643A62653A58
:100FA00065663A66653A3030272073657420616E55
:100FB000642073746F7265204D41432D61646472C7
:100FC00065737320696E20454550524F4D0A27695D
:100FD00070205B69705B2C646E735B2C67775B2C95
:100FE0007375626E65745D5D5D5D27202D20736590
:100FF00074207374617469632049500A27736176A1
:101000006527202D20736176652063757272656E89
:101010007420636F6E66696720696E204E56524178
:101020004D3B204F4E7C4F4646202D20656E616221
:101030006C652F64697361626C65206175746F7390
:101040006176650A2767657427205B636F6E666942
:101050006720616464725D27202D206765742063BA
:101060006F6E6669672066726F6D207072652D63A2
:101070006F6E666967757265642055524C20616EAB
:10108000642073746F726520616464722C204F4E0B
:101090007C4F4646202D20656E61626C652F646929
:1010A0007361626C6520646F776E6C6F6164206F32
:1010B0006E20737461727475700A276C6F61642797
:1010C000202D206C6F616420636F6E6669672066F7
:1010D000726F6D204E5652414D0A2770776427205B
:1010E0002D20646566696E6520616E642073746F7F
:1010F0007265204D5154542070617373776F726420
:101100000A276F746170776427202D2064656669F3
:101110006E6520616E642073746F7265204854544C
:1011200050204150492070617373776F72640A27B1
:101130006C6F67205B73657269616C5F6C6F676C65
:101140006576656C5D205B7564705F6C6F676C6560
:1011500076656C5D27202D20646566696E65206C60
:101160006F67206C6576656C2028302E2E37290A33
:10117000276B696C6C27202D207465737420776150
:10118000746368646F670A27636C65617227202D3A
:1011900020636C65617220454550524F4D0A27729D
:1011A00065626F6F7427202D207265626F6F7420E7
:1011B000636F6E74726F6C6C657200536F6674202F
:1011C0007265626F6F74696E672E2E2E0052414DEC
:1011D0003D000A5379736C6F6720000A6D71747457
:1011E00020000A696E7075747320000A6974656D59
:1011F0007320000A436F6E666967757265643A0012
:101200003B003D0050696E3A003B003D4C4F57009B
:10121000546865726D6F3A004170706C79696E67E1
:1012200020636F6E66696700436F6E666967206151
:1012300075746F736176653A000A5379736C6F67E2
:10124000206465627567206C6576656C3A0053654D
:101250007269616C206465627567206C6576656C87
:101260003A0053617665640A005365742064796EB0
:10127000616D69632049500A00454550524F4D2029
:10128000636C65617265640A004D5154542050616D
:101290007373776F726420757064617465640A009B
:1012A0004F54412050617373776F7264207570647E
:1012B000617465640A00636F756C64206E6F7420DE
:1012C00070617273653A2000557064617465640AD8
:1012D000004E6F204950206164726573730052653F
:1012E0006C656173696E6720736F636B65742061F1
:1012F0006E642072657472790020536176656400B3
:101300004C6F6164696E67204854545020636F6E5F
:10131000666967206F6E20737461727475703A002D
:101320004F4646004F4E002B002D00455461673A52
:10133000200047657420455441473A2000485454E2
:10134000502F312E310025733A2025730D0A0020CD
:10135000485454502F312E310D0A486F73743A207F
:1013600025730D0A4163636570743A202A2F2A0D94
:101370000A436F6E6E656374696F6E3A20636C6FBB
:1013800073650D0A0025730020000D0A00474554BF
:10139000006661696C656420746F20636F6E6E65B2
:1013A00063740A004552524F523A20536572766573
:1013B000722072657475726E65642000436F6E668C
:1013C0006967206E6F74206368616E6765640A00E8
:1013D000446F6E652E0A00436F6E66696720706108
:1013E0007273696E67206661696C65640A00676F75
:1013F0007420436F6E6669670A00687474702072A7
:101400006574636F64652000667265652000436FD4
:101410006E666967205552493A20687474703A2F95
:101420002F002044656661756C7420636F6E666979
:10143000672073657276657220757365643A200063
:101440006C617A79686F6D652E7275000A282D2996
:101450004D554C544956454E54000A282B29505797
:101460004D5F52454C4159000A282B294D444E539B
:10147000000A282D295541525442524944474500FB
:101480000A282B295359534C4F47000A282D29501D
:101490004944000A282D294D43503233303137005A
:1014A0000A282D294152544E4554000A282B294F11
:1014B0005441000A282D29535049204C4544000A24
:1014C000282D294D4F544F5220435452000A282BA7
:1014D000294143204841494552206F6E205365728F
:1014E00069616C33000A282D294343533831312078
:1014F000262048444331303830000A282B295245F1
:1015000053544152545F4C414E5F4F4E5F4D5154C6
:10151000545F4552524F5253000A282D29484152D8
:101520004452455345542C207573696E6720736F80
:101530006674000A282D29434F554E544552000A1F
:10154000282D29444854000A282D294F574952452F
:10155000000A282D2949504D4F44425553000A286E
:101560002D294D4F44425553000A282D29444D58EA
:10157000000A282B2957697A6E6574357830300057
:101580000A282B294672656552616D207072696E5A
:1015900074696E67000A282B295741544348444F09
:1015A00047006C617A79686F6D652E7275000A4329
:1015B0006F6E666967207365727665723A003230C5
:1015C000313730334C0020432B2B20766572736902
:1015D0006F6E3A00326532313336325F3230323339
:1015E0002D31312D3132000A4C617A79686F6D6589
:1015F0002E7275204C6967687448756220636F6E3F
:1016000074726F6C6C65722000204F464600204F4C
:101610004E002042595041535300757074696D65F6
:10162000006672656568656170002054696D657259
:101630003A00204C6F636B733A002000204C6F63BC
:101640006B733A000A52414D3D0020457870697233
:1016500065640A00202D746172676574207A6F6E6C
:10166000652D0020416C61726D204578706972654E
:10167000640A0020636D643A00204375723A0020CA
:101680005365743A00536176656420746F20454554
:1016900050524F4D00536176696E6720636F6E66DE
:1016A000696720746F20454550524F4D2E2E004CD7
:1016B0006F6164656420455441473A004E6F207362
:1016C000746F72656420636F6E666967004C6F614A
:1016D0006465642066726F6D20454550524F4D0021
:1016E0006C6F6164206661696C6564004A534F4E9B
:1016F000206465746563746564004C6F6164696E31
:101700006720436F6E6669672066726F6D2045457E
:1017100050524F4D00203C3C0041433A2000414391
:101720003A2053657269616C207573656420627933
:10173000204143202D2064697361626C696E6720CB
:1017400073657269616C206C6F6767696E67206191
:101750006E6420636D640041433A204F7574206FBE
:1017600066206D656D6F72790041433A20496E695C
:10177000743A200041433A2044652D496E69743A19
:1017800020004F4646004452590046414E5F4F4E9E
:101790004C59004845415400434F4F4C004552526C
:1017A0000041433A204F4B00203E3E200041433A47
:1017B000200041433A20506F6C6C696E67004C4FBB
:1017C00057004D454449554D00484947480041554B
:1017D000544F0072617700717565697400737769A1
:1017E0006E67006C6F636B0020696E697400200087
:1017F00050574D2D4F75742023002073746F700067
:10180000200050574D2D4F75742023003D00506926
:101810006E3A0020696E69740052656C61792D4FD3
:1018200075742023002073746F700052656C6179A9
:101830002D4F75742023003D3E003A0070756220E4
:10184000616374696F6E200069646C65006F666621
:101850000068656174696E670066616E0064727924
:10186000696E6700636F6F6C696E67002069732033
:10187000004F75742000556E6B6E6F776E20737518
:10188000666669782000556E6B6E6F776E20636DAB
:10189000642000616374696F6E0072656C617943E6
:1018A00074723A20005B305D3A2000202D202D20FC
:1018B0002D20EFBBBF003E003E31202D2000200038
:1018C0002E00696E00735F6F7574006D79686F6DBF
:1018D00065004354524C2F657865633A204F757408
:1018E0004F664D656D6F72793A2000202D3E2000C5
:1018F000456D69743A2000202D3E20004974656DC5
:10190000436D643A2000202D3E20004974656D3AF5
:1019100020003E3E2000496E76616C696420636F52
:101920006D6D616E64003E3E3E004E6F204D414342
:1019300020636F6E666967757265643A20736574BB
:10194000206669726D776172652773204D41430A85
:1019500000454550524F4D207369676E6174757232
:1019600065206F6B00496E697469616C697A696E94
:101970006720454550524F4D2E0041424344454655
:101980004748494A4B4C4D4E4F505152535455566F
:101990005758595A6162636465666768696A6B6C17
:1019A0006D6E6F707172737475767778797A303185
:1019B00032333435363738392B2F3D004261736965
:1019C00063200061726475696E6F3A004F54412064
:1019D000696E697469616C697A65640A0044454698
:1019E00041554C542070617373776F726420666F39
:1019F00072204F5441204150492E20557365206F6D
:101A0000746170776420636F6D6D616E6420746FB4
:101A1000207365740070617373776F726400546F24
:101A20006F206D616E79204D51545420636F6E6E3E
:101A3000656374696F6E206572726F72732E2052C7
:101A4000657374617274204C414E00207472792069
:101A5000616761696E20696E2035207365636F6E02
:101A60006473006661696C65642C2072633D00419B
:101A700077616974696E6720666F72207265746140
:101A8000696E656420746F7069637300636F6E6E56
:101A900065637465642061732000202E2E2E002063
:101AA000757365723A003A000A417474656D70741A
:101AB000696E67204D51545420636F6E6E65637478
:101AC000696F6E20746F2000646973636F6E6E655A
:101AD00063746564005573696E67204D51545420DA
:101AE00070617373776F72642066726F6D20636FBD
:101AF0006E666967002E6C6F63616C006D444E53B7
:101B0000206E616D6520757064617465643A2000B3
:101B1000446576696365204E616D653A00417420C5
:101B20006C6561737420646576696365206E616DB0
:101B30006520616E642062726F6B6572204950206F
:101B40006D75737420626520636F6E666967757268
:101B5000656400757074696D652C6672656568658D
:101B600061700024737461747300326532313336EE
:101B7000325F323032332D31312D3132004C6967D2
:101B800068744875622000246E616D65007265613D
:101B900064790024737461746500526562696E64CF
:101BA00020737563636573732E20495020616464EC
:101BB000726573733A004572726F723A2072656291
:101BC000696E64206661696C0052656E6577656454
:101BD00020737563636573732E20495020616464BC
:101BE000726573733A004572726F723A2072656E55
:101BF00065776564206661696C000A4E6F206C69C8
:101C00006E6B0033307320454550524F4D20697341
:101C1000206E6F742072656C6F616465642E205253
:101C200065626F6F7400416363657074696E6720ED
:101C3000636F6D6D616E64732E2E2E0A004E6F20E1
:101C40004D51545420636F6E666967757265640008
:101C50004C6F6164696E6720636F6E6669672066AA
:101C6000726F6D20706F7274616C20646973616251
:101C70006C65642E2075736520676574204F4E2057
:101C8000746F20656E61626C6500436F6E66696794
:101C90002069732076616C696400436F6E74696EAD
:101CA000756520776974682070726576696F7573E1
:101CB0006C79206C6F6164656420636F6E66696720
:101CC0000000002100240027002A002D00300033EE
:101CD0000001010000040107010A010000220025A3
:101CE0000028002B002E0031003400020100000506
:101CF0000108010B0105050505070508080808028C
:101D00000202020A0A080804040404010101010194
:101D10000101010303030303030303040707070C83
:101D20000C0C0C0C0C0C0C02020202060606060639
:101D30000606060B0B0B0B0B0B0B0B05050508081A
:101D400007070404040A0A0A0A0A0A0102102020EA
:101D500008081020401020408002010201080402FF
:101D60000101020408102040808040201008040275
:101D700001800402018040201008040201080402CE
:101D800001010204081020408001020408102040D4
:101D90008004408004800810102040040810204077
:101DA0008000000B0C030A0D0E0F09080405020049
:101DB0000000000000000000000000000000000023
:101DC00000000000000000000000000000131211DD
:101DD0000000000000000000000000000000000003
:101DE00000000000000000000000000000000000F3
:101DF000000000000000002F64617461002F736B0D
:101E000065746368004163636573732D436F6E741B
:101E1000726F6C2D526571756573742D5072697691
:101E20006174652D4E6574776F726B3A20747275AC
:101E300065004163636573732D436F6E74726F6CDD
:101E40002D416C6C6F772D486561646572733A2023
:101E50002A004163636573732D436F6E74726F6CF8
:101E60002D416C6C6F772D4D6574686F64733A20EB
:101E7000504F53542C4745542C4F5054494F4E53B8
:101E8000004163636573732D436F6E74726F6C2DC5
:101E9000416C6C6F772D43726564656E7469616C1B
:101EA000733A2074727565004F5054494F4E530079
:101EB00044454C4554450050555400474554005046
:101EC0004F535400617574686F72697A6174696FF9
:101ED0006E3A2000417574686F72697A6174696F37
:101EE0006E3A2000436F6E74656E742D4C656E679C
:101EF00074683A20006F637465742F73747265613F
:101F00006D00696D6167652F6A70656700696D6155
:101F100067652F67696600746578742F68746D6CE7
:101F2000006170706C69636174696F6E2F6A736FA2
:101F30006E00746578742F706C61696E00436F6E0B
:101F400074656E742D547970653A2000436F6E6E1F
:101F5000656374696F6E3A20636C6F7365004163EB
:101F6000636573732D436F6E74726F6C2D416C6C6F
:101F70006F772D4F726967696E3A202A00556E6B34
:101F80006E6F776E004E6F74204D6F646966696581
:101F900064004F4B004D6F766564207065726D6113
:101FA0006E656E746C7900496E7465726E616C203A
:101FB000536572766572204572726F720050617956
:101FC0006C6F616420546F6F204C61726765004EC6
:101FD0006F7420666F756E64005757572D41757486
:101FE00068656E7469636174653A20426173696300
:101FF000207265616C6D3D2241636365737320726D
:102000006573747269637465642200556E617574DA
:10201000686F72697A6564005061796C6F616420E1
:1020200073697A652077726F6E670042616420720F
:1020300065717565737400485454502F312E3120EA
:102040000020000000000000000000004F4E0000D3
:1020500000000000004F464600000000000052450E
:1020600053540000000000544F47474C4500000007
:1020700048414C540000000000584F4E0000000042
:102080000000584F46460000000000494E435245AC
:1020900041534500444543524541534500454E4157
:1020A000424C4500000044495341424C4500005514
:1020B0004E465245455A4500465245455A45000050
:1020C000004155544F000000000046414E5F4F4E06
:1020D0004C59004849474800000000004D4544491C
:1020E000554D0000004C4F570000000000004845CF
:1020F00041540000000000434F4F4C00000000001E
:1021000044525900000000000053544F500000009A
:1021100000005247420000000000004853560000F3
:102120000000000057726F6E67207061796C616407
:10213000004354524C2F7478743A204F75744F6694
:102140004D656D6F72793A2000202D3E2041543A42
:10215000004368616E20747970653A004E6F207399
:10216000746F7265642076616C756573202D2064D0
:10217000656661756C743A2000536176656420452C
:102180005441473A0053657420455441473A200072
:102190002D3E005075623A20006374726C00454E0B
:1021A00041424C4500465245455A45004449534139
:1021B000424C45002D3E005075623A2000636D642C
:1021C0000046414E5F4F4E4C590044525900434F18
:1021D0004F4C0048454154004155544F002D3E009E
:1021E0005075623A20007365740064656C002D3E82
:1021F000005075623A20002D3E005075623A200072
:10220000556E6B6E6F776E20636D64200A004F46CB
:1022100046004F4E0000DDD605BF11241FBECFEF94
:10222000D1E2DEBFCDBF00E00CBF16E0A0E0B2E01F
:10223000E4EEF8ED01E00BBF02C007900D92AE3F57
:10224000B107D9F72DE0AEEFB6E001C01D92A33E75
:10225000B207E1F711E1CCE0D1E100E006C021973F
:102260000109802FFE010E9442E4CB30D10780E0BB
:102270000807A9F70E9422BF0C9460EC0C940000A0
:10228000CF93DF931F92CDB7DEB76983DC01ED9169
:10229000FC910280F381E02D41E050E0BE016F5FD0
:1022A0007F4F19950F90DF91CF910895FC01818D9B
:1022B000928D0895CF93DF931F92CDB7DEB76983D8
:1022C000DC01ED91FC910280F381E02D41E050E0D2
:1022D000BE016F5F7F4F19950F90DF91CF910895E9
:1022E000FC019485FB018485981303C081E098303C
:1022F00008F080E00895CF93DF931F92CDB7DEB74B
:102300006983DC01ED91FC910280F381E02D41E0D5
:1023100050E0BE016F5F7F4F19950F90DF91CF9115
:10232000089585ED8093BC008091BC0084FDFCCFB6
:1023300010921F0808952091FB07260F3327331FA3
:1023400021323105ECF420911F08FC0190E080E07F
:10235000243069F082E00895A091FB072191AC013F
:102360004552584FA40FB52FB11D2C9301968617D7
:1023700098F38091FB07680F6093FB0780E0089556
:1023800081E008958FEF9FEF08958FEF9FEF0895FD
:102390008091DA0790E09195819591090895CF9306
:1023A000DF93CB01EA01642F0E949B11CE01DF91E4
:1023B000CF910895CF93DF931F92CDB7DEB7698396
:1023C00061E0CE0101960E949B1181E090E00F90A8
:1023D000DF91CF910895CF93DF93EA01282FDC019D
:1023E000ED91F0E094E0F595E7959A95E1F7ED5BD6
:1023F000FC4F80818883FD013197E081EF70F0E030
:10240000ED5BFC4F8081898322968A2F821B861781
:1024100038F3615070E0660F771F460F571FFA01BF
:102420001282DF91CF91089590E0FC01EB50F34EC2
:10243000E491F0E0EE0FFF1FE552F34EA591B49149
:102440002C91855B924EFC018491822391E009F4EA
:1024500090E0892F0895FC01DC018D918111FDCF61
:1024600030E020E050E040E08AE09191992301F1D2
:10247000443051055CF59E3271F42F3F310509F06F
:102480002CF5DB01A40FB51F12962C934F5F5F4F05
:1024900030E020E0EACF829FD001839FB00D11246D
:1024A000292F990F330B205331092A0F3B1FDDCF02
:1024B0002F3F310509F054F4443051053CF4640FCA
:1024C000751FFB01228381E090E0089590E080E099
:1024D0000895DC0115968D919C91009739F0DC01EF
:1024E000ED91FC910680F781E02D199408950895EF
:1024F00083E090E008950895DC011296ED91FC913F
:1025000013973097B9F016968D919C918430910570
:1025100041F08530910541F0039749F482E090E065
:10252000089581E090E0089581E190E0089580852C
:1025300090E0089590E080E00895089585E090E0AF
:102540000895DC011496ED91FC9180E0309711F034
:1025500085A1817090E008958FE090E09093350818
:102560008093340888EC90E00895FC018481958183
:102570000895FC01768765870895DC01ED91FC9153
:10258000068CF78DE02D199591E089270895862F07
:10259000089581E08627089521E0FC018485883034
:1025A00008F020E0822F0895FC0184859585089528
:1025B000FC0184899589089524E634E0FC01318387
:1025C0002083FB014089518962897389FC01428320
:1025D0005383648375830895DC01ED91FC91048C31
:1025E000F58DE02D19940F931F93CF93DF93DC01AA
:1025F000C62F1196EC911197E295EF70EC3008F030
:10260000BCC0F0E08827E85FFC4E8F4F0C9442E49A
:10261000141339133913BD13BD13BD139B13451385
:10262000BD13BD131C131C1370E060E0CB01DF91E0
:10263000CF911F910F91089514968D919D910D90BA
:10264000BC91A02D8F3F9105A105B10529F024F083
:102650008FEF90E0A0E0B0E0B7FF03C080E090E033
:10266000DC016FEF70E0681B790BC111DFCFBC019B
:10267000DDCF14966C9170E0CC23C1F28FEF90E027
:102680009C01261B370BB901D1CF862F14960C91D4
:10269000149715961C9115971696DC911697179618
:1026A000CC9120E030E0A901B801882331F18D2FD1
:1026B0009C2F0E9481E287FD1BC020E030E04FE7A5
:1026C00053E4B8018D2F9C2F0E9475E5181624F451
:1026D00000E010E0DFE7C3E498014D2F5C2F60E0DD
:1026E00070E08FE793E40E9460E40E943FE59ECF94
:1026F00000E010E0D0E0C0E0EFCF8D2F9C2F0E94D3
:1027000081E287FD13C020E030E04FE753E4B801D9
:102710008D2F9C2F0E9475E5181624F400E010E020
:10272000DFE7C3E4B8018D2F9C2FDFCF00E010E07E
:10273000D0E0C0E0F7CF14966D917D918D919C9182
:10274000179724E630E040E050E00E94EDE32F3F91
:1027500031054105510529F024F02FEF30E040E02C
:1027600050E057FF03C020E030E0A9016FEF70E0B8
:10277000621B730BC1115ACF86CF6FEF7FEF56CF1D
:10278000DC011196EC911197E295EF70E150EB307E
:1027900008F039C0F0E08827EF52FC4E8F4F0C94C0
:1027A00042E4F413F4130314DC13DC13E513FC13F9
:1027B000FC13FC13DC13DC1314966D917D918D9149
:1027C0009C9117970E9488E2089514966D917D91CF
:1027D0008D919C91179724E630E040E050E00E94F4
:1027E000EDE3CA01B901EECF14966C9170E090E070
:1027F00080E00E9486E2089514966D917D918D91FE
:102800009C911797089560E070E0CB010895FC015A
:10281000A7812A2F2E7FD1F0818182958F708150E0
:102820008330A0F4A695A150BB0B2BE531E00E94AC
:1028300059E424E630E040E050E00E94EDE3DA01A4
:10284000C90187569F4FAF4FBF4F08958FEF9FEF3E
:102850000895DC01ED91FC91309729F090859F70EF
:1028600081E0953009F080E00895FC01A481B581F4
:10287000109721F118969C9118979F708EEF890FF1
:10288000823010F091111AC019964D935D936D939B
:102890007C931C97A481B58118969C911897907F82
:1028A000926018969C930480F581E02D8085982F86
:1028B000907F903619F48F70806A80870895DC01CC
:1028C00019968D919C91009739F0DC01ED91FC9166
:1028D0000280F381E02D1994089588E090E0089536
:1028E000CF93DF93EC01E881F9810484F585E02D35
:1028F000199529893A892F5F3F4F3A8B298BDF91B0
:10290000CF910895CF93DF93EC018E8581110DC097
:1029100081E090E049895A892C853D85421753070B
:1029200008F080E0DF91CF910895E881F981048477
:10293000F585E02DCE0119958F3F910549F780E08F
:1029400090E0F0CFFC01848595856817790708F43D
:10295000CB01928B818B0895DC011E962C911E97E2
:10296000222339F0ED91FC910190F081E02D6FEF81
:1029700019940895FC0187859089089581E0089550
:1029800090E080E00895FC0122813381232B49F0FF
:10299000868197818130910539F01CF00397039768
:1029A00030F090E080E0089581E090E0089582E0CA
:1029B00090E00895DC011296ED91FC91309761F062
:1029C0000190F081E02D309739F0862F8295807F3D
:1029D00060856F70682B60870895DC011296ED9119
:1029E000FC91309751F00190F081E02D309729F063
:1029F000808582958F7090E0089590E080E0089542
:102A0000CF93DF93CDB7DEB760970FB6F894DEBFF4
:102A10000FBECDBF19821A821B821C821D821E82AC
:102A20001F8218868A818F7080618A836FEF3E8152
:102A30009F81888529817A815B814C814C873E8783
:102A4000888B372F452F5C857E85892F98896096E6
:102A50000FB6F894DEBF0FBECDBFDF91CF910895C2
:102A60000F931F93CF93DF9300D000D01F921F923C
:102A7000CDB7DEB781E028960FB6F894DEBF0FBE63
:102A8000CDBFDF91CF911F910F91089590E080E02D
:102A90000895CF92DF92EF92FF920F931F93CF93FF
:102AA000DF9300D000D0CDB7DEB78C016B017A0187
:102AB000FC01808D883010F40E94CC9884E694E06C
:102AC0009A838983F60182819381A481B5818B8366
:102AD0009C83AD83BE83B701CE0101960E940AAAF2
:102AE000F801808F8830A0F4F586E486128E118E6E
:102AF00081E026960FB6F894DEBF0FBECDBFDF9102
:102B0000CF911F910F91FF90EF90DF90CF9008959C
:102B100080E0EFCFCF93DF93EC01888D883020F4F5
:102B20000E94CC9888E0888FDF91CF910895FC01B6
:102B3000808D883040F4218D328D232B21F00E942E
:102B40009E9790E008958FEF9FEF0895CF93DF93C6
:102B5000FC012485283028F08FEF9FEFDF91CF9183
:102B60000895EC010190F081E02D0084F185E02DC5
:102B70001995892B89F38C850E949E9790E0EECF62
:102B8000CF93DF93FC01218D328D2115310529F47E
:102B90008FEF9FEFDF91CF910895EC01808D421769
:102BA000530708F0A9010E94ED971816190684F73B
:102BB000298D3A8D281B390B3A8F298FEBCF0F9334
:102BC0001F93CF93DF931F92CDB7DEB7FC01218D0A
:102BD000328D232B41F48FEF9FEF0F90DF91CF9138
:102BE0001F910F9108958C0141E050E0BE016F5F8D
:102BF0007F4FFC01808D0E94ED97181619065CF737
:102C0000F801818D928D0197928F818F898190E05B
:102C1000E4CFCF93DF931F92CDB7DEB741E050E012
:102C2000BE016F5F7F4FFC0184850E94ED971816EF
:102C3000190634F4898190E00F90DF91CF910895C7
:102C40008FEF9FEFF9CFFC018485883010F40C944E
:102C5000ED9790E080E00895FC018485883010F4C1
:102C60000C94C69790E080E008950F931F93CF9344
:102C7000DF9300D000D01F921F92CDB7DEB78C013A
:102C8000D80159964D915C915A974115510551F0D3
:102C9000ED91FC91048CF58DE02D70E060E0C801B1
:102CA0001995EECFF801808D0E94C697892BB1F15E
:102CB00048E050E0BE016F5F7F4FD80158968C917D
:102CC0000E94ED9718161906F4F4D801509684E086
:102CD000FE01319601900D928A95E1F78D8190E089
:102CE000982F88272E81820F911DF801958B848B58
:102CF0008F81282F30E0322F22278885820F932F53
:102D0000911D928F818F28960FB6F894DEBF0FBE6B
:102D1000CDBFDF91CF911F910F91089590E080E09A
:102D2000F2CFCF92DF92EF92FF920F931F93CF9348
:102D3000DF93CDB7DEB7AF970FB6F894DEBF0FBE07
:102D4000CDBF7C016A0104E614E01A8309831C8666
:102D50001B8688EE93E0A0E0B0E08D879E87AF876A
:102D6000B88B8AE394E09A878987188F0F8B198E26
:102D70001A8E1B8E1C8E88E089A31BA70AA71CA68F
:102D80001DA61EA61FA68091300B9091310BA0911D
:102D9000320BB091330B8EA39FA3A8A7B9A78B8347
:102DA0009C83AD83BE8318861F82AE01465D5F4F54
:102DB000CE0101960E94E5B281309105B1F4D701B0
:102DC000ED91FC910488F589E02D1DA30CA38CA541
:102DD0009DA5AEA5BFA58EA39FA3A8A7B9A7A60131
:102DE000BE016C5D7F4FC7011995AF960FB6F89481
:102DF000DEBF0FBECDBFDF91CF911F910F91FF902E
:102E0000EF90DF90CF9008950F931F93CF93DF93B0
:102E1000EC018B01888D883010F40E94CC98B801A9
:102E200082E00E941599888F883050F41D870C87A6
:102E30001A8E198E81E0DF91CF911F910F91089525
:102E400080E0F9CF0F931F93CF93DF938C01EA01BA
:102E5000FC018485883048F40E943C97892B39F422
:102E600081E090E0F80193838283D0E0C0E0CE015E
:102E7000DF91CF911F910F910895EF92FF920F93E1
:102E80001F93CF93DF937C0180911E09D4E083339D
:102E900009F0D8E00EE019E0C0E0F801219131918D
:102EA0008F01F701848195812817390729F0CF5FB9
:102EB000DC13F3CF80E006C08C2F0E94DA988431B7
:102EC000B1F781E0DF91CF911F910F91FF90EF90CB
:102ED0000895CF93DF93EC018C858830D0F40E9465
:102EE000DA98843189F0882379F0883169F021E01B
:102EF0008C3159F4E881F9810084F185E02DCE010F
:102F0000199521E0892B09F420E0822FDF91CF91E0
:102F1000089580E0FBCFCF92DF92EF92FF920F9364
:102F20001F93CF93DF93CDB7DEB7AF970FB6F8946B
:102F3000DEBF0FBECDBF8C016B017A0184E694E049
:102F40009A8389831B821C821D821E821C861B869B
:102F500048EE53E060E070E04D875E876F87788BC6
:102F60002AE334E03A872987988F8F8B198E1A8E3F
:102F70001B8E1C8E28E029A39BA78AA71CA61DA632
:102F80001EA61FA6D8011C968C91883060F40E9462
:102F9000DA98882321F0F80184850E94BE9888E0A1
:102FA000D8011C968C938091300B9091310BA0919D
:102FB000320BB091330B8EA39FA3A8A7B9A78B8325
:102FC0009C83AD83BE8318861F82AE01465D5F4F32
:102FD000B601CE0101960E94E5B20097C1F0D8017A
:102FE000ED91FC910684F785E02D84E694E09DA3A5
:102FF0008CA38CA59DA5AEA5BFA58EA39FA3A8A7B6
:10300000B9A7A701BE016C5D7F4FC8011995AF96A6
:103010000FB6F894DEBF0FBECDBFDF91CF911F91E9
:103020000F91FF90EF90DF90CF9008950F931F9333
:10303000182F0E940DAD04C09695879577956795DA
:103040001A95D2F78B019C01015011092109310910
:103050000E3F1F4F2F4F3F4F20F061E070E080E0A8
:1030600090E01F910F910895CF93DF93EC018C8531
:10307000883060F40E94DA98873111F08C3131F495
:103080008C850E941F978115984088F3DF91CF911E
:103090000895FC018485883010F40C941F9790E00B
:1030A00080E0089567E273E1811102C069E273E193
:1030B00084E19CE00C94D48A6BEB71E184E19CE0A8
:1030C0000E94D48AF0E0E0E0199584EF91E0089541
:1030D0006CE77AE0811102C067E77AE085EC9CE05A
:1030E0000C94D48ADC0155962C915597273781F49E
:1030F000ED91FC91008CF18DE02D19956BE377E05B
:1031000085EC9CE00E94D48A85EC9CE00C943E897E
:1031100008954F925F926F927F92AF92BF92DF922B
:10312000EF92FF920F931F93CF93DF9300D000D0C5
:10313000CDB7DEB77C01D62E8091D707882309F45E
:10314000BEC0D70114969C9180912902891708F47A
:10315000B6C08091D5079091D607BAE06B13F0C046
:103160008B57984FFC011082D70118960D911C9136
:103170000115110509F49FC0F8016185728561157B
:10318000710591F4458056806780708480912A0B88
:1031900090912B0BA0912C0BB0912D0B481659063A
:1031A0006A067B0609F487C0D8011B964D915C9195
:1031B0001C974115510509F47EC0F70124815396EF
:1031C0008C91539790E0322F377002C09595879578
:1031D0003A95E2F780FF6FC0A22EB12CC501887F1F
:1031E0009370892B39F451968D919C91887F9370BF
:1031F000A82AB92AD8018D919C91DC01ED91FC910E
:103200006115710509F486C00688F789E02D1995C6
:10321000019709F050C06CE3F801808191810E9410
:10322000DD89A50170E060E02AE0D8018D919C91D4
:103230000E94F288F80122818081918168EB78E117
:10324000222311F066EB78E10E94D48AD8011D9602
:103250006D917C911E978D919C910E946E8A60E287
:10326000F801808191810E94DD89D8011F966D91BE
:103270007C9150978D919C910E946E8AF8012281D9
:10328000808191816BEA78E1222311F065EA78E18F
:103290000E94D48A65E877E0D8018D919C910E94C4
:1032A0006E8AF80180819181DC01ED91FC91008CA6
:1032B000F18DE02D19951092D6071092D507D70100
:1032C00015968D919C911697009771F014963C91EC
:1032D00020912A02231740F0DC01ED91FC9101902E
:1032E000F081E02D6D2D199581E090E026960FB6C6
:1032F000F894DEBF0FBECDBFDF91CF911F910F912C
:10330000FF90EF90DF90BF90AF907F906F905F90B5
:103310004F9008950488F589E02D24E634E03A833F
:103320002983D80115964D905D906D907C901897EB
:103330004B825C826D827E82BE016F5F7F4F67CF62
:103340008F3491050CF0BBCFBDE06B1709F4B7CFFC
:103350009C012F5F3F4F3093D6072093D5078B57A3
:10336000984FFC016083ABCF0C94EFDA0C94EFDA4A
:103370000C94EFDACF93C1E068EE73E080E090E068
:103380000E94DBAC4AE050E06C2F84E19CE00E949C
:103390004289CF5FC43181F784EF91E0CF910895E6
:1033A000CF93DF93009709F490C0FC012081222382
:1033B00009F48BC0EC0166EE71E20E948CDC892B73
:1033C00009F45FC069E971E2CE010E948CDC892BAF
:1033D00009F45AC06DEB71E2CE010E948CDC892B9E
:1033E00009F455C06AEA77E0CE010E948CDC892B93
:1033F00009F450C066EA77E0CE010E948CDC892B8C
:1034000009F44BC062EA77E0CE010E948CDC892B84
:1034100009F446C06EE977E0CE010E948CDC892B6E
:1034200009F441C06AE977E0CE010E948CDC892B67
:10343000E9F166E977E0CE010E948CDC892BC9F1C5
:1034400061E977E0CE010E948CDC892BA9F16DE85F
:1034500077E0CE010E948CDC892B89F16AEE71E263
:10346000CE010E948CDC892B69F169E877E0CE01FE
:103470000E948CDC892B49F58DE090E0DF91CF91A3
:10348000089582E090E0FACF89E090E0F7CF81E004
:1034900090E0F4CF88E090E0F1CF85E090E0EECFCF
:1034A00086E090E0EBCF87E090E0E8CF8AE090E024
:1034B000E5CF8BE090E0E2CF8CE090E0DFCF83E0DF
:1034C00090E0DCCF84E090E0D9CF90E080E0D6CFF0
:1034D000CF93DF93EC016BE278E185EC9CE00E94F6
:1034E000D48A6C817D8185EC9CE00E94B49F65E26A
:1034F00078E185EC9CE00E94D48A85EC9CE00E94F7
:103500003E8960E08C810E9483ABE881F98106846A
:10351000F785E02D60E0CE01199581E090E0DF9124
:10352000CF910895EF92FF921F93CF93DF93192FBE
:103530007B01C82FD92FD7FF03C0D195C195D109E1
:1035400061E08C2F0E9483AB82E0E816F10499F4CD
:1035500060E08C2F0E9455AB62E176E185EC9CE047
:103560000E94D48A85EC9CE0DF91CF911F91FF905F
:10357000EF900C943E89612FEF2851F46095661FFF
:103580006627661F8C2F0E9455AB6EE076E1E6CF72
:10359000661F6627661F8C2F0E9455AB69E076E197
:1035A000DDCF65E0FC01808191810E94A59F00979D
:1035B00049F0FC018085982F907F21F082958F70D3
:1035C00090E0089590E080E00895FC018681978165
:1035D000009799F0FC0120852F70223029F4618535
:1035E0007285838594850895253039F460E00E94C2
:1035F000A59F009711F0FC01F2CF60E070E0CB01D5
:103600000895CF93C62F63E0FC01808191810E94D1
:10361000A59FFC01892B21F19085892F8D7001F5E3
:10362000907F9260908781859285A385B485882755
:10363000BB278C2B81879287A387B4876FEA77E0BB
:1036400085EC9CE00E94D48A4AE050E06C2F85EC27
:103650009CE00E94428985EC9CE0CF910C943E89CD
:10366000CF91089563E0FC01808191810E94A59F24
:10367000009719F0FC01818508958FEF0895FF925E
:103680000F931F93CF93DF93CDB7DEB764970FB639
:10369000F894DEBF0FBECDBF8C01F62E8FE290E016
:1036A0009A838983FE01339688E0DF011D928A9513
:1036B000E9F7F8016681FF2011F081E06827D80161
:1036C00014968C910E9455ABF80187819085A18555
:1036D000B285883E9340A105B10508F48BC061E72F
:1036E00078E185EC9CE00E94D48AD80114966D9113
:1036F0007C9185EC9CE00E94B49F6CE678E185ECBF
:103700009CE00E94D48A6F2D70E085EC9CE00E94C2
:10371000B49F85EC9CE00E943E8963E978E1CE018C
:1037200001960E9481DCF801828193810E94321B04
:10373000FF2009F46BC064E678E1843151F06DE557
:1037400078E1853131F061E578E18F3011F469E598
:1037500078E1CE010B960E9495DC6CE378E185EC74
:103760009CE00E94D48AD8011296ED91FC911397A7
:103770000190F081E02D60817181ED91FC910488D0
:10378000F589E02D9E012F5F3F4FAE01455F5F4FF2
:10379000C8011995BC0185EC9CE00E94B49F6AE3C6
:1037A00078E185EC9CE00E94D48AD8011296ED91D4
:1037B000FC910190F081E02D6081718185EC9CE0AD
:1037C0000E946E8ABE016F5F7F4F85EC9CE00E9475
:1037D0006E8A67E378E185EC9CE00E94D48ABE01A2
:1037E000655F7F4F85EC9CE00E946E8A85EC9CE0D3
:1037F0000E943E8964960FB6F894DEBF0FBECDBF1F
:10380000DF91CF911F910F91FF9008956DE478E1C2
:10381000823009F49ECF68E478E19BCF81E090E0AC
:103820000895DC011296ED91FC91309771F090852E
:103830009F70923039F0953041F4CF010E94BC9FC7
:1038400090E0089581E090E0089590E080E0089590
:103850000F931F93CF93DF93FC01C281D3812097F5
:10386000F9F088858F70823049F4672BC9F4898517
:103870009A85DF91CF911F910F910895853081F442
:103880008B01CE010E94BC9F8017110649F044F0C5
:10389000602FCE010E94A59FFC0181859285E9CF12
:1038A00090E080E0E6CFFC016115710519F4848198
:1038B0009581089586819781681779072CF0848116
:1038C0009581860F971F0895828193810C94281CFF
:1038D000CF93DF93EC0162E078E185EC9CE00E94FD
:1038E000D48A6C817D8185EC9CE00E94B49F60E06D
:1038F00078E185EC9CE00E94D48AEA81FB8101900A
:10390000F081E02D6081718185EC9CE00E946E8ADF
:103910006AEF77E185EC9CE00E94D48A85EC9CE01C
:103920000E943E89E881F981068CF78DE02DCE0159
:1039300019958130910529F0029759F060E08C814A
:103940001AC063E070E0CE010E94531C60E00E9448
:1039500083AB60E08C810E9483AB61E070E0CE01BC
:103960000E94531C60E00E9483AB62E070E0CE01D5
:103970000E94531C60E00E9483ABE881F9810684B9
:10398000F785E02D60E0CE01199581E090E0DF91B0
:10399000CF910895CF93DF93EC0160EF77E185EC51
:1039A0009CE00E94D48A6C817D8185EC9CE00E9421
:1039B000B49F6EEE77E185EC9CE00E94D48AEA81A8
:1039C000FB810190F081E02D6081718185EC9CE0AC
:1039D0000E946E8A68EE77E185EC9CE00E94D48AB2
:1039E00085EC9CE00E943E898A819B81892B09F4A9
:1039F00051C08C819D81892B09F04CC0E881F981EF
:103A0000068CF78DE02DCE0119958130910529F0B6
:103A1000029759F061E08C811AC063E070E0CE013A
:103A20000E94531C61E00E9483AB61E08C810E9484
:103A300083AB61E070E0CE010E94531C61E00E9404
:103A400083AB62E070E0CE010E94531C61E00E94F3
:103A500083AB8091A100887F8093A1008091910029
:103A6000887F809391008091A10082608093A10063
:103A700080919100826080939100E881F9810684B1
:103A8000F785E02D62E0CE01199581E090E0DF91AD
:103A9000CF91089590E080E0FACFCF93DF9300D0EC
:103AA00000D01F921F92CDB7DEB7EEEFFBE0128A77
:103AB000118A80E090E19587848784E890E0948B78
:103AC000838B81E0868780E090E2908B878787E711
:103AD000858B1C821B8281E393E09A838983FE831A
:103AE000ED838FEF9FEF98878F8365E976E184E11F
:103AF0009CE00E94D48A6091830770918407CE0174
:103B000001960E947A8F8EEF9BE00E94721865E802
:103B100076E184E19CE00E94D48A84E19CE00E94EA
:103B20003E890E94B9B528960FB6F894DEBF0FBE45
:103B3000CDBFDF91CF910895CF92DF92EF92FF92A8
:103B40000F931F93CF93DF93CDB7DEB760970FB678
:103B5000F894DEBF0FBECDBF7C016B01CA01B90175
:103B60002AE0AE014F5F5F4F0E9430DDD701ED913B
:103B7000FC910488F589E02D9801AE014F5F5F4FFD
:103B8000B601C701199560960FB6F894DEBF0FBE57
:103B9000CDBFDF91CF911F910F91FF90EF90DF90FC
:103BA000CF900895892B71F0FB01828193810E944F
:103BB000CAA060EA72E184E19CE00E94D48A88ECA9
:103BC00090E0089590E080E0F2CF892B71F0FB0146
:103BD000828193810E947CA069E872E184E19CE08B
:103BE0000E94D48A88EC90E0089590E080E0F2CFC3
:103BF000EF92FF920F931F93CF93DF93CDB7DEB772
:103C00002C970FB6F894DEBF0FBECDBF8C017B01A1
:103C100084E694E09A8389831B821C821D821E8223
:103C200098878F8319861A861B861C860530110596
:103C3000ECF0BE01695F7F4FF701808591850E949E
:103C40002B12892B99F0CE0107960E946DA1BE011F
:103C5000695F7F4FF701868197810E942B12892B24
:103C600061F0CE0107960E9417A20EC0CE01019608
:103C70000E946DA10430110554F7CE0101960E94F7
:103C800017A203301105A4F1BE01695F7F4FF70150
:103C9000848195810E942B12892B51F1CE010796C8
:103CA0000E94C2A1BE01695F7F4FF70182819381AB
:103CB0000E942B12892B19F1CE0107960E9418A1A0
:103CC00062E672E184E19CE00E94D48A80E00E9476
:103CD00003A388EC90E02C960FB6F894DEBF0FBEDD
:103CE000CDBFDF91CF911F910F91FF90EF9008957D
:103CF000CE0101960E94C2A1023011059CF6CE01B0
:103D000001960E9418A101301105D1F6CE0101964D
:103D10000E9418A169E672E184E19CE00E94D48AC5
:103D2000CFCF0F931F93CF93DF938C01EB010297BB
:103D3000C4F08A819B810E9420DC80932A0299270B
:103D40000E9416A30230110549F08C819D810E94CA
:103D500020DC8093290299270E9420A3C8ECD0E0A0
:103D600002C0C0E9D1E06EE472E184E19CE00E940F
:103D7000D48A4AE050E060912A0284E19CE00E94EB
:103D8000428969E372E184E19CE00E94D48A4AE0BE
:103D900050E06091290284E19CE00E94428984E124
:103DA0009CE00E943E89CE01DF91CF911F910F913F
:103DB0000895CF93DF93EB010297A4F164E273E1DE
:103DC0008A819B810E946EDC892B29F40E946CA25F
:103DD0006F770E94B3A260E273E18A819B810E94A7
:103DE0006EDC892B29F40E946CA260680E94B3A249
:103DF00068E272E184E19CE00E94D48A0E946CA295
:103E00006095661F6627661F70E084E19CE00E9453
:103E1000B49F84E19CE00E943E8988EC90E0DF91B1
:103E2000CF9108950E944D1DF8CFEF92FF920F930E
:103E30001F93CF93DF93EC017B018E819F81892BB0
:103E4000A9F4888199810E94BC9F082F10E0053059
:103E5000110564F40E944AA39F838E83BC0188816C
:103E600099810E942CA30F5F1F4FF1CFEE81FF813C
:103E70003097D9F08085982F9F70A9F4807F826059
:103E80008087EE81FF811186128613861486EE816B
:103E9000FF81F782E682C701DF91CF911F910F91D9
:103EA000FF90EF900895923061F3F12CE12CF3CF65
:103EB000CF93DF93FC0122813381232B59F1EC0155
:103EC00064E777E185EC9CE00E94D48A4AE050E008
:103ED0006E8185EC9CE00E94428985EC9CE00E940A
:103EE0003E898C819D810E94EFDA70E060E08A81DA
:103EF0009B810E94151F1D821C82E881F981068426
:103F0000F785E02D60E0CE01199581E090E0DF912A
:103F1000CF91089590E080E0FACF0F931F93CF9355
:103F2000DF93DC0112962D913C91232B81F1EC0162
:103F300069E677E185EC9CE00E94D48A4AE050E093
:103F40006E8185EC9CE00E94428985EC9CE00E9499
:103F50003E898C819D81892B61F40A811B818CE2D1
:103F600090E00E9453DABC01C8010E94151F9D8396
:103F70008C83EC81FD81309769F467E577E18EE110
:103F80009CE00E94D48A8EE19CE00E943E8990E0F1
:103F900080E058C085E2DF011D928A95E9F7EC8147
:103FA000FD8116A2EC81FD8115A2EC81FD8117A295
:103FB0000C811D8180E00E941618F80160A771A78E
:103FC00082A793A78E81811116C062E00E9483AB05
:103FD0006EE177E184E19CE00E94D48A84E19CE078
:103FE0000E943E8988E29CE00E94888010922A020A
:103FF00081E080932608EF81F885A089B18982E06D
:104000008C93A485B5851C92A685B7858FEC8C937F
:10401000108EA489B58986E08C93A289B3898C918E
:1040200088698C930288F389E02D80818F7D80835D
:10403000E881F9810684F785E02D62E0CE011995CB
:1040400081E090E0DF91CF911F910F910895CF9281
:10405000DF92EF92FF920F931F93CF93DF93EC01C8
:104060006A017B018E819F81892BA9F488819981C6
:104070000E94BC9F082F10E00530110564F40E94D7
:104080004AA39F838E83BC01888199810E942CA3BF
:104090000F5F1F4FF1CFEE81FF81309749F180858F
:1040A000982F9F7019F5807F82608087EE81FF8155
:1040B000C186D286E386F48667EB77E085EC9CE0E8
:1040C0000E94D48A2AE030E0B701A60185EC9CE08A
:1040D0000E94E48985EC9CE0DF91CF911F910F91C4
:1040E000FF90EF90DF90CF900C943E899230F1F2E8
:1040F000DF91CF911F910F91FF90EF90DF90CF90C4
:1041000008958F929F92AF92BF92CF92DF92EF92DB
:10411000FF920F931F93CF93DF93EC0188819981D6
:104120000E94BC9F082F10E00430110554F40E9437
:104130004AA3BC01888199810E942CA30F5F1F4F65
:10414000F3CF60E0888199810E94A59F7C01009750
:1041500051F1FC0180858F70843039F5C184D2849F
:10416000C114D10401F1F60180818823E1F08DEFC3
:10417000882E8AE0982EB12CA12C1A2DC4010E9401
:104180009CDCAC01B401C6010E94B5DC892B09F4AA
:1041900013C1FFEFAF1ABF0A89E0880E911CE7E157
:1041A000AE16B10451F71FEF03C08230E1F711855D
:1041B0001887C880D98061E0C6010E94A59F7C0154
:1041C0009B838A8362E0C6010E94A59F9D838C83A6
:1041D00064E0C6010E94A59F6C019F838E831A3004
:1041E000D1F1103109F475C0133021F58AE090E067
:1041F0000E9453DA8C01FC01D383C28385EA92E0EA
:104200009183808370E060E0CE010E94281C97FDBE
:104210001EC0F80195838483CE010E94111CF80111
:10422000978386838DEC92E091838083118610863C
:104230001A870987DF91CF911F910F91FF90EF901F
:10424000DF90CF90BF90AF909F908F900895919501
:1042500081959109DECF89E090E00E9453DA8C01CC
:10426000FC01D383C2838FE792E091838083C114E2
:10427000D10419F1F60180858F708230F1F48681C6
:104280009781F8019583848382E399E090878783FF
:10429000CE010E94111C892B59F270E060E0CE0122
:1042A0000E94281CF8018683813081F048F082301A
:1042B00009F0BECF8FEC99E005C090E080E0E1CF3F
:1042C00088E29CE0F80190878783B2CF8CE69AE081
:1042D000F9CF8BE090E00E9453DA8C01FC01D3838C
:1042E000C28385EF92E091838083168270E060E064
:1042F000CE010E94281C97FD41C0F801958384835C
:10430000F80184819581009719F0863591052CF08C
:1043100080E290E0F80195838483E114F104F1F1E7
:10432000F70180858F708530C9F5C7010E94BC9F59
:104330008230A0F161E0C7010E94A59FFC01892B9A
:1043400069F180858F70823011F561857285838572
:1043500094850E9488E220E030E04AE754E40E941D
:10436000E7E20E9446E56115710581059105D1F0EE
:10437000F80167837087818792875ACF91958195DD
:104380009109F8019583848381E08683B9CF8330D6
:1043900029F46185728583859485DDCF60E070E0C6
:1043A000CB01D9CF88E893E1A0E0B0E0F8018783A2
:1043B0009087A187B2873CCFC6010E94088F8A2DC3
:1043C00090E0B0E0A0E0F70181879287A387B487EF
:1043D0008085807F82608087EBCECF93DF93EC0176
:1043E000798368831A8619861B861C8E1B8E0E9411
:1043F0002914882329F0CE01DF91CF910C948120DC
:10440000DF91CF9108951F93CF93DF93FC01162F77
:10441000C389D489818992899C012F5F3F4F328B58
:10442000218BC80FD91FCE010E94A5E3181721F0D8
:10443000612FCE010E94ADE381E090E0DF91CF914A
:104440001F910895FC018189928924853585821701
:10445000930740F423893489820F931F0E94A5E3B8
:1044600090E008958FEF9FEF08952F923F924F9223
:104470005F926F927F928F929F92AF92BF92CF92F4
:10448000DF92EF92FF920F931F93CF93DF93CDB7FD
:10449000DEB762970FB6F894DEBF0FBECDBF5C01EA
:1044A0004B0129013A01CA01B9010E943FE51B01F4
:1044B0003F926F9387EB94E09F938F93CE01019689
:1044C0007C019F938F930E9428E90F900F900F908B
:1044D0000F900F900F9020E030E0A901C301B201CE
:1044E0000E9475E5181624F077FA709477F87094A6
:1044F000F70101900020E9F731976F01CE18DF082E
:104500008EE28083A2E0B0E0AC0FBD1FAC0DBD1DFC
:10451000BA8BA98BB10137FE03C071956195710902
:10452000072E000C880B990B0E9488E29B01AC01BE
:10453000C301B2010E9460E420E030E040E251E4B7
:104540000E94E7E20E943FE5605DE989FA896083A5
:10455000FE01EC0DFD1D1382D501ED91FC91048847
:10456000F589E02D9801A701B401C501199562965E
:104570000FB6F894DEBF0FBECDBFDF91CF911F9174
:104580000F91FF90EF90DF90CF90BF90AF909F90F2
:104590008F907F906F905F904F903F902F900895F5
:1045A000DA01E0912508F0E0FE2FEE27E60FF71F75
:1045B00090E0982F8827A901BD018E0F9F1F0C94B2
:1045C0009194CF93DF931F92CDB7DEB7209125084A
:1045D00030E0322F2227260F371F90E0982F8827B0
:1045E000498341E050E0BE016F5F7F4F820F931F10
:1045F0000E9491940F90DF91CF910895CF93DF9314
:104600001F92CDB7DEB741E050E0BE016F5F7F4F34
:104610000E94069489810F90DF91CF910895209197
:10462000250830E0322F2227620F731F90E0982F69
:104630008827860F971F0C94FE2263E070E00C948D
:104640000F239F92AF92BF92CF92DF92EF92FF9291
:104650000F931F93CF93DF93EC017B0180911E0991
:10466000811121C01B821A8288EE93E0A0E0B0E0A5
:104670008C839D83AE83BF8382EE93E0998388838E
:1046800088E08C8788EE93E09E878D87CE01DF914E
:10469000CF911F910F91FF90EF90DF90CF90BF903F
:1046A000AF909F90089534E0932E833311F028E06B
:1046B000922E8EE0C82E89E0D82E10E098E0B92E18
:1046C000A12CD6012D913D916D01F7018481958139
:1046D0002817390791F4812F0E94DA98082F873123
:1046E00011F08C3139F5812F0E94C697892B59F52D
:1046F0000C3119F4812F0E94BE981F5F9112E1CFF7
:10470000A11008C0D701ED91FC910084F185E02D46
:10471000C70119951B821A8288EE93E0A0E0B0E0F1
:104720008C839D83AE83BF8382EE93E099838883DD
:10473000BC86A8CF843149F08111DFCFF6013297D2
:1047400011821082DACFB12ED8CFAA24A394D5CF6C
:104750008F929F92AF92BF92CF92DF92EF92FF9291
:104760000F931F93CF93DF93CDB7DEB72F970FB67D
:10477000F894DEBF0FBECDBF5C014B017A01809182
:104780001E098823C9F104E0833309F008E0B5016C
:10479000CE0101960E9421238EE0C82E89E0D82EFA
:1047A00010E0F601219131916F01F501848195812D
:1047B0002817390751F4812F0E94DA98873129F49C
:1047C000A701B401812F0E943C971F5F0113E9CF1D
:1047D000C7012F960FB6F894DEBF0FBECDBFDF9195
:1047E000CF911F910F91FF90EF90DF90CF90BF90EE
:1047F000AF909F908F900895F12CE12CE9CFDA01D2
:10480000E0912508F0E0FE2FEE27E60FF71F90E07D
:10481000982F8827A901BD018E0F9F1F0C94069425
:1048200044E050E0BC018FE090E00C94919444E0AF
:1048300050E0BC0185E090E00C94919444E050E09D
:10484000BC0181E090E00C94919408959F92AF9206
:10485000BF92CF92DF92EF92FF920F931F93CF936D
:10486000DF938C015B01942EE52EFC01C688D7886E
:10487000F08C80E591E00E94D5A78F2D0E94E296F2
:10488000C92DDE2D8C179D0708F4EC019E01A501B2
:10489000B6018F2D0E945F96F801868997898C0F4B
:1048A0009D1F978B868BCE01DF91CF911F910F912A
:1048B000FF90EF90DF90CF90BF90AF909F900895C2
:1048C000CF93FC01C08D80E591E00E94D5A760E206
:1048D00070E08C2F0E94F69362E070E08C2F0E94B3
:1048E0000F2384FD16C062E070E08C2F0E940F231E
:1048F00083FF0AC048E162E070E08C2F0E94E12251
:1049000080E090E0CF91089580E591E00E94D5A7E6
:10491000E3CF40E162E070E08C2F0E94E12281E071
:10492000F0CFFF920F931F93CF93DF93EB01FC0126
:10493000178A168A2A81211109C02B81211106C0EC
:104940002C81211103C02D81222301F14115510534
:10495000E9F08A01FC01F08C80E591E00E94D5A786
:10496000AE014E5F5F4F24E030E06CE070E08F2DD1
:104970000E94D022B8018F2D0E94E99881E090E03A
:10498000DF91CF911F910F91FF90089580E0F7CFB5
:104990000F931F93CF938C01FC016481758181E299
:1049A0000E941599C82F8830F8F480E591E00E94A4
:1049B000D5A78C2F0E941D23833131F08C2FCF91EE
:1049C0001F910F910C94BE9862E070E08C2F0E94B2
:1049D000F693F80184819581EC2FF0E0EE0FFF1F34
:1049E000E25FF64F91838083CF911F910F910895DD
:1049F0000F931F93CF93DF931F921F92CDB7DEB714
:104A0000FC0124852830E0F48C0180E591E00E94CF
:104A1000D5A722E030E0AE014F5F5F4F60E170E06C
:104A2000F80184850E94FF2389819A81982789272C
:104A300098270F900F90DF91CF911F910F910895BC
:104A400090E080E0F6CF0F931F93CF93DF931F92F8
:104A50001F92CDB7DEB7FC0124852830E0F48C012D
:104A600080E591E00E94D5A722E030E0AE014F5FE3
:104A70005F4F64E070E0F80184850E94FF23898124
:104A80009A819827892798270F900F90DF91CF91CF
:104A90001F910F91089590E080E0F6CFCF93DF93C0
:104AA000EC0184E694E0998388831A821B821C823D
:104AB0001D8280E591E00E94D5A7BE016E5F7F4F09
:104AC00044E050E08FE090E00E940694CE01DF9138
:104AD000CF9108950E945295882331F080911E094C
:104AE000843329F0873381F090E080E0089580E5F9
:104AF00091E00E94D5A785E390E00E94FE2285FD0B
:104B00000DC082E090E0089580E591E00E94D5A775
:104B10008EE290E00E94FE2280FFF3CF81E090E0E1
:104B200008951F920F920FB60F9211240BB60F9299
:104B30002F933F934F935F936F937F938F939F93A5
:104B4000AF93BF93EF93FF938091B900887F803636
:104B500009F44DC008F040C0883209F4A7C028F518
:104B6000803109F49BC0C8F4882309F4F1C088306F
:104B700009F494C0FF91EF91BF91AF919F918F91F4
:104B80007F916F915F914F913F912F910F900BBE4D
:104B90000F900FBE0F901F901895883109F486C0B2
:104BA000803241F780931E0814C0803409F497C006
:104BB00040F48033B9F38833E9F680931E0885EC1E
:104BC000A8C0803509F481C0883509F490C08834C4
:104BD00089F60E949111CECF883909F486C038F544
:104BE000883729F050F4883611F0803719F683E0C1
:104BF00080931F0810921D0855C0883809F475C0AD
:104C0000803919F0803809F0B5CF80911D088032C5
:104C100008F06BC0E0911D0881E08E0F80931D08A5
:104C20008091BB00F0E0E350F84F80833BC0803BB5
:104C300039F0D0F4803A09F471C0883A09F09ACF7B
:104C400084E080931F081092FC071092FB07F0E0AD
:104C5000E0E019958091FB0781110FC081E08093FE
:104C6000FB071092DB0709C0803C09F4A8CF883C01
:104C700009F4A5CF883B09F07DCFE091FC0781E0E6
:104C80008E0F8093FC07F0E0E552F84F808180930F
:104C9000BB009091FC078091FB0725C08091240800
:104CA0008093BB0085EC8093BC0064CF9091230877
:104CB00080912208981728F5E091230881E08E0F53
:104CC00080932308F0E08081EBCFE091230881E01E
:104CD0008E0F809323088091BB00F0E08083909139
:104CE0002308809122089817E8F285E8DCCFE0914C
:104CF000230881E08E0F809323088091BB00F0E0B1
:104D0000808380912108811164CF81E08093200805
:104D100084EA8093BC0010921F082CCF85EC80930E
:104D2000BC0010921F0880911D08803230F4E09181
:104D30001D08F0E0E350F84F108260911D0870E00C
:104D40008DEF97E0F0E0E0E0199510921D0812CF8A
:104D500010921E083ECF4F925F926F927F92AF9259
:104D6000BF92CF92DF92EF92FF920F931F93CF9358
:104D7000DF9300D01F92CDB7DEB72B013C01298312
:104D80003A834B835C83A6019501C801B701640D8A
:104D9000751D861D971D211531054105510511F021
:104DA0000E94CBE329813A814B815C8162177307B2
:104DB00084079507D0F4241535054605570530F5C9
:104DC00021E0822F0F900F900F900F90DF91CF91E5
:104DD0001F910F91FF90EF90DF90CF90BF90AF9019
:104DE0007F906F905F904F90089546165706680623
:104DF000790650F421E089819A81AB81BC818415C8
:104E00009505A605B705E8F220E0DBCF21E04616C0
:104E1000570668067906A8F2F7CF6F927F928F92B5
:104E20009F92AF92BF92CF92DF92EF92FF920F9339
:104E30001F93CF93DF93EC018C819D81892B09F423
:104E4000A8C08A819B81892B09F4A3C03A014B0138
:104E5000E881F9810484F585E02DCE011995039749
:104E600001F5EC81FD8180A591A5A2A5B3A5892BB3
:104E70008A2B8B2BB1F00E940DAD9B01AC01EC8114
:104E8000FD8160A571A582A593A5A12CB12C65011A
:104E900016E9E12EF12C00E010E00E94AB268823F9
:104EA00001F38F81988521E0621A7108DC01ED9190
:104EB000FC910280F381E02DA301B40119958F814B
:104EC0009885DC01ED91FC910190F081E02DD401F9
:104ED000129660E09D01281939092615370518F446
:104EE0002D91620FF7CF19950C811D8180E00E94F2
:104EF0001618F80160A771A782A793A769E177E167
:104F000085EC9CE00E94D48A4AE050E06E8185ECFA
:104F10009CE00E94428965E177E185EC9CE00E947B
:104F2000D48A8401C8018819990986159705B8F4AF
:104F3000D8016C9140E150E06A3050F466E674E0CC
:104F400085EC9CE00E946E8A40E150E0F8016081AF
:104F500085EC9CE00E9442890F5F1F4FE3CF85ECF8
:104F60009CE00E943E89E881F9810684F785E02D66
:104F700063E0CE01DF91CF911F910F91FF90EF90F1
:104F8000DF90CF90BF90AF909F908F907F906F9069
:104F90001994DF91CF911F910F91FF90EF90DF90C7
:104FA000CF90BF90AF909F908F907F906F9008951B
:104FB0008F929F92AF92BF92CF92DF92EF92FF9229
:104FC0000F931F93CF93DF937C014A015901C09146
:104FD000D807D091D907062F660F110B209709F437
:104FE0005CC088858F70863009F055C068E674E033
:104FF000CE010E942D9F6C0182E08816910449F039
:105000006DE674E0E3E08E16910429F0D0E0C0E094
:1050100006C061E774E0CE010E942D9FEC01C1142F
:10502000D104D9F1F60180858F708430B1F56185A6
:105030007285A801C7010E94D1E8A80166E774E063
:10504000C7010E94B3E8209779F188858F7084307A
:1050500059F569857A85A801C7010E94B3E8A801BE
:1050600066E774E0C7010E94B3E8A114B10429F017
:10507000A801B501C7010E94B3E8C701DF91CF9134
:105080001F910F91FF90EF90DF90CF90BF90AF9066
:105090009F908F900895D0E0C0E0A8016BEC78E17C
:1050A000C7010E94C3DCC9CFF2E08F16910481F0E2
:1050B00083E08816910429F06091270870912808F0
:1050C000CACFA80165EC78E1C7010E94A5DCC7CF73
:1050D000A80162EC78E1F8CFCF92DF92EF92FF92D5
:1050E0000F931F93CF93DF93CDB7DEB7C154D10990
:1050F0000FB6F894DEBF0FBECDBF6C01AB0130E040
:1051000020E060E4CE0101967C010E94D827F701DF
:1051100001900020E9F731978F010E191F09A801AE
:10512000B701C6010E94C3E8892B11F010E000E02E
:10513000C801CF5BDF4F0FB6F894DEBF0FBECDBF07
:10514000DF91CF911F910F91FF90EF90DF90CF9063
:105150000895CF92DF92EF92FF920F931F93CF9318
:10516000DF93CDB7DEB7C054D1090FB6F894DEBFD8
:105170000FBECDBF8091340890913508059709F492
:1051800049C06115710509F445C069017A018B01B7
:1051900040E450E0CE0101960E94D1E86FE270E059
:1051A000CE0101960E9498E8892B41F4980143E0D2
:1051B00050E060E4CE0101960E94D8274FE350E012
:1051C000B601CE0101960E94B3E80E944B9F88234E
:1051D00009F180913408909135080697D9F48091AF
:1051E0003009811117C0B701CE0101960E94DBADD5
:1051F00081E090E0C05CDF4F0FB6F894DEBF0FBED9
:10520000CDBFDF91CF911F910F91FF90EF90DF9075
:10521000CF90089590E080E0EDCFEF92FF920F9352
:105220001F93CF937C018C01C0E0C330E1F0F80103
:10523000428150E070E060E02AE030E084E19CE0F0
:105240000E94E48960EC78E184E19CE00E94D48AC9
:10525000CF5F0F5F1F4FC43041F7CF911F910F9168
:10526000FF90EF900895F701458150E070E060E015
:105270002AE030E084E19CE00E94E4896EEB78E172
:10528000E3CFCF93DF931F921F92CDB7DEB780910C
:10529000D70D9091D80D009711F483EE9DE0BE01DB
:1052A0006F5F7F4F681B790B072E000C880B990BE3
:1052B0000F900F90DF91CF9108954F925F926F9270
:1052C0007F929F92AF92BF92CF92DF92EF92FF9226
:1052D0000F931F93CF93DF93CDB7DEB760970FB6D1
:1052E000F894DEBF0FBECDBFFC0119861A861B865F
:1052F0001C869A859F7090669A87A081B1811097CD
:1053000009F4EEC08C91882309F4EAC00081118170
:10531000D8019C91992309F466C09D3209F4E4C038
:1053200090539A3028F00F5F1F4F11830083EECF08
:10533000C801912CDC016D01C81AD90A2D91022EE9
:10534000000C330B205331092A303105A0F37F01C3
:105350006EE270E0C8010E9498E8FC01DC01892B34
:1053600009F045C0C8010E943EDC2A852F70206AE2
:105370002A872B013C016CE270E0D7018D919C9152
:105380000E9498E8009709F0A6C0F70111821082E8
:105390004D865E866F86788A88E0FE013996DE014A
:1053A000119601900D928A95E1F729813A814B81FE
:1053B0005C816D817E818F81988560960FB6F894AF
:1053C000DEBF0FBECDBFDF91CF911F910F91FF9038
:1053D000EF90DF90CF90BF90AF909F907F906F90B5
:1053E0005F904F900895912CD12CC12CB0CF5D01CE
:1053F000AE1ABF0A11968C911197082E000C990BCA
:10540000C09711960A9798F32181022E000C330B56
:10541000205331092A30310508F050C02A303105B7
:1054200014F029E030E037FF02C030E020E0032E26
:10543000000C440B550BAAE0B0E00E940CE42B01D9
:105440003C018281082E000C990BC0978A3091058F
:1054500088F48A30910514F089E090E097FF02C04B
:1054600090E080E0092E000CAA0BBB0B480E591EE1
:105470006A1E7B1EA114B10409F474CFC801B3E005
:10548000AB16B104FCF4E8E0CE16D104DCF40E94C3
:105490003EDC9B01AC01A4E6B0E00E940CE4992044
:1054A00041F07094609450944094411C511C611CD4
:1054B000711C460E571E681E791E5DCF20E030E03D
:1054C000A901B9CF0E941CDC2B013C018A858F7099
:1054D00080678A8750CF0196D7018D939C9358CFD0
:1054E000412C512C320154CFC80101969924939438
:1054F00021CFCF92DF92EF92FF920F931F93CF9322
:10550000DF93EC01A881B981109781F18C918823F8
:1055100069F108811981F8019081992351F09D3238
:1055200041F090539A3028F00F5F1F4F1983088382
:10553000F0CFC8010E943EDC6B017C016CE270E0A0
:10554000C8010E9498E8009769F419821882C7017F
:10555000B601DF91CF911F910F91FF90EF90DF90F7
:10556000CF900895019699838883F1CFC12CD12CD7
:105570007601EDCF67EE75E184E19CE00E94D48A6C
:1055800064ED75E184E19CE00E94D48A66EC75E1EB
:1055900084E19CE00E94D48A6EEB75E184E19CE09A
:1055A0000E94D48A84E19CE00E943E896EEA75E103
:1055B00084E19CE00E94D48A62EA75E184E19CE087
:1055C0000E94D48A65E975E184E19CE00E94D48A56
:1055D00060E875E184E19CE00E94D48A61E775E1AE
:1055E00084E19CE00E94D48A69E675E184E19CE054
:1055F0000E94D48A6EE575E184E19CE00E94D48A21
:1056000061E575E184E19CE00E94D48A67E475E17C
:1056100084E19CE00E94D48A6FE375E184E19CE020
:105620000E94D48A63E375E184E19CE00E94D48AFD
:1056300069E175E184E19CE00E94D48A6AEF74E13B
:1056400084E19CE00E94D48A65EE74E184E19CE0F0
:105650000E94D48A6DEC74E184E19CE00E94D48ABB
:105660006FEB74E184E19CE00E94D48A63EB74E107
:1056700084E19CE00E94D48A6BEA74E184E19CE0BE
:105680000E94D48A60EA74E184E19CE00E94D48A9A
:1056900063E974E184E19CE00E94D48A6BE874E1E0
:1056A00084E19CE00E94D48A60E874E184E19CE09B
:1056B0000E94D48A61E774E184E19CE00E94D48A6C
:1056C00068E674E184E19CE00E94D48A6AE574E1B2
:1056D00084E19CE00E94D48A6CE474E184E19CE063
:1056E0000E94D48A84E19CE00C943E890F931F931E
:1056F000CF93DF9300D000D0CDB7DEB70E94BA2A97
:1057000064E47FE084E19CE00E94D48ACE010196AB
:105710000E944E25CE0101960E940D2904E614E058
:105720001A8309838091300B9091310BA091320B39
:10573000B091330B8B839C83AD83BE83CE010196E6
:105740000E940D291A8309831B821C821D821E82DE
:1057500080E591E00E94D5A744E050E0BE016D5F76
:105760007F4F81E090E00E940694CE0101960E9456
:105770000D291A8309831B821C821D821E8280E5EB
:1057800091E00E94D5A744E050E0BE016D5F7F4FDD
:1057900085E090E00E940694CE0101960E940D29BA
:1057A0006AE67FE084E19CE00E94D48A88EC90E085
:1057B00026960FB6F894DEBF0FBECDBFDF91CF9116
:1057C0001F910F910895009789F0FC0120852F709B
:1057D000253061F40E94A59F009741F0FC012085CF
:1057E0002F70243019F481859285089590E080E02F
:1057F0000895CF92DF92EF92FF920F931F93CF9372
:10580000DF9300D000D0CDB7DEB78091D7078111EC
:105810009AC0809134089091350802970CF493C097
:105820008091830790918407009709F48CC06AE700
:1058300074E00E942D9F8C01009709F484C00E949F
:10584000BC9FE82EF12CE114F10409F47CC070E057
:1058500060E0C8010E94E32B6C01EA94EF2809F490
:1058600081C061E0C8010E94A59FFC0101851285ED
:10587000CE0101960E944E25CE0101960E94D8A726
:1058800062E27EE084E19CE00E94D48AB60184E179
:105890009CE00E946E8A61E874E084E19CE00E94D2
:1058A0006E8AB80184E19CE00E94B49F61E874E0D4
:1058B00084E19CE00E946E8A6FE179E084E19CE0E3
:1058C0000E946E8A84E19CE00E943E8962E072E060
:1058D00083EE9CE00E940417D092D90CC092D80CA1
:1058E0001093DB0C0093DA0C8FE199E0892BE9F53A
:1058F00088E794E09093DD0C8093DC0C80912C0879
:1059000090912D08009741F070E060E00E94E32B39
:105910009093280880932708809127089091280861
:10592000009731F19093DF0C8093DE0C1092E10C24
:105930001092E00C81E08093D70769E07EE084E17B
:105940009CE00E94D48A26960FB6F894DEBF0FBE64
:10595000CDBFDF91CF911F910F91FF90EF90DF901E
:10596000CF90089502E012E083CF8FE199E0C2CF9B
:1059700081E693E0892B19F488E794E0D3CF81E6A0
:1059800093E0D0CF0F931F93CF9364E07EE084E148
:105990009CE00E94D48A08EF1BE0C0E0F8018191EE
:1059A0008F01803130F466E674E084E19CE00E946F
:1059B0006E8AC530C9F0F8013197408150E070E03F
:1059C00060E020E130E084E19CE00E94E48962E054
:1059D0007EE084E19CE00E94D48ACF5FC630F1F67D
:1059E000CF911F910F9108954091FD0B50E070E011
:1059F00060E020E130E084E19CE00E94E48984E101
:105A00009CE00E943E89E9CFEF92FF920F931F9393
:105A1000CF93DF9300D000D01F92CDB7DEB77B01CC
:105A2000CE0107969F938F9301979F938F93019732
:105A30009F938F9301979F938F9301979F938F933A
:105A400001979F938F938E010F5F1F4F1F930F93AB
:105A500083E894E09F938F93DB0113968C911397C7
:105A60008F9312968C918F930E9458E90FB6F894F9
:105A7000DEBF0FBECDBF0697ECF466EB72E18EE1A0
:105A80009CE00E94D48AD70112966D917C918EE1A0
:105A90009CE00E946E8A80E991E027960FB6F89408
:105AA000DEBF0FBECDBFDF91CF911F910F91FF9051
:105AB000EF9008958091F00B9091F10B892BA9F153
:105AC0000E940DA0882389F182E70E94F89F8091AF
:105AD000F00B9091F10BDC01ED91FC910088F189C4
:105AE000E02D64E070E019958091F00B9091F10B3E
:105AF000DC01ED91FC910280F381E02D46E050E065
:105B0000B801199586E0F801A8EFBBE001900D926D
:105B10008A95E1F78091F00B9091F10BDC01ED910A
:105B2000FC910488F589E02D19950E94C22C68EC3F
:105B300072E184E19CE00E94D48A88EC90E0ADCFD1
:105B40002F923F924F925F926F927F928F929F928D
:105B5000AF92BF92CF92DF92EF92FF920F93CF93CB
:105B6000DF9300D01F92CDB7DEB77C017A836983C3
:105B70005C834B83DB011C92FC016081662309F48A
:105B80004EC030FF4CC0F9E06F9FB00111246D5B37
:105B90007F4DCD010E94C3DCD70111968C91807F8F
:105BA00041F04B815C8167E974E089819A810E94B0
:105BB000B3E8E981FA8101900020E9F73197298162
:105BC0003A81E21BF30B19012E0E3F1E4B815C81C3
:105BD0004E1B5F0B415051095C834B83D7011196DB
:105BE000EC9111978E2F807F09F4F7C0E295EF704A
:105BF000E150EC3008F0F1C0F0E08827ED5FF14DA6
:105C00008F4F0C9442E4122EB52E222F812F9C2F01
:105C1000602E322F322F322F4E2E362EB82F298063
:105C20003A80DCCFF7018481282F30E050E040E05B
:105C3000002359F030E0A4E6B0E00E941FE42FEF0B
:105C400030E040E050E00E94EDE35F934F933F93DC
:105C50002F9389E994E09F938F93FC81FF932B818D
:105C60002F933F922F920E94EBE8B2C017968C912F
:105C700017978F9316968C9116978F9315968C91F4
:105C800015978F9314968C918F938CE994E09F9342
:105C90008F93BC81BF93EB81EF93E3CF17968C91E9
:105CA00017978F9316968C9116978F9315968C91C4
:105CB00015978F9314968C918F9380EA94E0E7CF99
:105CC0001496CD90DD90ED90FC901797F7FE34C0C0
:105CD00084E6882E912CA12CB12CC701B601A50118
:105CE00094010E94EDE39B01AC0188279927DC0118
:105CF000821B930BA40BB50BBF93AF939F938F9312
:105D000066277727CB016C197D098E099F09A501AC
:105D100094010E94EDE35F934F933F932F9384EAA6
:105D200094E09F938F933C813F934B814F933F929D
:105D30002F920E94EBE84CC0C701B60124E630E088
:105D400040E050E00E94EDE39F938F937F936F9329
:105D50005F934F933F932F9385EA94E09F938F93A4
:105D60009C819F93AB81AF93E2CFC7010E94071440
:105D7000BC01D7011696CC9016971796DC90179712
:105D8000D0FADD24D0F814969C9114971596FC90C7
:105D9000EB80BC80292F30E050E040E077FD35C03B
:105DA000011135C07F936F931F921F921F929F9393
:105DB0001F92FF92DF92CF928EEA94E09F938F938F
:105DC000FC81FF932B812F933F922F920E94EBE84F
:105DD0000FB6F894DEBF0FBECDBF89819A810F90B8
:105DE0000F900F900F90DF91CF910F91FF90EF9058
:105DF000DF90CF90BF90AF909F908F907F906F90EB
:105E00005F904F903F902F900895002361F0292FCD
:105E100030E0A4E6B0E00E941FE42FEF30E040E065
:105E200050E00E94EDE35F934F933F932F931F92B7
:105E3000FF92DF92CF9281EB94E09F938F93BF927A
:105E4000EF9275CF15968C9115971F928F9316969A
:105E50009C91169717968C9181708F939F9384EBEA
:105E600094E015CF14968D909D90AD90BC901797AF
:105E700020E030E0A901C501B4010E9481E22401C3
:105E8000350187FF04C077FA709477F87094C301E6
:105E9000B2010E943FE56B01072E000C880B990BA5
:105EA0000E9488E29B01AC01C301B2010E9460E440
:105EB00020E030E04AE754E40E94E7E20E94CAE5AD
:105EC0000E943FE5062F772E20E030E0A901C501B2
:105ED000B4010E9481E287FF07C07F920F93DF9297
:105EE000CF928AEB94E0D3CE7F920F93DF92CF9242
:105EF0008BEB94E09F938F933C813F934B814F9327
:105F0000B0CE14968C9114971F928F9315968C9106
:105F100015971F928F9316968C911F928F9381EBFA
:105F200094E09F938F93BC81BF93EB81EF933F925B
:105F30002F920E94EBE84CCF17968C9117971F92E7
:105F40008F9314968C9114971F928F9315968C9122
:105F500015971F928F9316968C911F928F938EEAAE
:105F600094E09F938F93BC81BF93EB81EF93DFCE3F
:105F700014966D917C914B815C81C1010E94D1E8A6
:105F80002CCFEF92FF920F93CF93DF93CDB7DEB775
:105F9000A0970FB6F894DEBF0FBECDBF7C0100E026
:105FA00020E033E040E250E0BE016F5F7F4F0E948F
:105FB000A02DBE016F5F7F4F85EC9CE00E946E8A32
:105FC00061E77CE085EC9CE00E94D48AF701618166
:105FD00062956F704AE050E085EC9CE00E94428937
:105FE0006AE67CE085EC9CE00E94D48AF70161813E
:105FF0006F704AE050E085EC9CE00E94428985EC9D
:106000009CE00E943E89A0960FB6F894DEBF0FBEBA
:10601000CDBFDF91CF910F91FF90EF900895AF9298
:10602000BF92CF92EF92FF920F931F93CF93DF9384
:1060300000D000D01F921F92CDB7DEB75C0109835C
:106040001A832B833C834D835E836F8378876AE951
:1060500078E185EC9CE00E94D48ACE0101960E94F2
:10606000C12FE114F10439F063E978E1C7010E941E
:106070008CDC009721F1F5010281138101151105D6
:10608000E1F0898181115BC08A818F70813009F4D0
:106090005EC038F1823019F1082F10E066E778E130
:1060A00085EC9CE00E94D48AB80185EC9CE00E94BB
:1060B000B49F85EC9CE00E943E8990E080E02896A9
:1060C0000FB6F894DEBF0FBECDBFDF91CF911F9109
:1060D0000F91FF90EF90CF90BF90AF900895CC209C
:1060E000C1F060E0CE0101960E94F312892B09F401
:1060F00047C0C8010E94E51A672B682B692BE1F4A1
:1061000080E00E941618AB01BC01C8010E94272044
:1061100013C0C8010E94321B8E3019F050F4813038
:1061200059F460E0CE0101960E94F312892B21F010
:10613000E0CF83518330A8F381E090E0C0CF80317D
:10614000D0F48E30B0F68130A1F28230C9F066E82A
:1061500078E185EC9CE00E94D48A4AE050E06981B5
:1061600085EC9CE00E94428985EC9CE00E943E897F
:1061700001E010E093CF8351833008F4BACFE7CF2A
:1061800040E050E0BA01C8010E94272060E0C5014C
:106190000E943F1BD1CFCF92DF92EF92FF920F93DD
:1061A0001F93CF93DF936115710509F458C06A01FD
:1061B0007B018C01CB010E942914D82F882371F117
:1061C000D70114968D919C910097E9F1FC01C0854F
:1061D0002C2F2F703EEF320F323010F0211128C0DB
:1061E000C295CF70D0FE59C0C7010E94321BF80182
:1061F0008083CC2351F1C295C07F81818F70C82BE1
:10620000C183D7011496ED91FC9181859285A38578
:10621000B485F80184839583A683B7838D2FDF919E
:10622000CF911F910F91FF90EF90DF90CF90089545
:10623000253049F460E00E94A59F009721F0DC0121
:106240001896CC91CDCFC0E0CDCFD7011496ED916B
:10625000FC9180858F70823021F0833081F0D0E016
:10626000DDCF4185528563857485F80181818F700A
:10627000806A81834483558366837783CFCF41854A
:10628000528563857485F80181818F708067818371
:106290004483558366837783C1CFCC23B1F2C29503
:1062A000C07FF801AACF0F931F93CF93DF9300D045
:1062B00000D01F921F92CDB7DEB719821A821B82BF
:1062C0001C821D821E821F8218862A812F702A83BB
:1062D000FC0102811381C8010E94321B813041F010
:1062E00020F0823011F0853081F490E080E002C02F
:1062F00081E090E028960FB6F894DEBF0FBECDBFC8
:10630000DF91CF911F910F91089540E052E0B801C5
:10631000CE0101960E94CB3060E0CE0101960E9432
:10632000F312E8CFCF93DF9300D000D01F921F92DB
:10633000CDB7DEB7FC01862F8F706181607F682B3F
:10634000618388E0DE01119601900D928A95E1F754
:1063500029813A814B815C816D817E818F81988515
:1063600028960FB6F894DEBF0FBECDBFDF91CF9158
:106370000895CF93DF9300D000D01F921F92CDB726
:10638000DEB7FC01608398E0DE01119601900D926A
:106390009A95E1F729813A814B815C816D817E81FB
:1063A0008F81988528960FB6F894DEBF0FBECDBFBB
:1063B000DF91CF910895DC011196EC911197E29550
:1063C000EF70E150EB3008F037C0F0E08827E4517F
:1063D000FE4C8F4F0C9442E4FE31FE311C32F731FB
:1063E000F7310D32043204320432F731F7311496AA
:1063F0006D917D918D919C911797089514966C9154
:1064000070E090E080E0089514966D917D918D91FB
:106410009C9117970E943FE5089514966D917D9188
:106420008D919C91179724E630E040E050E00E9467
:10643000EDE3CA01B901089560E070E0CB01089571
:10644000CF92DF92EF92FF920F931F93CF93DF9340
:10645000CDB7DEB762970FB6F894DEBF0FBECDBFE3
:106460006C010B871C872D873E874F87588B698B64
:106470007A8B63EE77E1C7010E948CDCEEE0F0E0FE
:10648000892BF1F06DED77E1C7010E948CDCE0E132
:10649000F0E0892BA9F067ED77E1C7010E948CDC61
:1064A000EFE0F0E0892B61F01F7063ED77E1C70149
:1064B0000E948CDCE12FF0E0892B11F4EDE0F0E09C
:1064C0009B85992341F0309731F4EF2809F461C09E
:1064D0008FEF9FEF96C0E131F10508F03CC08827AF
:1064E000EB58FD4C8F4F0C9442E46832C93286322F
:1064F000AB32AB32AB32AB3254339C33AB32AB3218
:10650000AB32AB32AB32A633EF33B433CE010B96A2
:106510000E94DB3120EF260F2931D0F6D6011496E8
:10652000ED91FC91159723A39B01AC0133274427E0
:1065300055271296ED91FC9113970190F081E02D73
:1065400060817181ED91FC910088F189E02D03EC6F
:1065500014E0C6011995D6011496ED91FC9115979A
:10656000118A1496ED91FC91159781E0818714961C
:10657000ED91FC9115978DE482871496ED91FC9135
:1065800015978FE5838714966D917C9145E250E0D5
:1065900033C0F601A481B58191509531E0F6E92F21
:1065A000F0E08827E952FD4C8F4F0C9442E4EC3226
:1065B0001033AB32AB321033EC32AB32AB32AB32E6
:1065C000AB32AB32AB32AB3221333933AB32AB32DD
:1065D000AB3235333133373395968C9195975D9641
:1065E0008C93D6011496ED91FC91858D8160858FF9
:1065F0004DE050E06CE172E0C6010E940D2781E0A1
:1066000090E062960FB6F894DEBF0FBECDBFDF916B
:10661000CF911F910F91FF90EF90DF90CF90089551
:1066200095968C9195975D968C93D6011496ED91E5
:10663000FC91858D8E7F858F4DE050E06FE072E09C
:10664000DBCF57961C92D6011496ED91FC911597CD
:1066500085A1858F1496ED91FC91858D8160858F44
:106660007ACF81E057968C93EECF82E0FBCF84E027
:10667000F9CF83E057968C93D6011496ED91FC9157
:10668000159785A1858F1496ED91FC911597858DB1
:106690008160858F1496ED91FC91818D833009F096
:1066A0005ACF82E0818F57CF1982F601048115817C
:1066B0009031B1F150F49E3091F0CE010B960E94D2
:1066C000DB31D80159966C9314C0913171F192313C
:1066D000A1F782E0F801818F6EEB77E106C083E0DD
:1066E000D80159968C936EEC77E1CE0101960E9409
:1066F00095DCD6011296ED91FC9113970190F081F3
:10670000E02D60817181ED91FC910488F589E02D87
:1067100028EC34E0AE014F5F5F4FC60119951BCFE7
:10672000F801118E69EC77E1E0CF81E0D80159964C
:106730008C9362EC77E1D9CFCE010B960E94DB31CE
:10674000D6011496ED91FC91678B05CFD601149676
:10675000ED91FC91913029F0923009F0FCCE148E2D
:10676000FACE80E5848FF7CEF60104811581913051
:1067700049F09230F1F0CE010B960E94DB31F80126
:10678000638FE9CE83E0D8015B968C93D6010280BB
:10679000F381E02D0190F081E02D60817181ED9118
:1067A000FC910488F589E02D2DEC34E044ED54E0B3
:1067B000B4CFF801138ED6011296ED91FC91139788
:1067C0000190F081E02D60817181ED91FC91048850
:1067D000F589E02D2DEC34E047ED54E09ECFD60155
:1067E0001496ED91FC91913031F0923009F0B3CED6
:1067F000858D877F34CF858D886031CF8F929F9232
:10680000AF92BF92CF92DF92EF920F931F93CF93ED
:10681000DF9300D000D01F921F92CDB7DEB7FC01EE
:1068200009831A832B833C834D835E836F83788730
:10683000808191810097A1F490E080E028960FB6C6
:10684000F894DEBF0FBECDBFDF91CF911F910F91A6
:10685000EF90DF90CF90BF90AF909F908F90089572
:106860008F010E94BC9FC82ED12C86E0C816D1048F
:1068700064F40E944AA3BC01F801808191810E94C6
:106880002CA3FFEFCF1ADF0AF0CF65E0F80180817B
:1068900091810E94A59F8C01892B71F289818031A1
:1068A00058F6CE0101960E94DB311616170618061F
:1068B000190644F4F8018085982F9D70A1F08F701F
:1068C000873089F0F80180858F7080876FEF77E0DF
:1068D00085EC9CE00E94D48A85EC9CE00E943E8975
:1068E00081E090E0ABCF0E940DAD4B015C01CE0189
:1068F00001960E94DB31860E971EA81EB91EF80174
:1069000081869286A386B48682E0E11087E0998131
:106910009295907F892BF801808764EF77E085EC72
:106920009CE00E94D48ACE0101960E94DB31AB012B
:10693000BC012AE030E085EC9CE00E94E4896EEE28
:1069400077E085EC9CE00E94D48AF801418552856D
:10695000638574852AE030E085EC9CE00E94E48940
:10696000BBCFCF93DF93EC016115710539F48F81B3
:1069700081708F8381E0DF91CF9108958981982F75
:1069800092959F7029F180E09430A8F79B01770FD2
:10699000440B550B2959310941095109A4E6B0E0CE
:1069A0000E940CE42BE531E040E050E00E94EDE372
:1069B00037FF02C030E020E02536310514F024E630
:1069C00030E02F5F220F8F818170282B2F83D2CF51
:1069D0008F7080628983DACF2F923F924F925F92BD
:1069E0006F927F928F929F92AF92BF92CF92DF92DF
:1069F000EF92FF920F931F93CF93DF93CDB7DEB744
:106A000068970FB6F894DEBF0FBECDBF1C01098793
:106A10001A872B873C874D875E876F87788B22E1AB
:106A2000E216F10408F035C0F701EF58FC4F308151
:106A3000398BCE0109960E94071497FD04C0BC0152
:106A4000C1010E94B1349A85892F8F70D1011196AE
:106A5000EC911197E07FE82B1196EC9311978985C3
:106A60008C93E295EF70EC3008F063C0F0E088277B
:106A7000E35CFA4C8F4F0C9442E44A376635663536
:106A8000E8364B357637B136F236F236F236B13675
:106A9000B136198ACECFB12C92959F709D3008F0F7
:106AA000C9C4E92FF0E08827E75AFA4C8F4F0C94BD
:106AB00042E49935B037D037B03779377937B037C6
:106AC000B0371A3A1A3AB037B0377D3692959F7080
:106AD0009D3008F022C1E92FF0E08827ED58FA4CEC
:106AE0008F4F0C9442E4993551364536073683353D
:106AF0008035283655368D368D36123612367D362F
:106B00008889F10187838F85D10116968C9316971A
:106B10008E8515968C9315978D8514968C93149766
:106B20009295907F11968C9111978F70982B11965A
:106B30009C93B989BB2309F467C0F10181818295D7
:106B40008F702B2F30E08217130609F45DC061EDC2
:106B50007BE085EC9CE00E94D48AD10111966C9177
:106B600062956F704AE050E085EC9CE00E9442899B
:106B70006EEC7BE085EC9CE00E94D48A4AE050E019
:106B8000698985EC9CE00E9442896CEC7BE085EC95
:106B90009CE00E94D48AF101008119821A821B8232
:106BA0001C821D821E821F82188689898295807FA1
:106BB0009A819F70892B8A830983EE24EA94FE2CA4
:106BC0001181228133814481558166817781CE0193
:106BD00001960E94EC34D1012C9311963C931197AD
:106BE00012964C93129713965C93139714966C938A
:106BF000149715967C93159716968C93169717965F
:106C00009C93C1010E94C12F88E0F10182C18F8550
:106C10009889F1018683878190FB80F987838E852F
:106C2000858387CF8D859E85AF85B8898F3F9105F8
:106C3000A105B10529F024F08FEF90E0A0E0B0E0CD
:106C4000B7FF03C080E090E0DC01F101848371CFE5
:106C50006D857E858F85988924E630E040E050E0A0
:106C60000E94EDE32F3F31054105510529F024F045
:106C70002FEF30E040E050E057FF03C020E030E06D
:106C8000A901D10114962C9354CF8F859889F101D5
:106C90008683878190FB80F987838E8585838D85A8
:106CA000D5CF8D8514968C9344CFCD84DE84EF842C
:106CB000F88820E030E0A901C701B6010E9481E216
:106CC00087FD17C020E030E04FE753E4C701B6016D
:106CD0000E9475E5181634F4C12CD12CAFE7EA2ECA
:106CE000A3E4FA2EC701B6010E9446E5F1016483D0
:106CF00020CFC12CD12C7601F5CFD10111968C91EA
:106D000011978F70806C11968C9311978D859E854D
:106D100015969C938E9314970CCF61E57CE085ECDF
:106D20009CE00E94D48A6A8562956F704AE050E0C8
:106D300085EC9CE00E9442896EE47CE085EC9CE05E
:106D40000E94D48AF101618162956F704AE050E03F
:106D500085EC9CE00E94428985EC9CE00E943E8983
:106D6000E8CE92959F70933091F09C3031F24D8532
:106D70005E856F857889F1014483558366837783C7
:106D80009295907F81818F70982B9183D2CE60E015
:106D9000C1010E94F312D10114968C9314978F8530
:106DA000988916968C93169717968C91179790FB47
:106DB00080F917968C9317978E8515968C93159757
:106DC00011968C9111978F70806211968C93B1CE31
:106DD00060E0CE0109960E94F312D10114968C93C3
:106DE0001497EECF92959F709D3008F066C0E92F02
:106DF000F0E08827E150F94C8F4F0C9442E499352C
:106E00001A374937C736493749370C373937393791
:106E10003937283734377D368D859E85AF85B889DB
:106E2000F10184839583A683B78381818F70806607
:106E300081837FCE6D8570E090E080E00E9486E2E5
:106E4000D10114966D937D938D939C93179771CE7A
:106E50006D857E858F8598890E9488E2F101648323
:106E600075838683978365CE6D857E858F859889AA
:106E7000E5CF9295907FF10181818F70982B91835E
:106E80008D859E85AF85B88984839583A683B783D6
:106E900050CE9295907FD10111968C9111978F7061
:106EA000982B11969C938D859E85AF85B889F101AD
:106EB00084839583A683B7833CCE6CE37CE085EC2A
:106EC0009CE00E94D48A6A8562956F704AE050E027
:106ED00085EC9CE00E94428969E37CE085EC9CE0C3
:106EE0000E94D48AD10111966C912ECFBB24B39409
:106EF000D3CD4D855E856F857889F10144835583B7
:106F0000668377839295907F81818F70982B918390
:106F100088E0DE01119601900D928A95E1F72981B2
:106F20003A814B815C816D817E818F8198856896E5
:106F30000FB6F894DEBF0FBECDBFDF91CF911F918A
:106F40000F91FF90EF90DF90CF90BF90AF909F9008
:106F50008F907F906F905F904F903F902F9008950B
:106F6000963009F43AC148F46D85913071F06FEFB5
:106F700070E0933051F060E008C0973009F439C1F7
:106F80009A506D857E859230B0F784E68F87888928
:106F90008E7F888B1E868A858F7080628A876D8738
:106FA0002E8530E0AFEFB0E00E941FE424E630E031
:106FB00040E050E00E94EDE369017A01FFEFCF1657
:106FC000D104E104F10429F024F0C12CD12C760184
:106FD000CA9486012D852A8B622E712CBB2009F460
:106FE00071C088898695A82FA150BB0B2D01BFEFDA
:106FF0004B165B0609F01EC1003811050CF000C1EC
:107000008FE790E08C199D09869DD001879DB00D7A
:10701000969DB00D11242FEF30E00E9459E421E835
:107020003EE740E050E00E94EDE3F1012783ABE949
:10703000B0E0A70196010E940CE4EFE78E2E912CA0
:10704000A12CB12CA50194010E94EDE389019A01C4
:107050000C591F4F2F4F3F4FAEEFB1E0A7019601E4
:107060000E940CE4A50194010E94EDE3D3010E946B
:107070000CE42FEF30E040E050E00E94EDE33901F6
:107080002FEF6216710421F01CF066246A94712CB3
:107090006CE27CE085EC9CE00E94D48AB80185EC2F
:1070A0009CE00E94B49F6EE17CE085EC9CE00E9435
:1070B000D48AB30185EC9CE00E94B49F85EC9CE0EF
:1070C0000E943E89E5EFFCE1E491F0E0EE0FFF1F46
:1070D000E552F34E85919491EBE4FDE1E4912F8527
:1070E00038893170AFEFBFEF0E941FE42DE631E029
:1070F00040E050E00E94EDE344275527AAEFB5E0B9
:107100000E940CE4DC01CB019058AF4FBF4FCD0182
:10711000BB2797FDB095AB2F8E3FE1E09E0708F0AF
:1071200062C1382F8F3F910508F47FC14EEF481B95
:1071300050E03FEFF301319678012FEFE21AF20AA7
:10714000009510E03E9DC0013F9D900D1124292F18
:107150003327200F311FDF010E9459E44B015C01EE
:107160008824AA24BB245E9D90015F9D300D1124CC
:10717000232F3327200F311F0E9459E4BB27A92F4B
:10718000982F872F882A992AAA2A4E9D90014F9DD1
:10719000300D1124232F3327200F311FDF010E94D0
:1071A00059E4B82FA72F962F882788279927BB2720
:1071B00088299929AA29F101A6839583848362EFFE
:1071C0007BE085EC9CE00E94D48AC1010E94C12F23
:1071D00060E080E00E9483ABACCC6D857E858F85BE
:1071E000988924E630E040E050E00E94EDE3B901E8
:1071F000CCCE6D857E858F8598890E943FE5C5CE72
:10720000A70196012058310941095109ABE9B0E0C5
:107210000E940CE42FE730E040E050E00E94EDE3F4
:1072200089019A010C591F4F2F4F3F4FD1011796DB
:107230001C922ECF9201AAEBBFEF0E9451E444E6CC
:10724000842E912CA12CB12CA50194010E94EDE378
:10725000DA01C9018C599F4FAF4FBF4F8B8B9C8B6D
:10726000AD8BBE8B26E430E0D2010E9459E4A5012B
:1072700094010E94EDE349015A019EE1890E911C9F
:10728000A11CB11C003811050CF093C08FE790E0F1
:107290008C199D09869DD001879DB00D969DB00DDE
:1072A0001124A50194010E9417E49B01AC01AFEFEA
:1072B000B0E00E940CE424E63AE640E050E00E9490
:1072C000EDE3D10117962C932B893C894D895E897A
:1072D0002C0D3D1D4E1D5F1DAEEFB1E00E940CE474
:1072E00023EE30E040E050E00E94EDE329013A0156
:1072F000388F2F8BAFEFB0E0A70196010E940CE40E
:107300002FE730E040E050E00E94EDE38901EA8998
:10731000AE2FB0E0A30192010E940CE42FEF30E009
:1073200040E050E00E94EDE339012F3F310521F0AC
:107330001CF066246A94712C68E17CE085EC9CE08A
:107340000E94D48A2AE030E04B895C896D897E896D
:1073500085EC9CE00E94E48962E17CE085EC9CE0A5
:107360000E94D48A2AE030E0B501A40185EC9CE0BB
:107370000E94E4896AE07CE085EC9CE00E94D48A6B
:10738000B80185EC9CE00E94B49F62E07CE085EC53
:107390009CE00E94D48AB30185EC9CE00E94B49FDB
:1073A00069EF7BE085EC9CE00E94D48A6F89788D40
:1073B00081CEA70196012058310941095109ABE955
:1073C000B0E00E940CE42FE730E040E050E00E9483
:1073D000EDE389019A010C591F4F2F4F3F4FD10107
:1073E00017961C92A9CF8C3FF3E09F0768F48D3F5E
:1073F00022E0920728F452E0580F3FEF40E09ACE87
:107400003CEF381B5FEFFACF8A3F35E0930781F0FE
:107410008B3FE4E09E0728F444E0480F5FEF30E044
:1074200089CE5AEF581B30E001C050E04FEF82CEBA
:1074300050E0F9CF60EE7BE085EC9CE00E94D48ABE
:107440006A8562956F704AE050E085EC9CE00E948E
:1074500042896DED7BE042CDAF92BF92CF92DF9239
:10746000EF92FF920F931F93CF93DF93CDB7DEB7C9
:1074700068970FB6F894DEBF0FBECDBFFC01098B35
:107480001A8B2B8B3C8B4D8B5E8B6F8B788F828115
:107490009381009709F49FC024813581232B09F43F
:1074A0009AC0CC2009F497C06F0170E060E00E94A0
:1074B000281C192FD601ED91FC91068CF78DE02D3B
:1074C000C60119955C018230910509F478C00397D3
:1074D00009F447C095E0F1E0AF16B10409F091E07E
:1074E00019861A861B861C861D861E861F86188A8C
:1074F0009295907F8A858F70892B8A87EE24EA94F3
:10750000FE2C09891A892B893C894D895E896F89EE
:10751000788DCE0109960E94EC34F1E0AF16B104EB
:1075200009F44FC082E0A816B10409F045C06F8588
:1075300070E0D60114968C910E94BFAB61E070E0C0
:10754000C6010E94531C6E8570E00E94BFAB62E0D2
:1075500070E0C6010E94531C6D8570E00E94BFABB5
:107560002BC0612F661F6627661FCE0141960E94C1
:10757000F3125C01BC01D60114968C910E94BFAB42
:107580006EE078E185EC9CE00E94D48AF60164818B
:10759000758185EC9CE00E94B49F6CE078E185ECFD
:1075A0009CE00E94D48AB50185EC9CE00E94B49FC7
:1075B00085EC9CE00E943E8981E090E00EC094E062
:1075C0008FCF63E070E0C6010E94531C688970E0B1
:1075D0000E94BFABACCF90E080E068960FB6F89405
:1075E000DEBF0FBECDBFDF91CF911F910F91FF90F6
:1075F000EF90DF90CF90BF90AF900895FC01918104
:10760000892F82958F7021F0823029F080E00895D3
:107610009F70906291839B0177FF02C030E020E071
:107620002E3681E0380714F02DE631E0268387817D
:1076300030FB80F9878381E008950F931F93CF93E8
:10764000DF938C01FC01C081D1816FE270E0CE013B
:107650000E94E0E80097D9F0FC011192CF010E944E
:10766000D019EC0163EC77E085EC9CE00E94D48AB1
:10767000BE0185EC9CE00E94B49F85EC9CE00E94DA
:107680003E89CE01DF91CF911F910F910895CE01D8
:107690000E94D019EC01892BA1F3F801118210820C
:1076A000F0CF8F929F92AF92BF92CF92DF92EF92E4
:1076B000FF920F931F93CF93DF93CDB7DEB76797FA
:1076C0000FB6F894DEBF0FBECDBF8C017B014C011D
:1076D0008BE0880E911C9F8A8E8AF8011286118693
:1076E0001386148E138E672B09F463C0A09036089E
:1076F000B0903708A114B10409F45BC06FE270E0E8
:10770000C7010E9498E86C01892B09F44AC0F7016F
:10771000DE01119690E080E0BD012191222341F02D
:107720002F3231F08431910519F02D930196F5CF68
:10773000860F971FFC011082C5010E942D9FF80142
:1077400091838083B6016F5F7F4F4FE050E0C401AB
:107750000E94D1E8CE0146960E941D3BF801948F0D
:10776000838F8E899F89892B09F41386C8010E9413
:107770002914882319F0C8010E94812067960FB64A
:10778000F894DEBF0FBECDBFDF91CF911F910F9157
:10779000FF90EF90DF90CF90BF90AF909F908F9031
:1077A0000895B701C5010E942D9FF8019183808340
:1077B000DDCFF80111821082D9CF8F929F92AF92C4
:1077C000BF92CF92DF92EF92FF920F931F93CF93CE
:1077D000DF93CDB7DEB7CD55D1090FB6F894DEBF34
:1077E0000FBECDBF8C016B016115710519F04115FC
:1077F0005105D1F460E07EE085EC9CE00E94D48AE3
:1078000067EF7DE085EC9CE00E94D48AB80185ECAE
:107810009CE00E946E8A65EF7DE085EC9CE00E9412
:10782000D48A85EC9CE030C0460F571FDA011C92C9
:107830000E9441294B0163EF7DE085EC9CE00E94B2
:10784000D48AB40185EC9CE00E94B49F60EF7DE097
:1078500085EC9CE00E94D48AB80185EC9CE00E94F3
:107860006E8A6DEE7DE085EC9CE00E94D48ABAE3DE
:107870008B16B1E09B06F4F460EE7DE08EE19CE0B7
:107880000E94D48A8EE19CE00E943E89C35ADF4F59
:107890000FB6F894DEBF0FBECDBFDF91CF911F9121
:1078A0000F91FF90EF90DF90CF90BF90AF909F909F
:1078B0008F9008956EED7DE085EC9CE00E94D48A67
:1078C000B60185EC9CE00E946E8A6CED7DE085EC53
:1078D0009CE00E94D48A85EC9CE00E943E891A823A
:1078E0001982FE0133968EE3DF011D928A95E9F736
:1078F0008091340890913508059791F563E070E028
:10790000C8010E946C287C01892BE9F5E0913A0BB3
:10791000F0913B0B808180FFB9CF61E070E0C8013E
:107920000E946C28892B09F4B1CF64E270E0C80191
:107930000E94E0E8892B09F0A9CF64EC7DE085EC9A
:107940009CE00E94D48AB80185EC9CE00E946E8A7B
:1079500085EC9CE00E943E89C8010E94C1A996CF97
:1079600061E070E0C8010E946C287C01892B21F540
:1079700062E070E0C8010E946C287C0169EB7DE048
:10798000892B09F44ACFE00EF11E60EB7DE0C701C0
:107990000E948CDC892BC1F4F60101900020E9F7EC
:1079A0003197EC19FD09329778F0C8010E94C1A9FE
:1079B000C6010E94448E6ACF4FE350E0B801CE0169
:1079C00001960E94D1E8DFCF64E270E0C8010E9416
:1079D000E0E8892B09F05ACFB701CE018F5B9F4FAA
:1079E0000E94513BCE018F5B9F4F0E942914882338
:1079F00039F1B601CE018F5B9F4F0E94ECA31816A0
:107A00001906F4F489818823D9F080913408909183
:107A100035080597A9F068E97DE085EC9CE00E94B7
:107A2000D48ABE016F5F7F4F85EC9CE00E946E8A16
:107A300085EC9CE00E943E89CE0101960E94C1A97E
:107A4000CE018F5B9F4F0E945F1420CFCF92DF92B9
:107A5000EF92FF926A017B0163E0FC0180819181DA
:107A60000E94A59FFC01892BA9F080858D7091F45F
:107A7000C094D094E094F094CC24CA9481859285EB
:107A8000A385B4858C219D21AE21BF21818792875A
:107A9000A387B487FF90EF90DF90CF900895CF92A7
:107AA000DF92EF92FF926A017B0163E0FC0180812B
:107AB00091810E94A59FFC01892BA9F09085892FB7
:107AC0008D7089F4907F92609087CC24FF2441854B
:107AD0005285638574854C295D296E297F294187EC
:107AE000528763877487FF90EF90DF90CF9008955F
:107AF000CF92DF92FF920F931F93CF93DF93F12CDE
:107B00006115710509F499C06A01EB018C01CB0183
:107B10000E942914F82E882309F48FC0D2FE09C0D0
:107B2000D8018C918B3009F44BC0E8F58A3009F408
:107B30004CC0D0FE09C0F801608186EF860F84300A
:107B400018F0CE010E94011BD1FE6EC0D801149620
:107B50004D915D916D917C91179711968C918295C5
:107B60008F70873038F0893008F43EC08A508230F8
:107B700008F46CC0CE010E943514EC81FD81309771
:107B800009F452C080858F709EEF980F923010F0EC
:107B900081114AC0D80111969C91907F80858F7089
:107BA000892B808741C08C30B9F040E050E062E022
:107BB00070E08D3009F0BDCFCE010E944F3DB9CFAE
:107BC00040E050E061E070E0F7CF40E050E061E07D
:107BD00070E0CE010E94263D40E050E062E070E09F
:107BE000CE010E94263DA5CFEC81FD813097E1F0CA
:107BF00080858F709EEF980F923010F0811114C025
:107C00004187528763877487EC81FD818085807FFF
:107C100083608087EC81FD818085982F907F8F70B5
:107C20008067903609F4BDCF63E67CE085EC9CE08C
:107C30000E94D48AC8010E94C12F8F2DDF91CF915D
:107C40001F910F91FF90DF90CF900895CE010E9479
:107C50003514EACFCF92DF92EF92FF926A017B0157
:107C600063E0FC01808191810E94A59F009791F0C3
:107C7000FC0120852F70223069F46185728583852F
:107C800094856C217D218E219F21FF90EF90DF90C4
:107C9000CF90089560E070E0CB01F7CFCF92DF92F4
:107CA000EF92FF920F931F93CF93DF9300D000D0FA
:107CB0001F921F92CDB7DEB76C017B0160FF03C03E
:107CC000E894E0F8F4F8F4FC0DC00E94412966390C
:107CD00071058105910530F0809134089091350847
:107CE000059709F5A70144275770052E000C660B70
:107CF000770BC6010E944F3D6CEE7AE085EC9CE06C
:107D00000E94D48A8FEF9FEF28960FB6F894DEBFBB
:107D10000FBECDBFDF91CF911F910F91FF90EF90DC
:107D2000DF90CF90089519821A821B821C821D82D7
:107D30001E821F8218868A818F708A8340E053E0FA
:107D4000B601CE0101960E94CB3040E057E060E0E2
:107D500070E0C6010E942A3EE62AF72A09811A81AC
:107D60002B813C814D815E816F817885C6010E94A7
:107D7000F6ADCACF4F925F926F927F928F929F9291
:107D8000AF92CF92EF92FF920F931F93CF93DF9317
:107D900000D000D01F921F92CDB7DEB74C010983EF
:107DA0001A832B833C834D835E836F83788762E3E2
:107DB00077E085EC9CE00E94D48ACE0101960E9477
:107DC000C12F8981811135C00A810F700130B1F155
:107DD00068F1023021F010E0053009F042C0D40112
:107DE000ED91FC9102A0F3A1E02D09811A812B8174
:107DF0003C814D815E816F817885C401199581E058
:107E000090E028960FB6F894DEBF0FBECDBFDF918D
:107E1000CF911F910F91FF90EF90CF90AF909F90D7
:107E20008F907F906F905F904F900895CC24C39473
:107E3000D6CF813061F1823009F4EEC065E277E09F
:107E400085EC9CE00E94D48A4AE050E0698185EC90
:107E50009CE00E94428985EC9CE00E943E8901E002
:107E600010E065E177E085EC9CE00E94D48AB801DF
:107E700085EC9CE00E94B49F85EC9CE00E943E89CA
:107E8000CE0101960E94C12F90E080E0BACF1A8106
:107E900012951F701C30A0F4E12FF0E08827EC5AF7
:107EA000F04C8F4F0C9442E4E93F9C3F9C3F603F75
:107EB000603F603FD03FA93F603F603F883F883FC1
:107EC0002FEF3FEF24313105D0F4163009F49FC075
:107ED00008F082C01150123008F48DC0F4016281A4
:107EE000738140E052E0CE0101960E94783D60E04F
:107EF00072E1D40112968D919C910E944E3ED40164
:107F0000ED91FC9102A0F3A1E02DCC24C3946DCFA0
:107F10008D819E81AF81B88585369105A105B1051A
:107F200024F084E690E0A0E0B0E0B7FF03C080E07A
:107F300090E0DC019C01C6CF2D8130E0A4E6B0E0EA
:107F40000E941FE42FEF30E040E050E00E94EDE39C
:107F5000B9CF4D805E806F80788420E030E0A90149
:107F6000C301B2010E9481E287FD11C020E030E030
:107F700048EC52E4C301B2010E9475E5181654F4AE
:107F8000412C512C88EC682E82E4782E03C0412CC1
:107F9000512C3201C301B2010E943FE59B0192CFF7
:107FA0006D817E818F81988524E630E040E050E04D
:107FB0000E94EDE3253631054105510524F024E604
:107FC00030E040E050E057FF7DCF20E030E0A901F5
:107FD00079CF30E020E076CF173081F01A508CE472
:107FE00090E0A0E0B0E0123008F078CF8D839E835F
:107FF000AF83B88773CF8CE48D8370CF80E090E03F
:10800000A8E9B2E48D839E83AF83B88767CF82EE01
:108010009DE1A0E0B0E0EACF1D821E821F8218869B
:10802000D401ED91FC9102A0F3A1E02DCC24C394E6
:1080300002E01A812B813C8140E0DCCEAF92BF92FE
:10804000CF92EF920F931F93CF93DF93CDB7DEB70D
:10805000C856D1090FB6F894DEBF0FBECDBF5C0184
:10806000A2960FAFA297A3961FAFA397A4962FAF88
:10807000A497A5963FAFA597A6964FAFA697A796AC
:108080005FAFA797A8966FAFA897A9967FAFA9975C
:108090009E2D28E0FE01EF59FF4FDE01A75ABF4F8A
:1080A00001900D922A95E1F7A296EFADA297E150CB
:1080B000ED3008F0F2C0EC2CF0E08827ED59FF4BD2
:1080C0008F4F0C9442E4DA40E34041414B41374149
:1080D0007040D1404D414D41EC40FE4024411141A2
:1080E000992331F0C5010E94D11A009709F449C0C3
:1080F00067E0CE01875A9F4F0E94B9316AED77E061
:1081000085EC9CE00E94D48A4AE050E06A966FAD0C
:108110006A9785EC9CE00E9442896FEC77E085ECE1
:108120009CE00E94D48ACE01875A9F4F0E94DB3187
:10813000AB01BC012AE030E085EC9CE00E94E489C0
:1081400085EC9CE00E943E896A960FAD6A976B961B
:108150001FAD6B976C962FAD6C976D963FAD6D977D
:108160006E964FAD6E976F965FAD6F97A0966FADA1
:10817000A097A1967FADA197C5010E94FE3381E033
:1081800090E0C859DF4F0FB6F894DEBF0FBECDBFE9
:10819000DF91CF911F910F91EF90CF90BF90AF9053
:1081A0000895911105C0C5010E94D11A009749F3A5
:1081B00066E09FCF992329F0C5010E94D11A00974C
:1081C00001F362E096CF911105C0C5010E94D11A5A
:1081D0000097B9F261E08DCF40E050E061E070E0DF
:1081E000C5010E942A3E672B682B692B29F4C50123
:1081F0000E94D11A009729F26BE07BCF40E050E05B
:1082000061E070E0C5010E942A3E672B682B692B54
:1082100031F0C5010E94D11A009709F4B2CF6AE08B
:1082200068CF40E050E062E070E0C5010E942A3E65
:10823000672B682B692B31F0C5010E94D11A00977A
:1082400009F49FCF6CE055CF40E050E062E070E071
:10825000C5010E942A3E672B682B692B31F4C501AA
:108260000E94D11A009709F48CCF6DE042CF911192
:1082700006C0C5010E94D11A009709F482CF63E0BD
:1082800038CF992331F0C5010E94D11A009709F423
:1082900078CF65E02ECF64E02CCF90E080E071CF06
:1082A0002F923F924F925F926F927F928F929F9206
:1082B000AF92BF92CF92DF92EF92FF920F931F93F4
:1082C000CF93DF93CDB7DEB7C35CD1090FB6F89477
:1082D000DEBF0FBECDBF3C01C755DF4F0883C95A73
:1082E000D040C655DF4F1883CA5AD040C555DF4F1E
:1082F0002883CB5AD040C455DF4F3883CC5AD04066
:10830000C355DF4F4883CD5AD040C255DF4F588305
:10831000CE5AD040C155DF4F6883CF5AD040C055A8
:10832000DF4F7883C05BD040CF54DF4FF982E882C3
:10833000C15BD040CB54DF4FC882C55BD040C35433
:10834000DF4FA882CD5BD0400E9441296B01CD5404
:10835000DF4F79836883C35BD040683C7105A4F428
:1083600063E67AE08EE19CE00E94D48AB6018EE159
:108370009CE00E94B49F8EE19CE00E943E89AA246A
:10838000AA94BA2C0C944E4B0E940DADC054DF4FF2
:10839000688379838A839B83C05CD040C655DF4F56
:1083A0008881CA5AD0408F70282E312C20913408F1
:1083B00030913508C254DF4F39832883CE5BD040DB
:1083C000CF54DF4FE881F981C15BD040309721F075
:1083D000808181110C942A4FD3011B968C918823A4
:1083E00041F0C3010B96CF54DF4F99838883C15B63
:1083F000D0402114310411F00C94734FCF54DF4F4F
:10840000E881F981C15BD040309711F00C942E4F78
:10841000F301238C348C2114310411F40C94734F28
:10842000C655DF4F8881CA5AD0408F7011F00C9426
:10843000734F622DCE0187559F4F0E949231C756D0
:10844000DF4F2883C959D040C656DF4F3883CA59F9
:10845000D040C556DF4F4883CB59D040C456DF4F7C
:108460005883CC59D040C356DF4F6883CD59D04094
:10847000C256DF4F7883CE59D040C156DF4F888334
:10848000CF59D040C056DF4F9883C05AD0400C948B
:10849000734FD3018D919C91892B09F470CFB4E077
:1084A0002B16310499F5C354DF4FE880CD5BD040E3
:1084B000C755DF4F0881C95AD040C655DF4F1881D4
:1084C000CA5AD040C555DF4F2881CB5AD040C45539
:1084D000DF4F3881CC5AD040C355DF4F4881CD5A49
:1084E000D040C255DF4F5881CE5AD040C155DF4FE2
:1084F0006881CF5AD040C055DF4F7881C05BD040F3
:10850000C3010E94FE335C010C944E4BC755DF4FF4
:108510001881C95AD040143009F4B6C248F4112366
:1085200009F435C0912C812CAA24AA94BA2C23C317
:1085300088EF810F8230B0F788E0FE01E755FF4FEA
:10854000DE01119601900D928A95E1F7C655DF4F35
:10855000E881CA5AD0408E2F807F09F438C3E29553
:10856000EF70E150EB3008F032C3F0E08827E454BC
:10857000FD4B8F4F0C9442E4D545D545E745C645A4
:10858000C6453A46294629462946C645C645198262
:108590001A821B821C821D821E821F8218868A817B
:1085A0008F708A83C655DF4F8881CA5AD040807F3A
:1085B00009F4B8CF0AE02016310409F421C25CF4B2
:1085C0002114310459F122E02216310409F4D4C0F7
:1085D000912C812C10C23BE02316310409F4BCC15C
:1085E0008CE028163104A1F7B301CE0101960E9458
:1085F00057A3CE0187559F4F0E940714BC01CE019F
:1086000001960E94B13488E0FE013196DE01A75543
:10861000BF4F01900D928A95E1F7EAC1EF2B59F017
:1086200060E27AE085EC9CE00E94D48A85EC9CE0D4
:108630000E943E89CDCFC3010E94985C8C0161E00D
:1086400070E01816190614F070E060E085EC9CE00C
:108650000E94B49F67E974E085EC9CE00E946E8AFA
:10866000CE0187559F4F0E94DB31AB01BC012AE050
:1086700030E085EC9CE00E94E48985EC9CE00E945F
:108680003E89CE0187559F4F1016110614F00C94A9
:108690001E4F0E94DB31912C812C672B682B692B9C
:1086A00089F562E0CE0187559F4F0E94B931CF56C0
:1086B000DF4F2883C159D040CE56DF4F3883C2598F
:1086C000D040CD56DF4F4883C359D040CC56DF4F02
:1086D0005883C459D040CB56DF4F6883C559D0402A
:1086E000CA56DF4F7883C659D040C956DF4F8883BA
:1086F000C759D040C856DF4F9883C859D040882406
:108700008394982C44244394DD24D3943AC061E0AC
:10871000CE0187559F4F0E94B931C757DF4F28833D
:10872000C958D040C657DF4F3883CA58D040C557C4
:10873000DF4F4883CB58D040C457DF4F5883CC58C5
:10874000D040C357DF4F6883CD58D040C257DF4F6A
:108750007883CE58D040C157DF4F8883CF58D04060
:10876000C057DF4F9883C059D04088248394982CF9
:1087700044244394D12C05C0912C812C412CDD2420
:10878000DA94B301CE0101960E9457A38A81982FF3
:1087900092959F70945F9F70923060F4C655DF4F42
:1087A0009881CA5AD04092959F70923019F48F7078
:1087B00080628A83D30118969C91973071F4C655D4
:1087C000DF4F8881CA5AD040807E803211F08034D9
:1087D00021F48A818F7080628A83F301A185B2853A
:1087E000892F90E0109741F0ED91FC911197068C44
:1087F000F78DE02DCD0119957C01C755DF4F08811C
:10880000C95AD040C655DF4F1881CA5AD040C55505
:10881000DF4F2881CB5AD040C455DF4F3881CC5A26
:10882000D040C355DF4F4881CD5AD040C255DF4FAD
:108830005881CE5AD040C155DF4F6881CF5AD040C1
:10884000C055DF4F7881C05BD040CE0101960E94B9
:10885000EC34CF57DF4F2883C158D040CE57DF4F7D
:108860003883C258D040CD57DF4F4883C358D040DB
:10887000CC57DF4F5883C458D040CB57DF4F688365
:10888000C558D040CA57DF4F7883C658D040C95723
:10889000DF4F8883C758D040C857DF4F9883C858E8
:1088A000D040CE0101960E94C12F442069F1C655E7
:1088B000DF4F8881CA5AD04082958F709FE0980F11
:1088C0009F70923020F08A5F8F708230E8F48A8146
:1088D00082958F7081508230B8F42D8130E0AFEFF7
:1088E000B0E00E941FE424E630E040E050E00E9447
:1088F000EDE32F3F31054105510529F024F02FEF1D
:1089000030E040E050E02D8388E0FE013196DE014A
:10891000A755BF4F01900D928A95E1F7F2E19F2A8A
:10892000512CAA24AA94BA2CD30118968C9118978A
:10893000873009F0E4C5CD54DF4FE881F981C35B8E
:10894000D040EE35F1400CF0EDC36CED79E08EE1F6
:108950009CE00E94D48A0FCDB301CE0101960E9403
:1089600057A3C255DF4F8881CE5AD0409A81929545
:108970009F7039F0923049F0912C812C55245394FA
:108980003BC09A819F7090629A8390E085369105F2
:1089900014F084E690E08E8388E0FE013196DE01DB
:1089A000A755BF4F01900D928A95E1F762E0CE0185
:1089B00087559F4F0E949231EA962FAFEA97EB9628
:1089C0003FAFEB97EC964FAFEC97ED965FAFED971F
:1089D000EE966FAFEE97EF967FAFEF97C158DF4FF0
:1089E0008883CF57D040C058DF4F9883C058D040BD
:1089F000812CE2E19E2E512C412CDD24DA9491CF82
:108A0000B301CE0101960E9457A3C155DF4F688183
:108A1000CF5AD040C055DF4F7881C05BD0407170D5
:108A2000CE0101960E94FE3A482E912C812C5524AD
:108A30005394882311F388E0FE013196DE01A75597
:108A4000BF4F01900D928A95E1F762E0CE01875504
:108A50009F4F0E949231E2962FAFE297E3963FAF8D
:108A6000E397E4964FAFE497E5965FAFE597E69618
:108A70006FAFE697E7967FAFE797E8968FAFE897F7
:108A8000E9969FAFE997B4CF09E02016310409F4C5
:108A900059C0C3010E94985C1816190654F562E08B
:108AA000CE0187559F4F0E94B931AA962FAFAA9742
:108AB000AB963FAFAB97AC964FAFAC97AD965FAF71
:108AC000AD97AE966FAFAE97AF967FAFAF97E0968C
:108AD0008FAFE097E1969FAFE19788248394982C1D
:108AE000AA24AA94BA2C512C44244394DD24D39470
:108AF0001BCF61E0CE0187559F4F0E94B931A296EE
:108B00002FAFA297A3963FAFA397A4964FAFA4977A
:108B1000A5965FAFA597A6966FAFA697A7967FAFCE
:108B2000A797A8968FAFA897A9969FAFA9978824D3
:108B30008394982CAA24AA94BA2C512C44244394AC
:108B4000D12CF2CE40E050E061E070E0C3010E9421
:108B50002A3E672B682B692B89F040E050E061E0EA
:108B600070E0C3010E94263D8824839494E0992EEE
:108B7000AA24A394B12C512C412C41C140E050E0D7
:108B800061E070E0C3010E944F3DEECFC355DF4F5F
:108B9000288139814A815B81CD5AD040A4E6B0E07A
:108BA0000E940CE46B017C010DC0C355DF4FC880EF
:108BB000CD5AD04024E6C29E600111240D2C000C39
:108BC000EE08FF08C114D104E104F10429F485E0A2
:108BD000C82ED12CE12CF12C193041F4F094E09402
:108BE000D094C094C11CD11CE11CF11CB301CE0176
:108BF00087559F4F0E9457A360E0CE0187559F4F36
:108C00000E94B9316A962FAF6A976B963FAF6B9708
:108C10006C964FAF6C976D965FAF6D976E966FAF1A
:108C20006E976F967FAF6F97A0968FAFA097A19624
:108C30009FAFA19732E02316310409F474C01CF5EC
:108C4000442443942114310409F46EC0912C812CE6
:108C500040C220E030E048EC52E4C355DF4F688169
:108C600079818A819B81CD5AD0400E94E7E20E949F
:108C70003FE598CFC355DF4FC880D980EA80FB809D
:108C8000CD5AD0409FCF9AE02916310409F4C4C1CF
:108C9000ABE02A163104D1F6C655DF4F8881CA5A97
:108CA000D04082958F70823009F02FC2C701B60183
:108CB00024E630E040E050E00E94EDE3C255DF4F93
:108CC0008881CE5AD04090E0280F391F37FF02C06C
:108CD00030E020E02536310514F024E630E0C255BE
:108CE000DF4F2883CE5AD04062E0CE0187559F4F98
:108CF0000E9492312A962FAF2A972B963FAF2B973F
:108D00002C964FAF2C972D965FAF2D972E966FAF69
:108D10002E972F967FAF2F9760968FAF60976196B3
:108D20009FAF6197D3C1412CF30181859285009754
:108D300081F5808590E010E5812E912CA12CB12C3D
:108D40008530910549F0812C912C5401449721F0F4
:108D5000812C912C54018A94C655DF4FE881CA5A60
:108D6000D040E295EF70E150EB3008F046C1F0E002
:108D70008827E254F94B8F4F0C9442E4D146D146F8
:108D8000FD47FD47FD47CA47884788478847024750
:108D90000247DC01ED91FC91068CF78DE02D1995D1
:108DA000CACFC355DF4F1881CD5AD040C701B60195
:108DB00024E630E040E050E00E94EDE3DA01C90132
:108DC000810F911DA11DB11DB7FF03C080E090E090
:108DD000DC018F3F9105A105B10529F024F08FEF4B
:108DE00090E0A0E0B0E0C355DF4F8883CD5AD0407B
:108DF000812CB2E19B2E512CAA24AA94BA2CDD24FA
:108E0000DA9492CDC355DF4F088119812A813B81C5
:108E1000CD5AD040C754DF4F088319832A833B8340
:108E2000C95BD04014E6C116D104E104F1040CF092
:108E300041C0A4E6B0E0C754DF4F288139814A81A0
:108E40005B81C95BD0400E940CE4C60ED71EE81EB1
:108E5000F91E81149104A104B104B9F0A501940193
:108E60000E940CE4362F272FB701A60177FF03C01D
:108E700040E050E0BA01C32ED22E7C014C155D05B6
:108E80006E057F0514F46A017B01C355DF4FC8826C
:108E9000D982EA82FB82CD5AD040C655DF4F888105
:108EA000CA5AD0408F708066C655DF4F8883CA5A31
:108EB000D0409ECFC701B60124E630E040E050E04C
:108EC0000E94EDE3C754DF4F88819981AA81BB815D
:108ED000C95BD040280F391F4A1F5B1F81149104C2
:108EE000A104B10461F057FF03C020E030E0A90104
:108EF00082169306A406B50614F4A5019401C35581
:108F0000DF4F288339834A835B83CD5AD04070CFAB
:108F1000C355DF4F688179818A819B81CD5AD040CA
:108F20000E943FE5C754DF4F688379838A839B8320
:108F3000C95BD040C701B60124E630E040E050E014
:108F40000E94EDE3C754DF4F688179818A819B815C
:108F5000C95BD040620F731F841F951F8114910459
:108F6000A104B10461F097FF03C060E070E0CB01A1
:108F700086169706A806B90614F4C501B4010E9426
:108F800088E2C355DF4F688379838A839B83CD5AF8
:108F9000D0402ECFC355DF4F88819981AA81BB81F4
:108FA000CD5AD040C80ED91EEA1EFB1E8114910472
:108FB000A104B104C9F0A4E6B0E0A50194010E94A7
:108FC0000CE4362F272FB701A60177FF03C040E03E
:108FD00050E0BA01C32ED22E7C014C155D056E0502
:108FE0007F0514F46A017B01C355DF4FC882D98223
:108FF000EA82FB82CD5AD040FBCE88E0FE0131965A
:10900000DE01A755BF4F01900D928A95E1F7912C93
:10901000812C55245394F0CEC655DF4F8881CA5A0F
:10902000D04082958F70823009F055C0C701B601DB
:1090300024E630E040E050E00E94EDE3C155DF4F10
:109040008881CF5AD040C055DF4F6881C05BD04087
:10905000962F9170280F391F2E3691E039072CF486
:1090600037FF05C02DE631E002C030E020E0C155F9
:10907000DF4F2883CF5AD040C055DF4F8881C05B77
:10908000D04030FB80F9C055DF4F8883C05BD040B3
:1090900062E0CE0187559F4F0E94923162962FAFBA
:1090A000629763963FAF639764964FAF64976596F8
:1090B0005FAF659766966FAF669767967FAF679766
:1090C00068968FAF689769969FAF6997812CA2E1E8
:1090D0009A2E512C18C088E0FE013196DE01A7556A
:1090E000BF4F01900D928A95E1F764E17AE08EE13D
:1090F0009CE00E94D48A8EE19CE00E943E89912CE3
:10910000812C55245394412C77CE88E0FE01319672
:10911000DE01A755BF4F01900D928A95E1F768E0F7
:109120007AE0E5CFCB54DF4F1881C55BD0401123E7
:1091300009F467C01296ED91FC9180858F7085309F
:1091400009F070C0C254DF4FE881F981CE5BD04096
:10915000359709F467C0C3010E94985C21E0181696
:1091600019060CF020E0D22ECF54DF4F48815981F0
:10917000C15BD040C354DF4F2881CD5BD040BE01DE
:1091800067557F4FD30112968D919C910E94D15BC0
:10919000B1E02B16310409F045C0C655DF4F1881E8
:1091A000CA5AD040812F807FE9F1C354DF4FC88075
:1091B000CD5BD040ED2CC755DF4F0881C95AD04058
:1091C000C555DF4F2881CB5AD040C455DF4F388179
:1091D000CC5AD040C355DF4F4881CD5AD040C255FC
:1091E000DF4F5881CE5AD040C155DF4F6881CF5AEA
:1091F000D040C055DF4F7881C05BD040C3010E9492
:109200001E40C755DF4F8881C95AD040853009F4C8
:1092100045C170F48330C9F1CD54DF4F1882C35B70
:10922000D040B8C0CB54DF4F1882C55BD040E9CFE7
:10923000863009F47CC0873079F7C3010E94321B65
:10924000182F863009F062C060EB79E085EC9CE075
:109250000E94D48A66E070E085EC9CE00E94B49F96
:1092600085EC9CE00E943E8962E0CE0187559F4FCD
:109270000E94B93129AF3AAF4BAF5CAF6DAF7EAF53
:109280008FAF21969FAF21973DC0C3010E94321B33
:10929000853021F093E0A92EB12C00C267EC79E073
:1092A00085EC9CE00E94D48A65E070E085EC9CE04F
:1092B0000E94B49F85EC9CE00E943E89B301CE01E0
:1092C00087559F4F0E9457A361E0CE0187559F4F5E
:1092D0000E94B93122962FAF229723963FAF239752
:1092E00024964FAF249725965FAF259726966FAFAC
:1092F000269727967FAF279728968FAF289729968E
:109300009FAF2997689480F890F886CF62E979E05A
:1093100085EC9CE00E94D48A612F70E085EC9CE093
:109320000E94B49F85EC9CE00E943E89B3CF40E050
:1093300050E061E070E0C3010E942A3E672B682B79
:10934000692B09F0A8C0EFEFDE129BC0C3010E9499
:10935000985C181619060CF497C0B301CE01875516
:109360009F4F0E9457A361E0CE0187559F4F0E94F7
:10937000B93129AB3AAB4BAB5CAB6DAB7EAB8FABD2
:1093800098AF689480F890F8F6E0CD54DF4FF883FA
:10939000C35BD04084010160C655DF4F8881CA5A43
:1093A000D040982F9F70923050F4C755DF4F98816E
:1093B000C95AD040992319F0840101601160807F5F
:1093C00009F492C01260CB54DF4F2881C55BD040B6
:1093D00021111D7FA801B301CE0187559F4F0E9427
:1093E000783D4801AA24A394B12C5110CAC5D301D9
:1093F00019968D919C91009709F070C340E050E060
:1094000062E070E0C3010E942A3E672B682B692B43
:1094100009F496C364E378E08EE19CE00E94D48A6C
:109420008EE19CE00E943E8992FCF3C469E178E001
:1094300085EC9CE00E94D48AB50185EC9CE00E94FA
:10944000B49F62E178E085EC9CE00E94D48A0E949F
:109450000DADAB01BC01C054DF4F088119812A81D9
:109460003B81C05CD040401B510B620B730B2AE068
:1094700085EC9CE00E94F28885EC9CE00E943E898D
:109480000DC1DD2009F469CF68E779E085EC9CE047
:109490000E94D48AFFCE63E679E0F8CF0FEFD012B6
:1094A00009C0C3010E94985C181619062CF066E4E6
:1094B00079E0ECCFDD20D9F362E0CE0187559F4FF4
:1094C0000E94B93129A73AA74BA75CA76DA77EA731
:1094D0008FA798AB689480F890F815E0CD54DF4FD3
:1094E0001883C35BD04056CF40E052E0B301CE01B9
:1094F00087559F4F0E94CB30811164CF64CF3FEFDF
:10950000D312E7C0C3010E94985CDD24D3941816DF
:1095100019060CF4E1C0D12C68E379E085EC9CE0FD
:109520000E94D48A0D2D0D2C000C110BC754DF4F57
:1095300019830883C95BD040B80185EC9CE00E9488
:10954000B49F61E379E085EC9CE00E94D48A642DAD
:1095500070E085EC9CE00E94B49F85EC9CE00E944A
:109560003E89CF54DF4FE880F980C15BD040E114E1
:10957000F10409F4BAC062E172E2C7010E948CDC16
:1095800001E010E0892B09F44BC06EE072E2C701E4
:109590000E948CDC02E010E0892B09F441C06DE0F0
:1095A00078E0C7010E948CDC05E010E0892BC1F156
:1095B00069E078E0C7010E948CDC06E010E0892BAE
:1095C00079F163ED71E2C7010E948CDC03E110E0E8
:1095D000892B31F16EEC71E2C7010E948CDC04E151
:1095E00010E0892BE9F068ED71E2C7010E948CDC84
:1095F0000EE010E0892BA1F061EC71E2C7010E943E
:109600008CDC0FE010E0892B59F06AEC71E2C701A5
:109610000E948CDC10E000E0892B11F405E110E0E1
:10962000C3010E94321B282F30E0CD54DF4F398315
:109630002883C35BD040232B61F4C754DF4F88815C
:109640009981C95BD040CD54DF4F99838883C35B38
:10965000D0400115110509F491C0CD54DF4FA88108
:10966000B981C35BD040A017B107C9F165E179E0CA
:1096700085EC9CE00E94D48ACD54DF4F68817981CB
:10968000C35BD04085EC9CE00E94B49F85EC9CE0DD
:109690000E943E896DEFA62EBB24BA94C501CD531E
:1096A000DF4F0FB6F894DEBF0FBECDBFDF91CF9175
:1096B0001F910F91FF90EF90DF90CF90BF90AF90F0
:1096C0009F908F907F906F905F904F903F902F90E2
:1096D0000895DD2009F420CF442443941DCFCF54B6
:1096E000DF4F19821882C15BD040B1E02B163104E4
:1096F000A9F4CB54DF4FE881C55BD040EE2399F04D
:10970000C655DF4F8881CA5AD040807FF1E0CB54E4
:10971000DF4FF883C55BD040811105C0CB54DF4FCC
:109720001882C55BD040C755DF4F0881C95AD04069
:10973000CD54DF4F0883C35BD040063108F0B8C179
:10974000E02FF0E08827E855F44B8F4F0C9442E46B
:10975000FB4B1B4D0B4D3E4CFB4BEE4CB44C854C28
:10976000FB4BFB4B554D554D654D654D364D364DBF
:10977000584D584D584D364D364D364DF301818577
:109780009285009709F4B1CFDC01ED91FC91068838
:10979000F789E02DC354DF4FA880CD5BD040C42CA7
:1097A000C755DF4F0881C95AD040C655DF4F1881D1
:1097B000CA5AD040C555DF4F2881CB5AD040C45536
:1097C000DF4F3881CC5AD040C355DF4F4881CD5A46
:1097D000D040C255DF4F5881CE5AD040C155DF4FDF
:1097E0006881CF5AD040C055DF4F7881C05BD040F0
:1097F00019950C948342CD54DF4F1882C35BD0403F
:10980000CB54DF4F2881C55BD040222309F4EDCD36
:109810003D2D3170E32EC354DF4FC880CD5BD04067
:10982000C755DF4F0881C95AD040C655DF4F188150
:10983000CA5AD040C555DF4F2881CB5AD040C455B5
:10984000DF4F3881CC5AD040C355DF4F4881CD5AC5
:10985000D040C255DF4F5881CE5AD040C155DF4F5E
:109860006881CF5AD040C055DF4F7881C05BD0406F
:10987000C3010E941E40E89491F8B7CDC3010E9435
:10988000321B853009F006CD60E079E085EC9CE084
:109890000E94D48A65E070E085EC9CE00E94B49F51
:1098A00085EC9CE00E943E89B301CE0187559F4F15
:1098B0000E9457A3D30118968C918530B9F46EE0BD
:1098C000CE0187559F4F0E94B93129A33AA34BA3DC
:1098D0005CA36DA37EA38FA398A7689480F890F8EB
:1098E000CD54DF4F1882C35BD0406FC061E0CE0122
:1098F00087559F4F0E94B931298F3A8F4B8F5C8FCC
:109900006D8F7E8F8F8F98A3E8CFC3010E94321B8B
:10991000182F863031F569EE78E085EC9CE00E94E6
:10992000D48A66E070E085EC9CE00E94B49F85ECF0
:109930009CE00E943E8962E0CE0187559F4F0E94C5
:10994000B931298B3A8B4B8B5C8B6D8B7E8B8F8BDC
:10995000988F40E050E068E070E0C3010E94263D2F
:10996000BCCF6BEC78E0D4CC40E050E061E070E03C
:10997000C3010E942A3E672B682B692B61F5D11029
:1099800027C0B301CE0187559F4F0E9457A361E0C6
:10999000CE0187559F4F0E94B93129873A874B875F
:1099A0005C876D877E878F87988B40E050E068E00A
:1099B00070E0C3010E944F3D689480F890F8B6E0D3
:1099C000CD54DF4FB883C35BD0404424439418CFB9
:1099D00061EB78E05BCD6CE978E058CDDD20C1F03B
:1099E00062E0CE0187559F4F0E94B93129833A83A7
:1099F0004B835C836D837E838F839887689480F824
:109A000090F8E5E0CD54DF4FE883C35BD040DDCF75
:109A10006FE778E03BCDC655DF4F8881CA5AD0400A
:109A20008F70823008F05CCFC3010E94321B8530FA
:109A300009F053CF2FCCC655DF4F8881CA5AD0408A
:109A40008F70823008F04CCFDD2081F066E678E040
:109A500085EC9CE00E94D48A61E0C3010E94011B56
:109A600060E071E1C3010E944E3E14CCC655DF4F49
:109A70008881CA5AD040982F9F70923008F030CF1A
:109A8000CD54DF4FF881C35BD040FF2309F49DCF55
:109A9000807F31F4B301CE0187559F4F0E9457A3B9
:109AA000689480F803E0902A1BCF689492F818CF4E
:109AB000C655DF4F8881CA5AD040807F19F4689418
:109AC00090F80ECF13E0912A0BCFCD54DF4F1882C0
:109AD000C35BD040812C54E0952E77CFDC01ED9113
:109AE000FC91028CF38DE02DC755DF4F0881C95AD8
:109AF000D040C655DF4F1881CA5AD040C555DF4FF8
:109B00002881CB5AD040C455DF4F3881CC5AD04041
:109B1000C355DF4F4881CD5AD040C255DF4F5881E1
:109B2000CE5AD040C155DF4F6881CF5AD040C05582
:109B3000DF4F7881C05BD040199581115FCC6ACC32
:109B4000F30181859285892B09F473C081149104F6
:109B500039F0A401B301CE0187559F4F0E94783D93
:109B6000D30119968D919C91CF54DF4FE880F980F5
:109B7000C15BD040DC01ED91FC910688F789E02DB6
:109B8000C354DF4FA880CD5BD040C42CC755DF4FF6
:109B90000881C95AD040C655DF4F1881CA5AD040F3
:109BA000C555DF4F2881CB5AD040C455DF4F38818F
:109BB000CC5AD040C355DF4F4881CD5AD040C25512
:109BC000DF4F5881CE5AD040C155DF4F6881CF5A00
:109BD000D040C055DF4F7881C05BD04019955C0103
:109BE000F30181859285DC01ED91FC91068CF78D66
:109BF000E02D1995059711F4689480F892FC01C145
:109C0000CD54DF4FB881C35BD040BB2321F06B2F15
:109C1000C3010E94011BC254DF4FE881F981CE5B72
:109C2000D040B401359709F401CCC3010E944E3EE7
:109C3000FDCB8085853009F476C0863009F7C7559D
:109C4000DF4FD880C95AD040DD2009F46CC070E0E5
:109C500060E0C3010E94281C8C018114910439F03A
:109C6000A401B301CE0187559F4F0E94783D011595
:109C7000110531F2F12CE12C17FF06C01195019569
:109C80001109EE24E394F12CC80101978635910562
:109C900008F0B6CFC02E61E0802F0E9483ABEFEFBB
:109CA000ED0DE53110F5F0E08827E65AF14B8F4FC6
:109CB0000C9442E46F4E714E754E754E714E6F4E60
:109CC000714E754E754E754E754E754E754E6F4E86
:109CD0006F4E754E754E754E754E6F4E6F4EF1E070
:109CE000EF266E2D8C2D0E9455AB6FE278E085EC4F
:109CF0009CE00E94D48AB80185EC9CE00E94B49F4D
:109D00006DE278E085EC9CE00E94D48AB70185EC96
:109D10009CE00E94B49F85EC9CE00E943E89689480
:109D200080F890F86EC08114910439F0A401B30159
:109D3000CE0187559F4F0E94783D02E020163104E6
:109D400009F463C013E02116310429F02A94232872
:109D500009F056CFE4CFC3010E94E51A892B49F4DC
:109D6000D301ED91FC91608171818BED94E00E94B3
:109D7000DBB0CE0187559F4F0E94C01320E030E03A
:109D800048EC52E40E94E7E20E943FE5CB54DF4FEB
:109D9000688379838A839B83C55BD040CB54DF4F34
:109DA000C880D980C55BD04088E00E9416181B018E
:109DB0002C0169E278E085EC9CE00E94D48ACB54C7
:109DC000DF4F68817981C55BD04085EC9CE00E94C3
:109DD000B49F64E278E085EC9CE00E94D48AB201F2
:109DE000A101662777272AE085EC9CE00E94F28893
:109DF00085EC9CE00E943E89B101A601C3010E944E
:109E00002720AA24A394B12CFBCE689480F891F863
:109E1000F8CFC254DF4F08811981CE5BD0400530A6
:109E2000110509F403CB40E054E0B301CE0187559E
:109E30009F4F0E94783D60E074E0F7CE0E94DB31D6
:109E4000672B682B692B11F00C948743912C812C84
:109E50000C94B8432114310409F045C08081882353
:109E600011F40C940842CE018F549F4F0E941D3B69
:109E70001C01C655DF4F8881CA5AD0408F7071F5DA
:109E8000622DCE0187559F4F0E949231CF55DF4FF3
:109E90002883C15AD040CE55DF4F3883C25AD040B4
:109EA000CD55DF4F4883C35AD040CC55DF4F588340
:109EB000C45AD040CB55DF4F6883C55AD040CA55ED
:109EC000DF4F7883C65AD040C955DF4F8883C75AC1
:109ED000D040C855DF4F9883C85AD0402114310470
:109EE00011F40C94084268E57AE085EC9CE00E944D
:109EF000D48AB60185EC9CE00E94B49F61E57AE0CB
:109F000085EC9CE00E94D48AD301ED91FC916081A4
:109F1000718185EC9CE00E946E8A6BE47AE085ECAE
:109F20009CE00E94D48ACF54DF4F68817981C15B65
:109F3000D04085EC9CE00E946E8A69E47AE085EC72
:109F40009CE00E94D48ACE0187559F4F0E94C12F6A
:109F5000CF54DF4FE881F981C15BD040309711F4D5
:109F60000C9449428081843211F00C94494265E39B
:109F70007AE085EC9CE00E94D48A85EC9CE00E940B
:109F80003E898CEFA82EBB24BA9488CB2F923F92A7
:109F90004F925F926F927F928F929F92AF92BF92F9
:109FA000CF92DF92EF92FF920F931F93CF93DF93A5
:109FB000CDB7DEB7C955D1090FB6F894DEBF0FBED5
:109FC000CDBF3C01562E6296EFAE62976396FFAE10
:109FD000639764960FAF649765961FAF6597669613
:109FE0002FAF669767963FAF679768964FAF6897B2
:109FF00069965FAF69976A96CFAE6A972D2C4A2C07
:10A000003B2C009709F464C1FC0180858F7084307B
:10A0100009F449C128F4882309F44EC180E02DC019
:10A02000853009F444C08630C9F76AEE74E0C30194
:10A030000E942D9F4C01009709F46FC0B12CA12CF8
:10A04000D12CC12C6296EFAC62976396FFAC6397FC
:10A0500064960FAD649765961FAD659766962FADB4
:10A06000669767963FAD679768964FAD6897699614
:10A070005FAD6997652D0E94C64FC75ADF4F0FB677
:10A08000F894DEBF0FBECDBFDF91CF911F910F912E
:10A09000FF90EF90DF90CF90BF90AF909F908F9008
:10A0A0007F906F905F904F903F902F900895809198
:10A0B00030088F5F809330088680978081149104E8
:10A0C00031F1A42CB32C6A96CFAC6A97D22C62964D
:10A0D000EFAC62976396FFAC639764960FAD64979D
:10A0E00065961FAD659766962FAD669767963FADEF
:10A0F000679768964FAD689769965FAD6997652DCC
:10A10000C4010E94C64FF40182809380D7CF809112
:10A11000300881508093300881CF6EEE74E0C30127
:10A120000E942D9F7C0163EF74E0C3010E942D9F6C
:10A130006C01552039F0F1E05F1609F495C010E08C
:10A1400000E00CC068EF74E0C3010E942D9F4C0139
:10A150006DEF74E0C3010E942D9F8C018114910466
:10A1600009F443010115110509F48301E114F10417
:10A1700021F46A96EFAC6A97F22CC114D10411F461
:10A18000C42CD32C8114910409F49FC0F401808560
:10A190008F70843009F099C0818492840115110573
:10A1A00009F49EC0F80180858F70843009F098C052
:10A1B00001851285E114F10409F4E0C081149104D1
:10A1C00009F49DC06BE079E185EC9CE00E94D48AA3
:10A1D000F7016185728585EC9CE00E946E8A66E0DD
:10A1E00079E185EC9CE00E94D48AB40185EC9CE086
:10A1F0000E946E8A85EC9CE00E943E89CE018F5AB7
:10A200009F4F0E94C12FC114D10409F0C0C0F701B3
:10A2100080858F70843009F00CC161857285CE0114
:10A2200001960E94513BCE0101960E942914882379
:10A23000B1F00E9441296B01683C71050CF073C0BC
:10A2400062ED78E18EE19CE00E94D48AB6018EE155
:10A250009CE00E94B49F8EE19CE00E943E89CE016A
:10A2600001960E945F14E5C062E075E0C3010E94A0
:10A270002D9F4C0167E075E0C3010E942D9F8C016A
:10A280008114910409F0D7C068EF74E0C3010E9403
:10A290002D9F4C010115110509F45ACF892B09F0A6
:10A2A00065CF430163CF10E000E0912C812CD12CCD
:10A2B000C12CF12CE12C52CF10E000E0912C812C2C
:10A2C000D12CC12CF12CE12C51CF912C812C66CFBB
:10A2D000CA2CDB2C6A96EFAC6A97F22C912C812C5D
:10A2E00000E020E033E040E150E0BE016F5B7F4FD3
:10A2F000CE018F5A9F4F0E94A02D8C015BCF6CEF37
:10A3000078E185EC9CE00E94D48AF7016185728532
:10A3100085EC9CE00E946E8A67EF78E185EC9CE01A
:10A320000E94D48A6BCF8114910431F0B401CE0124
:10A3300001960E94ECA393CFA12CCC24C394F12CC2
:10A34000E12C62960FAD629763961FAD639764969A
:10A350002FAD649765963FAD659766964FAD66974E
:10A3600067965FAD679768966FAD689769967FADA2
:10A370006997CE0101960E94504171CFC114D1045A
:10A3800009F457C00115110509F453C004C00115A3
:10A39000110509F43CCFF60180858F70843009F0F7
:10A3A00044C060EF78E185EC9CE00E94D48AF6011D
:10A3B0006185728585EC9CE00E946E8A6BEE78E187
:10A3C00085EC9CE00E94D48AB80185EC9CE00E9458
:10A3D0006E8A85EC9CE00E943E89F601618572855B
:10A3E00040E450E0CE0101960E94D1E80E944B9FCC
:10A3F0008823D9F080913009811117C06FE270E095
:10A40000CE0101960E9498E8892B51F4F60121852E
:10A41000328543E050E060E4CE0101960E94D827E7
:10A42000B801CE0101960E94DBADE114F10409F000
:10A43000EECE81E022CE892B09F098CE89CEAF9264
:10A44000BF92CF92DF92EF92FF920F931F93CF9321
:10A45000DF9300D000D01F921F92CDB7DEB7E98204
:10A46000FA820B831C832D833E834F835887DC0144
:10A470001296ED91FC91309781F1028113810115C3
:10A48000110559F1F80180858F70853031F57B0118
:10A49000C8010E94BC9F823000F161E0C8010E94A7
:10A4A000A59F0097D1F0DC0118962C912F702630D3
:10A4B000A1F4B7010E942D9F009779F0B12CA12C37
:10A4C000D12CC12CE980FA800B811C812D813E8129
:10A4D0004F8158856FEF0E94C64F28960FB6F894AB
:10A4E000DEBF0FBECDBFDF91CF911F910F91FF90C7
:10A4F000EF90DF90CF90BF90AF9008954F925F9212
:10A500006F927F928F929F92AF92BF92CF92DF9283
:10A51000EF92FF920F931F93CF93DF93CDB7DEB7E8
:10A52000C258D1090FB6F894DEBF0FBECDBFDC0113
:10A5300014962D913C911597232B09F496C43B0159
:10A540004C01ED91FC910484F585E02D199597FD62
:10A5500040C0823091050CF488C40397D1F5D40132
:10A560001496ED91FC9180A591A5A2A5B3A5892B88
:10A570008A2B8B2B71F10E940DAD9B01AC01D40194
:10A580001496ED91FC9160A571A582A593A5A12CCF
:10A59000B12C650116E9E12EF12C00E010E00E94DB
:10A5A000AB268823B1F0D401ED91FC910684F785A8
:10A5B000E02D62E0C4011995F401E480F58080E0AB
:10A5C0000E941618D70198966D937D938D939C9356
:10A5D0009B9790E080E06A94672809F048C4D40112
:10A5E000ED91FC910484F585E02DC4011995029745
:10A5F00031F50E940DAD9B01AC01D4011496ED9193
:10A60000FC9160A571A582A593A5A12CB12C650133
:10A6100018E8E12E13E1F12E00E010E00E94AB26D5
:10A62000882369F062EB77E185EC9CE00E94F88A70
:10A630004DE050E062E072E0C4010E940D27F40199
:10A6400087819085DC01ED91FC910084F185E02DFE
:10A65000199585970CF423C3F4016481758145E253
:10A6600050E0878190850E94C088D40117968D9113
:10A670009C91DC01ED91FC910084F185E02D199510
:10A680007C01892B89F062E070E080E090E00E941C
:10A69000DBACF40187819085DC01ED91FC910284B3
:10A6A000F385E02D1995E1CF6DEA77E185EC9CE02B
:10A6B0000E94D48A4AE050E0F401668185EC9CE077
:10A6C0000E94428968EA77E185EC9CE00E94D48A86
:10A6D000D4011496ED91FC91EE0DFF1D608140E1D7
:10A6E00050E06A3078F466E674E085EC9CE00E9405
:10A6F0006E8AD4011496ED91FC91EE0DFF1D40E1A0
:10A7000050E0608185EC9CE00E944289BFEFEB1A2B
:10A71000FB0AE4E2EE16F104D9F6D4011496ED91A9
:10A72000FC91159784A197A1891709F4B4C287A356
:10A730001496ED91FC91EF961CAE1DAE1EAE1FAEB1
:10A74000EF97C158DF4F188219821A821B82CF57A8
:10A75000D040ED968FADED978F70ED968FAFED9762
:10A7600083A190E06C01B0E1CB0ED11C499708F0B9
:10A770008CC2B584878986A3118D738CD4011496FD
:10A780002D913C91858DD90195968C93E48CF12C7B
:10A79000878DF40120813181A281B3810D90BC911C
:10A7A000A02D6D917C91D9015496ED91FC912CE0F6
:10A7B00035E044ED54E080FD02C047ED54E0C401B3
:10A7C0001995B0E8EB16F10409F09CC0D40112967B
:10A7D000ED91FC9113970190F081E02D60817181E2
:10A7E000ED91FC910488F589E02D23E135E044EDFD
:10A7F00054E0C401199569E175E085EC9CE00E9484
:10A800006E8AD4011496ED91FC914AE050E065A166
:10A8100085EC9CE00E94428985EC9CE00E943E8988
:10A82000D4011496ED91FC91159785A12D913C9141
:10A83000119712960D90BC91A02D0D90BC91A02D5A
:10A840006D917C91D9015496ED91FC9124E235E013
:10A8500044ED54E083FD02C047ED54E0C401199576
:10A86000D401ED91FC9111970488F589E02D1296A1
:10A870008D919C91DC018D919C91DC016D917C917D
:10A88000D40114968D919C91DC0195968C912BE2CC
:10A8900035E044ED54E081FD02C047ED54E0C401D1
:10A8A00019951982113009F4FDC108F442C0123023
:10A8B00009F41DC2133009F43FC26DE977E1CE01FE
:10A8C00001960E9495DC60E0CE0185589F4F0E9462
:10A8D000B93164962FAF649765963FAF65976696DA
:10A8E0004FAF669767965FAF679768966FAF689749
:10A8F00069967FAF69976A968FAF6A976B969FAF9D
:10A900006B973BC0EF2809F076CFD4011296ED91FA
:10A91000FC9113970190F081E02D60817181ED91A0
:10A92000FC910488F589E02D23E135E047ED54E002
:10A9300060CF69EC77E1CE0101960E9495DC60E181
:10A94000CE0185589F4F0E94B931E4962FAFE4970E
:10A95000E5963FAFE597E6964FAFE697E7965FAF90
:10A96000E797E8966FAFE897E9967FAFE997EA96A1
:10A970008FAFEA97EB969FAFEB97D4011296ED91CC
:10A98000FC9113970190F081E02D60817181ED9130
:10A99000FC910488F589E02D28EC34E0AE014F5F8E
:10A9A0005F4FC4011995EC96EFACEC97ED96FFACB8
:10A9B000ED97EE960FADEE97EF961FADEF97C1585E
:10A9C000DF4F2881CF57D040C058DF4F3881C05863
:10A9D000D040CF57DF4F4881C158D040CE57DF4FCE
:10A9E0005881C258D04069EC74E0C4010E941F52E3
:10A9F000F40180819181A281B3810D90BC91A02D41
:10AA00006D917C91DC015496ED91FC912DEC34E03C
:10AA100047ED54E0772011F044ED54E0C40119955E
:10AA20000D2C000CEE08FF08D4011296ED91FC915C
:10AA300013970190F081E02D60817181ED91FC917F
:10AA40000088F189E02D03EC14E0A7019601C40110
:10AA500019954B2C512C712C612CBFEFBB16A9F012
:10AA6000D4011296ED91FC9113970190F081E02DA5
:10AA700060817181ED91FC910088F189E02D07E3FF
:10AA800015E0A3019201C40119951B861C861D8641
:10AA90001E868C858F70806A8C878B854C853D8562
:10AAA0002E852C968FAF2C972D964FAF2D972E96E7
:10AAB0003FAF2E972F962FAF2F972C2D6396CCAEAE
:10AAC000DDAEEEAEFFAE6397E82EF42E032F2F9689
:10AAD0001FAD2F9761963FAD619762964FAD62971C
:10AAE00063965FAD639764EC74E0C4010E941F52EB
:10AAF0001B861C861D861E868C858F70806A8C87BF
:10AB00008B859C85AD85BE858B8B9C8BAD8BBE8BE1
:10AB10004F8A588E698E7A8E63E0CE0143960E94EA
:10AB2000923124962FAF249725963FAF25972696EE
:10AB30004FAF269727965FAF279728966FAF289736
:10AB400029967FAF29972A968FAF2A972B969FAF8A
:10AB50002B9779018A019B01AC0168E375E0C40180
:10AB60000E941F521982D4011496ED91FC9186A186
:10AB7000811107C16EEC77E1CE0101960E9495DC50
:10AB80006EE0CE0185589F4F0E94B9312BAF3CAF8C
:10AB90004DAF5EAF6FAF21967FAF219722968FAFFB
:10ABA000229723969FAF2397D4011496ED91FC91A1
:10ABB000159726A130E050E040E01296ED91FC910F
:10ABC00013970190F081E02D60817181ED91FC91EE
:10ABD0000088F189E02D0DE315E0C4011995D40139
:10ABE0001496ED91FC9185A180FD14C062E877E197
:10ABF000CE0101960E9495DC62E0CE0185589F4F00
:10AC00000E94B9312B873C874D875E876F87788B91
:10AC1000898B9A8BD4011296ED91FC911397019038
:10AC2000F081E02D60817181ED91FC910488F589BE
:10AC3000E02D23E435E0AE014F5F5F4FC40119956D
:10AC4000EC96EFACEC97ED96FFACED97EE960FAD72
:10AC5000EE97EF961FADEF97C158DF4F2881CF5782
:10AC6000D040C058DF4F3881C058D040CF57DF4F59
:10AC70004881C158D040CE57DF4F5881C258D0408C
:10AC800064E475E0C4010E941F5261EA77E185EC3B
:10AC90009CE00E94D48A85EC9CE00E943E8981E081
:10ACA00090E0E5C062EC77E1CE0101960E9495DC70
:10ACB00061E1CE0185589F4F0E94B931AC962FAF0C
:10ACC000AC97AD963FAFAD97AE964FAFAE97AF9600
:10ACD0005FAFAF97E0966FAFE097E1967FAFE197F8
:10ACE000E2968FAFE297E3969FAFE39746CE6EEB87
:10ACF00077E1CE0101960E9495DC62E1CE01855894
:10AD00009F4F0E94B931A4962FAFA497A5963FAF4D
:10AD1000A597A6964FAFA697A7965FAFA797A896B9
:10AD20006FAFA897A9967FAFA997AA968FAFAA975A
:10AD3000AB969FAFAB9721CE6EEC77E1CE0101963B
:10AD40000E9495DC6EE0CE0185589F4F0E94B9317C
:10AD50006C962FAF6C976D963FAF6D976E964FAF19
:10AD60006E976F965FAF6F97A0966FAFA097A19603
:10AD70007FAFA197A2968FAFA297A3969FAFA397FD
:10AD8000FCCD8130A9F468E977E1CE0101960E94FB
:10AD900095DC64E1CE0185589F4F0E94B9312BAB01
:10ADA0003CAB4DAB5EAB6FAB78AF89AF9AAFFCCE2F
:10ADB0008230A9F463E977E1CE0101960E9495DC27
:10ADC00063E1CE0185589F4F0E94B9312BA73CA764
:10ADD0004DA75EA76FA778AB89AB9AABE5CE833062
:10ADE000A9F46AE877E1CE0101960E9495DC6FE054
:10ADF000CE0185589F4F0E94B9312BA33CA34DA390
:10AE00005EA36FA378A789A79AA7CECE8430A9F4B2
:10AE100066E877E1CE0101960E9495DC65E1CE01FE
:10AE200085589F4F0E94B9312B8F3C8F4D8F5E8F7D
:10AE30006F8F78A389A39AA3B7CE8D3609F0B4CECD
:10AE40006DE977E1CE0101960E9495DC60E0CE01CC
:10AE500085589F4F0E94B9312B8B3C8B4D8B5E8B5D
:10AE60006F8B788F898F9A8F9FCE8FEF9FEFCE5702
:10AE7000DF4F0FB6F894DEBF0FBECDBFDF91CF918D
:10AE80001F910F91FF90EF90DF90CF90BF90AF9008
:10AE90009F908F907F906F905F904F9008956F92EA
:10AEA0007F928F929F92AF92BF92CF92DF92EF925A
:10AEB000FF920F931F93CF93DF93CDB7DEB7A09789
:10AEC0000FB6F894DEBF0FBECDBF8C01862E7A017F
:10AED000DC018D919C911197892B09F466C0149621
:10AEE000ED91FC91309709F460C080818071BFEFD3
:10AEF0006B135DC0B1F481E0A0960FB6F894DEBF8D
:10AF00000FBECDBFDF91CF911F910F91FF90EF90BA
:10AF1000DF90CF90BF90AF909F908F907F906F9079
:10AF200008954330510539F3818082942FE08222C5
:10AF30006FE777E085EC9CE00E94D48A4AE050E01D
:10AF4000D80113966C9185EC9CE00E9442896DE7D4
:10AF500077E085EC9CE00E94D48AD8011496ED91AC
:10AF6000FC9161816F704AE050E085EC9CE00E94AA
:10AF700042896AE777E085EC9CE00E94D48A4AE047
:10AF800050E0682D85EC9CE00E94428985EC9CE0B5
:10AF90000E943E89D8011496ED91FC9181818F70B9
:10AFA000881207C080818F7E808380E0A5CF8111C9
:10AFB000FCCF198E1A8E1B8E1C8E1D8E1E8E1F8E20
:10AFC00018A28A8D8F708A8FD8011496ED91FC910A
:10AFD00081818F708815A9F1B3E0EB16F10489F136
:10AFE00068E777E085EC9CE00E94D48A4AE050E074
:10AFF000F801638185EC9CE00E94428966E777E076
:10B0000085EC9CE00E94D48AD8011496ED91FC91C5
:10B0100061816F704AE050E085EC9CE00E944289BB
:10B0200063E777E085EC9CE00E94D48A4AE050E038
:10B03000682D85EC9CE00E94428985EC9CE00E9492
:10B040003E89F80120813181FCE0F81508F416C131
:10B05000E82DF0E08827E05DF74A8F4F0C9442E43A
:10B060003D587A58FB5812591E59FB58D458FB5872
:10B0700021592C59E8582F593B59D8011496CD9095
:10B08000DC90F60181818F70853009F4F7C050F4AF
:10B090008230C1F066E575E0C9010E942D9F3C0138
:10B0A000912C4BC08730D1F08A30A1F76FE475E066
:10B0B000C9010E942D9F3C01D6019C9092FA9924CF
:10B0C00090F83BC069E475E0C9010E942D9F3C01E6
:10B0D000D6019C9090FA992490F82FC068E475E00E
:10B0E000C9010E942D9F3C01F601908091FA99249C
:10B0F00090F823C06BE575E0C9010E942D9F3C01CB
:10B10000D8011496ED91FC91808180FB992490F8F0
:10B11000982F9E7F80FF916090836114710469F481
:10B1200061E0CE0149960E94B931298B3A8B4B8B55
:10B130005C8B6D8B7E8B8F8B988FF801A080B1809C
:10B140006EEE74E0C5010E942D9F6C0163EF74E008
:10B15000C5010E942D9F5C01892B81F4C114D1048B
:10B1600069F460E0CE0149960E94B93129833A839F
:10B170004B835C836D837E838F839887D80114967D
:10B18000ED91FC916114710409F07CC0898D8111ED
:10B1900079C0B82DBF708B2E8181807F882A8182F3
:10B1A00080818F7E8083A7CE60E675E0C9010E9412
:10B1B0002D9F3C01D8011496ED91FC91808181FB7B
:10B1C000992490F8982F9D7F81FF92609083B5CF4E
:10B1D00066E675E0C9010E942D9F3C01D8011496D6
:10B1E000ED91FC91808182FB992490F8982F9B7FB0
:10B1F00082FF9460EBCF66E575E0C9010E942D9F48
:10B200003C01892B09F04CCF62E0CE0149960E94A7
:10B21000B93129873A874B875C876D877E878F870F
:10B22000988B3ECF6CE675E0C9010E942D9F3C01D2
:10B23000D8011496ED91FC9190804CCF61E775E0B8
:10B24000F3CF67E775E0C9010E942D9F3C01D8014B
:10B250001496ED91FC9149CF6DE775E0F4CF64E869
:10B2600075E0C9010E942D9F3C01D8011496ED9113
:10B27000FC91908023CF6AE875E0F3CF912C712C7C
:10B28000612C5BCF83E0E816F104B9F0982D9F7034
:10B29000892E8181807F882A818280818F7E808330
:10B2A000E98CFA8C0B8D1C8D2D8D3E8D4F8D58A108
:10B2B000692DC3010E94C64F1ECE81818F708815F3
:10B2C00009F419CE829490EF8922882A81828081A4
:10B2D000806168CF2F923F924F925F926F927F92E0
:10B2E0008F929F92AF92BF92CF92DF92EF92FF9296
:10B2F0000F931F93CF93DF93CDB7DEB763970FB64E
:10B30000F894DEBF0FBECDBF4C013B0140E058E0DA
:10B3100060E070E00E942A3E672B682B692B09F4DD
:10B320005CC019821A821B821C821D821E821F82AF
:10B3300018868A818F708A8340E053E0B401CE0181
:10B3400001960E94CB30D40119968D919C91892B46
:10B3500009F443C040E058E060E070E0C4010E949E
:10B36000263D66EB7AE085EC9CE00E94D48AF401ED
:10B3700081859285DC01ED91FC910688F789E02DAD
:10B38000A12CCC24C394F12CE12C09811A812B81AE
:10B390003C814D815E816F81788519958F3F98073B
:10B3A000E1F0D401ED91FC9160817181892B09F06C
:10B3B000B8C085EC9CE00E946E8A64EB7AE085EC74
:10B3C0009CE00E94D48A6CEA7AE085EC9CE00E94C2
:10B3D000D48A85EC9CE00E943E8965E0F40180817E
:10B3E00091810E94A59F6C01009709F4D0C0DC01F7
:10B3F0001896BC91B98BBB2EB2942FE0B222FC01FF
:10B4000021843284438454840E940DADBB2009F40E
:10B41000BEC0261A370A480A590A19861A861B8698
:10B420001C86B9861A851F70106A1A872D863E867B
:10B430004F86588AF4E06F16710439F5E12C90E2DA
:10B44000F92E0B2D2B853C854D855E856F85788982
:10B45000C4010E94F6ADC201B10128EE33E040E024
:10B4600050E00E94EDE3BA01A9012AE030E085EC4A
:10B470009CE00E94E4896DED7AE085EC9CE00E94FE
:10B48000D48A85EC9CE00E943E8957FE80C022E071
:10B4900022163104410420E852060CF478C00E94C0
:10B4A00041291B017B8B6A8BE12C80E2F82E0985F8
:10B4B0001A852B853C854D855E856F857889C4010D
:10B4C0000E94F6AD8A899B89883C9105BCF564ECA5
:10B4D0007AE08EE19CE00E94D48AB1018EE19CE08A
:10B4E0000E94B49F8EE19CE00E943E898FEF9FEF07
:10B4F00063960FB6F894DEBF0FBECDBFDF91CF913C
:10B500001F910F91FF90EF90DF90CF90BF90AF9081
:10B510009F908F907F906F905F904F903F902F9073
:10B52000089585EC9CE00E946E8A6AEA7AE085ECD8
:10B530009CE00E94D48A66EA7AE047CFD60118964A
:10B540008C9118978F7018968C9319821A821B828F
:10B550001C821D821E821F8218868A818F708A83B8
:10B56000B98289898F70AA24A394873009F0A12C0D
:10B57000CC24C394F12CE12C09811A812B813C81CC
:10B580004D815E816F817885C4010E945041B1E098
:10B590006B167104E9F440E053E060E070E0C40130
:10B5A0000E942A3E611571058105910589F020915F
:10B5B0003408309135082630310551F4C4010E9419
:10B5C0004E3E40E053E060E070E0C4010E94263D42
:10B5D000F40181859285009719F490E080E088CF8E
:10B5E000DC01ED91FC910484F585E02D1995892B02
:10B5F000A1F3F40181859285DC01ED91FC91048039
:10B60000F581E02DB301199573CFAF92BF92CF9220
:10B61000DF92EF92FF920F931F93CF93DF93CDB7FB
:10B62000DEB76D970FB6F894DEBF0FBECDBF0E9498
:10B630000DAD9B01AC0160917F07709180078091F7
:10B64000810790918207A12CB12C650118EEE12EA3
:10B6500013E0F12E00E010E00E94AB26F82E8823C4
:10B6600051F00E940DAD60937F0770938007809327
:10B67000810790938207809130088F5F8093300814
:10B68000E0913608F09137080681178194E0C92EC1
:10B69000D12CF11003C082E0C82ED12CA090360826
:10B6A000B0903708A114B10429F10115110511F169
:10B6B000F80180858F708530A9F7C8010E94BC9F72
:10B6C000823080F3B801CE0101960E94ED21CE01B7
:10B6D00001960E942914882329F0B601CE01019613
:10B6E0000E946A59F80102811381CE0101960E94DD
:10B6F0005F14D4CF809130088150809330088091BE
:10B700003408909135080597D9F1FF20C9F110E070
:10B7100060917D0770917E076115710589F11111A6
:10B720002FC0FB0180858F70853091F4CE0101968A
:10B730000E94ED2161E070E0CE0101960E946A59FD
:10B7400011E0892B09F410E0CE0101960E945F14EC
:10B75000E0917D07F0917E07309791F0828193818F
:10B7600090937E0780937D07892B91F6E0913608B0
:10B77000F09137088681978190937E0780937D07AB
:10B780006D960FB6F894DEBF0FBECDBFDF91CF919F
:10B790001F910F91FF90EF90DF90CF90BF90AF90EF
:10B7A00008952F923F924F925F926F927F928F9265
:10B7B0009F92AF92CF92DF92EF92FF920F931F93DF
:10B7C000CF93DF93CDB7DEB76D970FB6F894DEBF9A
:10B7D0000FBECDBF009709F4A9C0FC0130853F70B2
:10B7E000353009F0A3C0D22E1A014B016680778054
:10B7F000809130088F5F809330086114710409F4E0
:10B8000090C0F30180858F70843009F086C0618517
:10B81000728580913608909137080E942D9F2C01E7
:10B82000009709F47AC0FC0180858F70853009F09B
:10B8300074C0B201CE0101960E94ED2181149104E1
:10B84000B1F0CE0101960E942914882381F0AD2C1D
:10B85000C12C7101F4010081118122813381448165
:10B86000558166817781CE0101960E94504160E04A
:10B87000C2010E94A59F0097E9F1FC0120852F706D
:10B880002230C1F581859285A385B4850797A105EE
:10B89000B10581F561E0C2010E94A59F2D2DA10196
:10B8A000B4010E94D15B8114910499F5882389F138
:10B8B00080913008815080933008CE0101960E941B
:10B8C0005F1481E06D960FB6F894DEBF0FBECDBF5A
:10B8D000DF91CF911F910F91FF90EF90DF90CF906C
:10B8E000AF909F908F907F906F905F904F903F9020
:10B8F0002F9008958114910461F4CE0101960E9465
:10B900002914882331F0CE0101960E94985C892B7E
:10B9100079F6CE0101960E945F14F3016280738074
:10B920006CCF8091300881508093300880E0CACF7E
:10B93000DF92EF92FF920F931F93CF93DF9300D08C
:10B9400000D01F921F92CDB7DEB77C0119821A82F8
:10B950001B821C821D821E821F8218868A818F7024
:10B960008A83D701ED91FC916081718185EC9CE027
:10B970000E946E8A64EA7AE085EC9CE00E94D48A98
:10B98000C7010E94291481111BC06BE97AE085EC84
:10B990009CE00E94D48A85EC9CE00E943E890FEFD7
:10B9A0001FEFC80128960FB6F894DEBF0FBECDBFBB
:10B9B000DF91CF911F910F91FF90EF90DF9008954D
:10B9C000C7010E94321BD82EF7018185928500970E
:10B9D00091F0DC01ED91FC91008CF18DE02D199539
:10B9E0008C0197FD08C081E00115110509F480E084
:10B9F0000E946818D6CFF7018085873009F42EC0E1
:10BA0000EFEFED0DE43150F5F0E08827E55FF24A05
:10BA10008F4F0C9442E41F5D285D2E5D2E5D285DE6
:10BA20001F5D2E5D2E5D2E5D2E5D2E5D2E5D2E5DCD
:10BA30001F5D2E5D2E5D2E5D2E5D1F5D1F5D6CE713
:10BA40007AE085EC9CE00E94D48A01E010E0A9CF66
:10BA500080E00E94681810E000E0A3CF40E052E0D0
:10BA6000B701CE0101960E94CB30D70118968C9178
:10BA70001897873079F160F4833009F455C0843029
:10BA800061F06CE87AE085EC9CE00E94D48AE3CF18
:10BA9000883009F449C08930A1F760E0CE010196F1
:10BAA0000E94F3128C0161E87AE085EC9CE00E9430
:10BAB000D48AB80185EC9CE00E94B49F85EC9CE0A0
:10BAC0000E943E8991E080E0012B09F490E0092F6B
:10BAD000182F67CF1296ED91FC9180858F7010E042
:10BAE00000E0853001F769E97AE085EC9CE00E948E
:10BAF000D48A20E050E040E070E060E0F70182810D
:10BB000093810E94D15BF82E082F10E066E97AE05D
:10BB100085EC9CE00E94D48A8F2D0E94681885ECE9
:10BB20009CE00E943E893DCFCE0101960E94DB3110
:10BB30008B01B9CF2F923F924F925F926F927F927B
:10BB40008F929F92AF92BF92CF92DF92EF92FF922D
:10BB50000F931F93CF93DF93CDB7DEB760970FB6E8
:10BB6000F894DEBF0FBECDBF6130710509F495C0FA
:10BB7000DC0112966D917C916115710509F48DC0FF
:10BB80004C0119821A821B821C821D821E821F8216
:10BB900018868A818F708A8340E052E0CE01019638
:10BBA0000E94CB3060E0CE0101960E94F3121C018E
:10BBB000F401828193810E94E51A2B013C01D4019A
:10BBC00017962D913D914D915C911A97D1010E944C
:10BBD00017E42FEF30E040E050E00E94CBE32987EC
:10BBE0003A874B875C870E940DAD9B01AC0189852C
:10BBF0009A85AB85BC850097A105B10509F468C09D
:10BC0000A12CB12C65017C018D01C301B2010E9400
:10BC1000AB2689874114510461047104F1F1D40108
:10BC200017968D919D910D90BC91A02D8D879E872B
:10BC3000AF87B88B0E940DAD9B01AC018D859E85B1
:10BC4000AF85B8890097A105B10561F0A12CB12C91
:10BC500065017C018D01C301B2010E94AB268823DE
:10BC600009F451C0D40112966D907C9080E00E943E
:10BC70001618AB01BC01C3010E942720232869F0DC
:10BC8000F40184810E941412D40116969C918913A8
:10BC900004C061E0C4010E943F1B90E080E0609618
:10BCA0000FB6F894DEBF0FBECDBFDF91CF911F91CD
:10BCB0000F91FF90EF90DF90CF90BF90AF909F904B
:10BCC0008F907F906F905F904F903F902F9008954E
:10BCD00091E099879FCFB985BB23F1F060E0C40163
:10BCE0000E943F1BF401828193810E94985C892B02
:10BCF000A1F640E050E0BA01D40112968D919C91DA
:10BD00000E942720CACFF40184810E941412D4011A
:10BD100016969C918913DFCF232809F4BECFF40136
:10BD200084810E941412D40116969C918913B5CF78
:10BD3000B985B111B2CFADCFCF93DF93EC0169E1FB
:10BD400078E185EC9CE00E94D48A6C817D8185EC51
:10BD50009CE00E94B49F63E178E185EC9CE00E9446
:10BD6000D48A85EC9CE00E943E8961E08C810E942F
:10BD700083AB6E818C810E9455AB8A819B81009739
:10BD800029F040E050E0BA010E942720E881F981C3
:10BD90000684F785E02D62E0CE0119958A819B81AA
:10BDA0000E94985C181619065CF40A80DB81C02D8D
:10BDB00080E00E941618AB01BC01CE010E94272032
:10BDC00081E090E0DF91CF9108952F923F924F92C2
:10BDD0005F926F927F928F929F92AF92BF92CF921B
:10BDE000DF92EF92FF920F931F93CF93DF93CDB724
:10BDF000DEB7C955D1090FB6F894DEBF0FBECDBF6F
:10BE00000E940DAD9B01AC016091790770917A079A
:10BE100080917B0790917C07A12CB12C650110E3E8
:10BE2000E12E15E7F12E00E010E00E94AB268823FA
:10BE300009F424C2E0913608F0913708309709F4EC
:10BE40001DC2809130088F5F809330082680378034
:10BE500010E02114310409F434C1F10180858F70A0
:10BE60008530F9F460E0C1010E94A59FFC01818545
:10BE70009285A385B4850597A105B10591F4B1011B
:10BE8000CE0101960E94ED21CE0101960E94291457
:10BE900066968FAF6697811108C0CE0101960E9409
:10BEA0005F14F10122803380D4CF25961CAE1DAEE5
:10BEB0001EAE1FAE259729961CAE1DAE1EAE1FAE40
:10BEC000299740E052E0BE016F5F7F4FCE018F5B4C
:10BED0009F4F0E94CB30CE0101960E94E51A6B0164
:10BEE0007C0169966FAF69976A96DFAE6A9770E0DA
:10BEF00060E0CE0101960E94281C4C01CE018F5BB0
:10BF00009F4F0E94C01365966CAF7DAF8EAF9FAF01
:10BF10006597CE0101960E94321B182FB601DD0CE9
:10BF2000880B990B0E9488E220E030E048EC52E454
:10BF30000E94CDE42B013C01CE0101960E94985C49
:10BF400068969FAF8EAF68976FE776E185EC9CE0CF
:10BF50000E94D48A65966CAD7DAD8EAD9FAD659720
:10BF60000E94E2A669E776E185EC9CE00E94D48A13
:10BF7000C301B2010E94E2A663E776E185EC9CE092
:10BF80000E94D48A612F70E085EC9CE00E94B49FEF
:10BF9000E114F10409F48EC088E00E9416189B0198
:10BFA000AC0144275527B70190E080E0AA24AA9469
:10BFB000BA2CC12CD12C17E2E12E19E0F12E00E0B1
:10BFC00010E00E94AB26882371F1F101608171813C
:10BFD0008EE19CE00E946E8A63E676E18EE19CE051
:10BFE0000E94D48AF1016081718181E995E00E940B
:10BFF000DBB090E080E0BC0169964FAD69976A962E
:10C000005FAD6A97CE0101960E94272062E070E042
:10C01000C4010E94921ACE0101960E945F14669696
:10C020001FAD66973ECF20E030E048E152E4C30107
:10C03000B2010E9475E518163CF4F101608171812E
:10C040008DE995E00E94DBB068968EAD9FAD689754
:10C05000892B19F461E070E0DBCF20E030E040E8AC
:10C060005FE365966CAD7DAD8EAD9FAD65970E942B
:10C0700060E49B01AC01C301B2010E9481E270E067
:10C0800060E087FDC5CFA301920165966CAD7DADE3
:10C090008EAD9FAD65970E9481E21816DCF664E5CF
:10C0A00076E185EC9CE00E94D48A85EC9CE00E94BD
:10C0B0003E89B1CF6AE476E185EC9CE00E94D48AA7
:10C0C000AACF809130088150809330080E940DAD36
:10C0D0006093790770937A0780937B0790937C072E
:10C0E0000E9441292B013C010E940DAD6B017C0196
:10C0F0000E944B9F882309F489C0809130098111E7
:10C1000085C030E020E041E050E060E4CE010196DF
:10C110000E94D8274FE350E063E67BE1CE01019611
:10C120000E94A5DC66E774E0CE0101960E948DE8CE
:10C130004FE350E061E276E1CE0101960E94A5DC7A
:10C140002AE0AE014F5B5F4FC301B2010E9430DDB8
:10C15000BE016F5B7F4FCE0101960E94DBAD30E0E8
:10C1600020E041E050E060E4CE0101960E94D82733
:10C170004FE350E063E67BE1CE0101960E94A5DC2F
:10C1800066E774E0CE0101960E948DE84FE350E02F
:10C190006AE176E1CE0101960E94A5DCC701B601F5
:10C1A00028EE33E040E050E00E94CBE3CA01B90141
:10C1B0002AE0AE014F5B5F4F0E9430DDBE016F5B36
:10C1C0007F4FCE0101960E94DBAD30E020E041E0E0
:10C1D00050E060E4CE0101960E94D8274FE350E082
:10C1E00063E97BE1CE0101960E94A5DC4FE050E0BF
:10C1F0006DE87BE1CE018F5B9F4F0E94C3DCBE01E7
:10C200006F5B7F4FCE0101960E94DBAD112309F4D5
:10C210004FC064E476E185EC9CE00E94D48A0E94E1
:10C220004129AB01BC012AE085EC9CE00E94F28828
:10C230006CE376E185EC9CE00E94D48A6091300842
:10C24000062E000C770B85EC9CE00E94B49F6AE2FE
:10C2500076E185EC9CE00E94D48A4091750750916C
:10C26000760760917707709178072AE085EC9CE06B
:10C270000E94F28885EC9CE00E943E89C75ADF4FFD
:10C280000FB6F894DEBF0FBECDBFDF91CF911F91E7
:10C290000F91FF90EF90DF90CF90BF90AF909F9065
:10C2A0008F907F906F905F904F903F902F90089568
:10C2B0006AE376E185EC9CE00E94D48A0E944129E1
:10C2C000AB01BC012AE085EC9CE00E94F28862E3AD
:10C2D00076E1B0CF3F924F925F926F927F928F92B2
:10C2E0009F92AF92BF92CF92DF92EF92FF920F9305
:10C2F0001F93CF93DF93CDB7DEB7CE56D1090FB6DC
:10C30000F894DEBF0FBECDBFDC0114962D913C9199
:10C31000232B09F424C69B01225031092230310518
:10C3200008F091C23B014C01FC018281803409F488
:10C33000F7C208F04AC0843008F085C2809109072E
:10C340008F5F80930907A3016FEFC4010E944F57CD
:10C35000D40112960C9112970695017013961C91B8
:10C3600013978AEC810F803108F043C06AEA75E0C8
:10C370008D919C910E942D9F7C010097D1F1FC0131
:10C3800080858F708530A9F58091040D181324C025
:10C390008091050D803401F58091060D9091070D77
:10C3A0005C01990FCC08DD0860E0C7010E94A59FE1
:10C3B000FC0181859285A385B485A816B906CA06B5
:10C3C000DB060CF065C0512C3EC0823409F4A8C2D3
:10C3D00008F439C28058AFCF1093040D80E48093E5
:10C3E000050D812F0E9496AC9093070D8093060D4A
:10C3F000D7CF212F30E0F901EF55F24E8491F901AA
:10C40000E55BF24E1491F901EB50F34EF490FF20EE
:10C4100009F43BC081110E94EEAAEF2DF0E0EE0F6F
:10C42000FF1FE75AF84FA591B491EC911E2331E01C
:10C4300020E009F430E0832F922F552453940817FD
:10C44000190609F0C0CFF3E06F16710409F488C033
:10C45000D4011496ED91FC91E181EF70E150EC3044
:10C4600008F07EC0F0E08827E75CFD498F4F0C9410
:10C4700042E45A62D6639062C662D663DF62D663D4
:10C480001363406359639B63BD6390E080E0D5CF45
:10C4900061E0C7010E94A59F55245394FC0181854A
:10C4A0009285A385B4858A159B05AC05BD050CF066
:10C4B000CACF89CF0E940DAD9B01AC0144275527FF
:10C4C000D4011496ED91FC916281738190E080E03B
:10C4D000AA24AA94BA2CC12CD12C18EEE12E13E078
:10C4E000F12E00E010E00E94AB268823C9F1F40190
:10C4F000008111816CE675E0C8010E942D9F892B97
:10C5000041F461E775E0C8010E942D9F892B09F471
:10C510000EC142E050E063E0C4010E944F5720C0CA
:10C520000E940DAD9B01AC0144275527D401149600
:10C53000ED91FC916281738190E080E0AA24AA943D
:10C54000BA2CC12CD12C1CE2E12EFF24F39400E084
:10C5500010E00E94AB2642E050E064E0811184C00C
:10C56000D4011496ED91FC91808183FB992790F979
:10C57000951509F4D2C1982F907E09F439C1982FEE
:10C58000907E90528F71892B808358C10E940DAD8F
:10C590009B01AC0144275527D4011496ED91FC91E1
:10C5A0006281738190E080E0AA24AA94BA2CC12C05
:10C5B000D12C16E9E12EF12C00E010E0CACF0E9448
:10C5C0000DAD9B01AC0144275527D4011496ED9184
:10C5D000FC916281738190E080E0AA24AA94BA2C35
:10C5E000C12CD12C18EEE12E13E0F12E00E010E06A
:10C5F0000E94AB26882309F4B3CFF4010081118196
:10C6000067E775E0C8010E942D9F892B41F46DE713
:10C6100075E0C8010E942D9F892B09F488C042E073
:10C6200050E068E079CF0E940DAD9B01AC0144273A
:10C630005527D4011496ED91FC916281738190E0AD
:10C6400080E0AA24AA94BA2CC12CD12C1CE2E12EA1
:10C65000FF24F39400E010E00E94AB2642E050E09B
:10C6600069E0882309F47CCFC4010E944F570E94DF
:10C670000DADD4011496ED91FC917383628370CF5C
:10C680000E940DAD9B01AC0144275527D40114969F
:10C69000ED91FC916281738190E080E0AA24AA94DC
:10C6A000BA2CC12CD12C16E9E12EF12C00E010E0BF
:10C6B000D3CF0E940DAD9B01AC0144275527D40177
:10C6C0001496ED91FC916281738190E080E0AA2440
:10C6D000AA94BA2CC12CD12C18EEE12E13E0F12E25
:10C6E00000E010E00E94AB26882309F439CFF40162
:10C6F0000081118164E875E0C8010E942D9F892B9B
:10C7000039F46AE875E0C8010E942D9F892B21F059
:10C7100042E050E06BE000CF66E675E0C8010E94A1
:10C720002D9F42E050E066E0892B09F4F5CE42E00F
:10C7300050E06DE0F1CE0E940DAD9B01AC014427AD
:10C740005527D4011496ED91FC916281738190E09C
:10C7500080E0AA24AA94BA2CC12CD12C1CE2E12E90
:10C76000FF24F39400E010E00E94AB26882309F434
:10C77000F7CE42E050E06CE077CF0E940DAD9B0118
:10C78000AC0144275527D4011496ED91FC916281A8
:10C79000738190E080E0AA24AA94BA2CC12CD12CF9
:10C7A00016E9E12EF12C00E010E0DECF0E940DAD85
:10C7B0009B01AC0144275527D4011496ED91FC91BF
:10C7C0006281738190E080E0AA24AA94BA2CC12CE3
:10C7D000D12C18E5E12E12E0F12E00E010E00E94CD
:10C7E000AB26882309F4BCCE42E050E060E094CE52
:10C7F0000E940DADD4011496ED91FC9115977383B1
:10C800006283E181EF70552009F445C0E230F1F018
:10C8100050F4EE23E9F1D4011496ED91FC9180815E
:10C8200050FA83F9B1CEE53089F0A3016AE0E73030
:10C8300091F7C4010E944F578111EDCF80910907F4
:10C8400081508093090790E080E08BC3F401008160
:10C85000118160E675E0C8010E942D9F892BA9F423
:10C8600067E775E0C8010E942D9F892B71F46DE781
:10C8700075E0C8010E942D9F892B39F468E475E0AA
:10C88000C8010E942D9F892B19F0A30166E0D1CF2A
:10C89000A30161E0CECFE150ED3008F0BCCFF0E075
:10C8A0008827EA5AFB498F4F0C9442E463640B6477
:10C8B000666466640B6469640B648A648A648A646F
:10C8C0008A648A646664A30162E0B3CFA30165E071
:10C8D000B0CF0D911C9160E675E0C8010E942D9FBC
:10C8E000892BA9F467E775E0C8010E942D9F892B69
:10C8F00071F46DE775E0C8010E942D9F892B39F412
:10C9000068E475E0C8010E942D9F892B19F0A301EE
:10C9100067E08FCFA30160E08CCF8F71806434CE4D
:10C92000B3E06B16710409F48ECF6AEA75E0F40186
:10C93000808191810E942D9F8C01D40113968C914E
:10C940009091040D8913EBC09091050D903409F07E
:10C95000E6C08091060D9091070D3C01011511056F
:10C9600009F40DC1F80120852F70253009F007C1A9
:10C97000C8010E94BC9F382EF3E0F81708F0DBC016
:10C9800063E0C8010E94A59FDC0119968D919C91DE
:10C990003AE0E32EE89E6001E99ED00C1124A396B4
:10C9A000DFAECEAEA39762E0C8010E94A59FDC0176
:10C9B00019968D919C91E89E2001E99E500C1124BE
:10C9C0006201052C000CEE08FF08AF96CCAEDDAE80
:10C9D000EEAEFFAEAF9761E0C8010E94A59F5C017B
:10C9E00060E0C8010E94A59FDC011996CD90DD9002
:10C9F000ED90FC901C97A796CCAEDDAEEEAEFFAEF0
:10CA0000A7979301072C000C440B550B2C193D09DB
:10CA10004E095F09A396CEACDFACA397B601DD0C3F
:10CA2000880B990BAF96CCACDDACEEACFFACAF97FE
:10CA30006C197D098E099F090E94BBE3D5011996E7
:10CA40002D913D914D915C911C97A796CCACDDAC9E
:10CA5000EEACFFACA7972C193D094E095F09A796CC
:10CA60002CAF3DAF4EAF5FAFA7970E94EDE3AF96FF
:10CA7000ACACBDACCEACDFACAF97A20EB31EC41E47
:10CA8000D51E45E0E42E3E1409F468C081E090E034
:10CA9000A396EEACFFACA397A701FF0C660B770B38
:10CAA0004A155B056C057D050CF461C0B601A50156
:10CAB0006201052C000CEE08FF084C155D056E05A3
:10CAC0007F050CF459C06A017B0122E032126BC071
:10CAD0006301770CEE08FF0860E0C8010E94A59F83
:10CAE000FC0181859285A385B485C816D906EA061E
:10CAF000FB060CF44FC261E0C8010E94A59FFC0137
:10CB000081859285A385B4858C159D05AE05BF05ED
:10CB10000CF099CE81E090E0A0E0B0E03EC28093BE
:10CB2000040D90E49093050D0E9496AC9093070D30
:10CB30008093060D12CF8AE0869D5001879DB00C30
:10CB400011240B2C000CCC08DD08512C412C20E0CA
:10CB500038E2A3963FAF2EAFA39798CF64E0C80109
:10CB60000E94A59FDC0119968D919C9191CF66241E
:10CB70006A9423E0722E9CCF712C612CA6CF2AE000
:10CB8000289F6001299FD00C11240D2C000CEE0869
:10CB9000FF08512C412C20E038E2A3963FAF2EAF86
:10CBA000A39781E090E0D4011496ED91FC9162810D
:10CBB0007381A301461B570B57FF03C05195419545
:10CBC0005109841795070CF4C1C08081982F929564
:10CBD00096959770963008F0BCC09F5F9295990F1C
:10CBE000907E8F71892BB4C0F70161857285DB015E
:10CBF0008C91811161C2A114B10409F473C0D501F3
:10CC000018968C9118978F70843009F06BC0199624
:10CC10006D917C91CE0101960E94513BCE0101960F
:10CC20000E942914882309F459C06114710409F47D
:10CC300060C0E114F10431F0F70180858F70843019
:10CC400009F442C025961CAE1DAE1EAE1FAE259740
:10CC500029961CAE1DAE1EAE1FAE299723961FADA2
:10CC600023971F7023961FAF239781E022968FAFE3
:10CC70002297A12CCC24C394F12CE12C01E0249622
:10CC80002FAD249725963FAD259740E027965FADC1
:10CC9000279728966FAD289729967FAD2997CE01C3
:10CCA00001960E9450411AC00115110529F0F801A2
:10CCB00080858F70843019F067ED74E0FDC1618567
:10CCC0007285FB01808195CF61857285FB01808132
:10CCD000882321F0CE0101960E94ECA3CE0101969B
:10CCE0000E945F14D4011496ED91FC9173826282CC
:10CCF000AACD0115110531F0D80118968C918F70CD
:10CD00008430F1F025961CAE1DAE1EAE1FAE2597E9
:10CD100029961CAE1DAE1EAE1FAE299723961FADE1
:10CD200023971F7023961FAF239782E022968FAF21
:10CD30002297A12CCC24C394F12CE12C02E09FCFAC
:10CD4000F80161857285DB018C91C2CF80818F7182
:10CD500080838081803AB8F0C201550CAA0BBB0BCE
:10CD6000C816D906EA06FB0671F0A396EEADFFAD34
:10CD7000A397CF01FF0FAA0BBB0BC816D906EA0673
:10CD8000FB0609F060CD6616770609F45CCD6D965A
:10CD90001CAE1DAE1EAE1FAE6D976B968FAD6B9722
:10CDA0008F7080666B968FAF6B976D968CAD9DADD7
:10CDB000AEADBFAD6D9765968CAF9DAFAEAFBFAF5B
:10CDC0006597AAE0B0E0A70196010E940CE469967D
:10CDD0006CAF7DAF8EAF9FAF699768E477E085EC6D
:10CDE0009CE00E94D48A4AE050E0D40113966C91F2
:10CDF00085EC9CE00E94428966E477E085EC9CE04B
:10CE00000E94D48ACE018F5A9F4F0E94C12F6AEE92
:10CE100074E0F401808191810E942D9FB12CA12C9E
:10CE2000D12CC12C6296EFAC62976396FFAC6397EE
:10CE300064960FAD649765961FAD659766962FADA6
:10CE4000669767963FAD679768964FAD6897699606
:10CE50005FAD69976FEF0E94C64FD4010D911C9191
:10CE60006EEE74E0C8010E942D9F7C0163EF74E0B8
:10CE7000C8010E942D9F8C010097E1F1FC01808583
:10CE80008F708430B9F56185728540E450E0CE0141
:10CE900001960E94D1E86FE270E0CE0101960E94F7
:10CEA00098E8892B59F4D80119962D913C9143E0CB
:10CEB00050E060E4CE0101960E94D82700E020E017
:10CEC00032E040E150E0BE016F5B7F4FCE018F5AF0
:10CED0009F4F0E94A02D0E944B9F882359F0809164
:10CEE0003009811107C0BE016F5B7F4FCE010196F3
:10CEF0000E94DBADE114F10409F4F4CEF701808562
:10CF00008F70843009F0EECE61857285CE01019676
:10CF10000E94513BCE0101960E942914882309F4F6
:10CF2000DDCEA12CCC24C394F12CE12C62960FAD64
:10CF3000629763961FAD639764962FAD649765966D
:10CF40003FAD659766964FAD669767965FAD6797FD
:10CF500068966FAD689769967FAD6997A0CE8FEFA1
:10CF60009FEFC259DF4F0FB6F894DEBF0FBECDBFA3
:10CF7000DF91CF911F910F91FF90EF90DF90CF90B5
:10CF8000BF90AF909F908F907F906F905F904F90E9
:10CF90003F90089580E090E0DC01F4012481358128
:10CFA000F90142815381052E000C660B770B841723
:10CFB0009507A607B70709F446CC3C01D4010D91AB
:10CFC0001C916EEE74E0C8010E942D9F5C0163EF1E
:10CFD00074E0C8010E942D9F6C01A114B10419F4E2
:10CFE000892B09F47FCE6BE575E0C8010E942D9F67
:10CFF0007C0166E575E0C8010E942D9F8C016EE4FE
:10D0000077E085EC9CE00E94D48A4AE050E0F4018D
:10D01000638185EC9CE00E9442896CE477E085ECBA
:10D020009CE00E94D48AB30185EC9CE00E94B49FEE
:10D0300085EC9CE00E943E89C114D10409F4DBCD4B
:10D04000D60118968C9118978F70843009F0D3CD43
:10D0500019966D917C9140E450E0CE0101960E94BA
:10D06000D1E80E944B9F882309F4C5CD80913009F7
:10D070008111C1CD6FE270E0CE0101960E9498E867
:10D08000892B51F4F6012185328543E050E060E4BC
:10D09000CE0101960E94D8276114710409F404CED0
:10D0A000E114F10439F0D70118968C918F70843017
:10D0B00009F49ACD64ED74E0CE0101960E94DBADD7
:10D0C0009ACDEF92FF920F931F93CF93DF93EC01D2
:10D0D0008B011D821C821A821B82E880F980E11478
:10D0E000F10409F474C08091830790918407892B1F
:10D0F00009F46DC0672B09F48701F80180858F70F2
:10D100008630A9F46EEA75E0C8010E942D9F009751
:10D1100019F0FC0181858A8363ED76E0C8010E94E5
:10D120002D9F009709F45AC0FC0181858B8360EB29
:10D1300075E0C7010E942D9F009709F045C061E48A
:10D1400077E085EC9CE00E94D48A4AE050E06B8155
:10D1500085EC9CE00E9442896FE377E085EC9CE0DF
:10D160000E94D48A4AE050E06A8185EC9CE00E94EB
:10D17000428985EC9CE00E943E89E880F9800E940B
:10D1800089918C01892BC1F082E0F801808711869A
:10D1900012861386148680819181009711F00E9477
:10D1A000088F80EB95E00E94378FF8019183808390
:10D1B000B801C7010E942CA360EB75E088819981BA
:10D1C0000E942D9F009719F009969D838C83DF9113
:10D1D000CF911F910F91FF90EF900895F8018081FA
:10D1E00091810E9420DCA2CF8F929F92AF92BF923A
:10D1F000CF92DF92EF92FF920F931F93CF93DF9323
:10D2000000D000D0CDB7DEB720913208309133087E
:10D21000232B09F484C020913108211180C04C01D6
:10D22000809131088F5F80933108809130088F5F43
:10D23000809330080E940DAD9B01AC016091710795
:10D24000709172078091730790917407A12CB12C93
:10D2500065011BE0E12EF12C00E010E00E94AB26FE
:10D26000882309F452C0E0913208F0913308068116
:10D27000178101151105B9F1F80180858F7086308D
:10D2800071F56AEE74E0C8010E942D9F0097D1F0FD
:10D29000FC0120852F702530A9F4E680F780E11489
:10D2A000F104E9F0FA82E982B801CE0101960E9408
:10D2B0006168B401CE0101960E946A61F701E280C3
:10D2C000F380EDCF1A83098370E060E0CE01019610
:10D2D0000E946168B401CE0101960E946A61F80162
:10D2E00002811381C6CFF3E08F16910451F00E94A2
:10D2F0000DAD6093710770937207809373079093DD
:10D3000074071092040D1092050D80913008815021
:10D31000809330088091310881508093310826969F
:10D320000FB6F894DEBF0FBECDBFDF91CF911F9136
:10D330000F91FF90EF90DF90CF90BF90AF909F90B4
:10D340008F900895809130098F5F80933009A89560
:10D3500083E090E00E94F4680E94B98E80913009C9
:10D360008150809330090895CF92DF92EF92FF921F
:10D37000CF93DF93EC018C85883068F40E94BE98CF
:10D380000E940DAD6B017C018C850E94DA988111A1
:10D3900009C088E08C87DF91CF91FF90EF90DF90FC
:10D3A000CF9008950E94A26961E070E080E090E073
:10D3B0000E94DBAC0E940DADAB01BC014C195D09B4
:10D3C0006E097F098D859E85B0E0A0E0481759075A
:10D3D0006A077B07C8F28C850E94CC98DACFCF927F
:10D3E000DF92EF92FF921F93CF93DF93EC017B01CB
:10D3F0006A018C85883048F40E94DA98882319F0F5
:10D400008C850E94BE9888E08C87F7018281938189
:10D41000A481B5810097A105B10551F490E080E0A9
:10D42000DF91CF911F91FF90EF90DF90CF90089503
:10D430008F3F9F4FAF4FBF4F89F370E060E081E2B5
:10D440000E941599182F8C87883040F780E591E06D
:10D450000E94D5A7A7014E5F5F4F24E030E06CE04B
:10D4600070E0812F0E94D022B601812F0E94E9989E
:10D4700064E070E0812F0E94F6930E940DAD6B0175
:10D480007C018C850E94DA98873121F18C3111F171
:10D49000882321F20E940DADAB01BC014C195D093E
:10D4A0006E097F098D859E85B0E0A0E08417950701
:10D4B000A607B70748F00E94A26961E070E080E02B
:10D4C00090E00E94DBACDDCF8C850E94CC9888E098
:10D4D0008C87A4CF81E090E0A3CF4F925F926F92B0
:10D4E0007F92AF92BF92CF92DF92EF92FF920F9313
:10D4F0001F93CF93DF93CDB7DEB76D970FB6F89438
:10D50000DEBF0FBECDBF2091830730918407FF247B
:10D51000F394232B09F403C1811149C0FF24F39430
:10D520006BEA7CE085EC9CE00E94D48A85EC9CE070
:10D530000E943E8980910A078F5F80930A07E091DD
:10D540003608F0913708309709F47EC006811781BC
:10D550000115110509F482C0D80118968C918F70BD
:10D56000853009F5C8010E94BC9F8823E1F0F801CD
:10D5700060817181CE0101960E94513BCE010196DE
:10D580000E942914882359F08A859B85009739F0D9
:10D59000DC01ED91FC910284F385E02D1995CE011B
:10D5A00001960E945F14F80102811381D1CF64EECD
:10D5B0007CE085EC9CE00E94D48A85EC9CE00E9493
:10D5C0003E890E940DAD2B013C01809130088823DB
:10D5D00051F10E940DAD9B01AC01A12CB12C650154
:10D5E00010E1E12E17E2F12E00E010E0C301B201DC
:10D5F0000E94AB26811117C00E94B98E8091340819
:10D6000090913508059741F0809136089091370840
:10D61000892B11F00E94055B0E94E55E82E090E09C
:10D620000E94F468D2CF80913008882309F476CF25
:10D6300061EC7CE08EE19CE00E94D48A8EE19CE06B
:10D640000E943E89F12C6CCF6BE97CE085EC9CE07C
:10D650000E94D48A85EC9CE00E943E8910927E074D
:10D6600010927D0763E97CE085EC9CE00E94D48AFF
:10D6700085EC9CE00E943E8964E670E080E090E0EA
:10D680000E94DBAC1092D70710922F086BE77CE06A
:10D6900085EC9CE00E94D48A0E944129AB01BC0128
:10D6A0002AE085EC9CE00E94F288809183079091AB
:10D6B0008407009711F00E94B6A61092840710927A
:10D6C0008307109233081092320810923708109294
:10D6D00036081092D9071092D80710922D08109290
:10D6E0002C08109228081092270866E77CE085EC49
:10D6F0009CE00E94D48A0E944129AB01BC012AE02F
:10D7000085EC9CE00E94F28885EC9CE00E943E89BA
:10D7100010922E0880910A07815080930A078F2D5E
:10D720006D960FB6F894DEBF0FBECDBFDF91CF91DF
:10D730001F910F91FF90EF90DF90CF90BF90AF902F
:10D740007F906F905F904F9008958F929F92BF92BD
:10D75000CF92DF92EF92FF920F931F93CF93DF93BD
:10D76000CDB7DEB7A3970FB6F894DEBF0FBECDBF1F
:10D770008091830790918407892B09F452C280918C
:10D78000300881114EC2809130088F5F809330083D
:10D7900068E172E184E19CE00E94D48A84E19CE02B
:10D7A0000E943E89009183071091840763EB75E026
:10D7B000C8010E942D9F909337088093360869EB2B
:10D7C00075E0C8010E942D9F9093D9078093D807D8
:10D7D0006BED75E0C8010E942D9F909333088093F4
:10D7E000320860EC75E0C8010E942D9F90932D08CF
:10D7F00080932C080E94F92B10927E0710927D07CF
:10D80000E0913608F0913708309709F4FAC0E680C5
:10D81000F78000913608109137080115110509F4B9
:10D82000E9C0E114F10409F4E5C0D70118968C9120
:10D830008F70853091F7C7010E94BC9F823068F3DA
:10D84000B701CE0101960E94ED21CE0101960E9402
:10D850002914882309F468C08A859B85009769F597
:10D8600070E060E0CE0101960E94281C8C01912C92
:10D87000812C97FF06C01195019511098824839486
:10D88000912CCE0101960E94321BC82ED12C898585
:10D89000853009F452C0863009F046C0B02E61E0F0
:10D8A000802F0E9483AB61E0892809F481C0CA946B
:10D8B000CD2809F081C060E07FC0DC01ED91FC91D2
:10D8C0000484F585E02D1995892B49F08A859B857F
:10D8D000DC01ED91FC910284F385E02D19958A8598
:10D8E0009B85DC01ED91FC910680F781E02D199577
:10D8F000892BD1F0CE0101960E94321B882341F082
:10D9000040E051E060E070E0CE0101960E944F3DA2
:10D910008D819E81892B41F040E052E060E070E013
:10D92000CE0101960E944F3DD7011296ED90FC90DA
:10D93000CE0101960E945F146CCFCD2829F462E0DD
:10D94000CE0101960E94011B40E051E060E070E0D2
:10D95000CE0101960E944F3D8D819E81892B41F021
:10D9600040E052E060E070E0CE0101960E944F3D41
:10D9700061E0802F0E9483AB60E0802F0E9455AB56
:10D9800060E172E185EC9CE00E94D48AB80185ECEC
:10D990009CE00E94B49F6BE072E185EC9CE00E94E9
:10D9A000D48A69E072E185EC9CE00E94D48ABCCF05
:10D9B000CA94CD2809F07FCFC62ED12C8B2D0E9482
:10D9C00055AB64E072E185EC9CE00E94D48AB8011A
:10D9D00085EC9CE00E94B49F62E072E185EC9CE0E3
:10D9E0000E94D48AB60185EC9CE00E94B49F60E05E
:10D9F00072E1D9CFF8018681978190937E07809359
:10DA00007D0785EC9CE00E943E89E0913208F09110
:10DA10003308309709F48AC0809130088F5F809373
:10DA20003008068117810115110509F47AC0D80163
:10DA300018968C918F70863009F069C01F8F0E8FF9
:10DA400070E060E0CE014E960E9461688AA19BA1C1
:10DA5000892B09F45CC08091830790918407892BFE
:10DA600009F455C0EE8CFF8CF70180858F708630ED
:10DA700099F56AEE74E0C7010E942D9F0097F1F0BE
:10DA8000DC0118962C9118972F702530B9F4169652
:10DA9000CD90DC90C114D104F9F0DA82C982B701CB
:10DAA000CE0101960E946168ED81FE811082118293
:10DAB00012821382F601C280D380ECCFFA82E9820F
:10DAC00070E060E0CE0101960E94616862E070E063
:10DAD000CE0101960E946A61EAA1FBA11082118227
:10DAE0001282138288A1843068F462E0823008F0E8
:10DAF00060E089A10E9483ABEAA1FBA18181807FC4
:10DB0000818305C0803441F060E0823431F0D80177
:10DB100012960D911C9187CF62E089A10E9483AB80
:10DB2000F6CF8091300881508093300863EF71E127
:10DB300084E19CE00E94D48A6BEE71E184E19CE078
:10DB40000E94D48A81E02091360830913708232B37
:10DB500009F480E00E94521862EE71E184E19CE0D9
:10DB60000E94D48A81E02091320830913308232B1F
:10DB700009F480E00E9452186BED71E184E19CE0B1
:10DB80000E94D48A81E020912C0830912D08232B0B
:10DB900009F480E00E94521862ED71E184E19CE09A
:10DBA0000E94D48A8091D7070E94521884E19CE099
:10DBB0000E943E896DEC71E184E19CE00E94D48A70
:10DBC0000E944129AB01BC012AE084E19CE00E9453
:10DBD000F28884E19CE00E943E8981E080932F08D6
:10DBE00081EE9BE00E946917882351F081EE9BE053
:10DBF0000E94B46984E090E09093350880933408E3
:10DC00008091340890913508079731F484E090E0D2
:10DC10009093350880933408809130088150809328
:10DC20003008A3960FB6F894DEBF0FBECDBFDF91CC
:10DC3000CF911F910F91FF90EF90DF90CF90BF9009
:10DC40009F908F900895AF92BF92DF92EF92FF92D4
:10DC50000F931F93CF93DF9300D000D0CDB7DEB7E3
:10DC60008C017B01D42EFB0184819581892BF9F0F5
:10DC7000A080B1806FE370E0C5010E9498E8009732
:10DC8000B1F09C012A193B0937FD11C050E040E07A
:10DC9000B701CE0101960E942488BE016F5F7F4FBD
:10DCA000C7010E94DA86CE0101960E94D48765ECF6
:10DCB00075E0C7010E945586882321F1F801128A78
:10DCC000118A80E090E19587848784E890E0948BC6
:10DCD000838B81E0868780E090E2908B8787D58A6E
:10DCE00081E090E026960FB6F894DEBF0FBECDBF60
:10DCF000DF91CF911F910F91FF90EF90DF90BF9038
:10DD0000AF90089562ED75E0C7010E9455868823A3
:10DD100069F0F801128A118A148A138A84E890E063
:10DD200095878487168680E090E3D7CF90E080E0E7
:10DD3000D9CFEF92FF920F931F93CF93DF9300D031
:10DD40001F92CDB7DEB78C017B01FB018485883043
:10DD5000A8F084E694E0F801918380831282138214
:10DD600014821582C8010F900F900F900F90DF91D1
:10DD7000CF911F910F91FF90EF90089580E591E072
:10DD80000E94D5A724E030E0AE014F5F5F4F6CE00A
:10DD900070E0F70184850E94FF23BE016F5F7F4F13
:10DDA000C8010E94198BDECF8F929F92AF92BF92D3
:10DDB000CF92DF92EF92FF920F931F93CF93DF9357
:10DDC000CDB7DEB7C456D1090FB6F894DEBF0FBE8B
:10DDD000CDBF84E694E02F969FAF8EAF2F976396CA
:10DDE0001CAE1DAE1EAE1FAE639765969FAF8EAF85
:10DDF000659769961CAE1DAE1EAE1FAE69976B96F9
:10DE00009FAF8EAF6B976F961CAE1DAE1EAE1FAE52
:10DE10006F97A1969FAF8EAFA197A5961CAE1DAE32
:10DE20001EAE1FAEA59767E37FE084E19CE00E94F1
:10DE3000D48A84E19CE00E943E898091F00B90910D
:10DE4000F10B8E010F5F1F4F892B09F452C00E9406
:10DE50000DA0882309F44DC082E70E94F89F8091AD
:10DE6000F00B9091F10BDC01ED91FC910088F189B0
:10DE7000E02D60E170E0199544E050E0B801809138
:10DE8000F00B9091F10B0E94C08889819A81AB813F
:10DE9000BC8163968CAF9DAFAEAFBFAF63978091EF
:10DEA000F00B9091F10BDC01ED91FC910488F58968
:10DEB000E02D199560968FAD60978823D1F08F3F44
:10DEC00079F461968FAD61978F3F51F462968FAD73
:10DED00062978F3F29F463968FAD63978F3F49F028
:10DEE0000E946CA270FF8BC180912B08833008F0D8
:10DEF00086C16BE27FE084E19CE00E94D48A0FB689
:10DF0000F894A895809160008861809360001092D9
:10DF100060000FBE8091690781112AC010925107DD
:10DF20001092500788EE93E0A0E0B0E08093520793
:10DF300090935307A0935407B09355078AE394E056
:10DF400090934F0780934E0784E694E090935D078B
:10DF500080935C0710925E0710925F071092600733
:10DF60001092610788E08093660781E080936907DB
:10DF70008BE097E090932A08809329080E9452959D
:10DF8000F12CE12C882309F4A6C080E591E00E94E1
:10DF9000D5A746E050E068EF7BE089E090E00E9482
:10DFA000919484E694E09A8389831B821C821D826B
:10DFB0001E82CE0103960E94102480912908909120
:10DFC0002A08FC0112A213A214A215A2DC0116A2B7
:10DFD00017A210A611A612A613A614A615A640EE07
:10DFE0005EE260E070E046AB57AB60AF71AF40EA15
:10DFF0005FE060E070E042AF53AF64AF75AF18967A
:10E0000026E0FD01322F11923A95E9F7AC01425F0B
:10E010005F4F34E1FA0111923A95E9F7E8EFFBE03E
:10E0200001900D922A95E1F7FC01EE5BFF4F108203
:10E030000E9472927C01019709F04DC080E591E049
:10E040000E94D5A76091290870912A08625F7F4FCE
:10E05000C8010E94198BCE0103960E941024609182
:10E06000290870912A086A5E7F4FC8010E94198BA7
:10E07000CE0103960E941E246091290870912A08FF
:10E080006E5E7F4FC8010E94198BCE0103960E94DD
:10E0900017246091290870912A08625E7F4FC80199
:10E0A0000E94198B8B819C81AD81BE818093300B46
:10E0B0009093310BA093320BB093330B0E94B6AC0C
:10E0C0007F7380912B0290912C026827792770939F
:10E0D0002C0260932B0288E199E20FB6F894A89580
:10E0E000809360000FBE90936000A895EF2809F41C
:10E0F0008CC262E87EE084E19CE00E94D48AC80180
:10E100000E944E258B819C81AD81BE8163968CAF30
:10E110009DAFAEAFBFAF639724E6E22E24E0F22EB0
:10E12000FA82E982C8010E940D2984E19CE00E94E4
:10E130003E89CE01835B9F4F0E9418A18091300BD6
:10E140009091310BA091320BB091330B8B839C8358
:10E15000AD83BE8369968CAF9DAFAEAFBFAF6997FD
:10E16000CE018D5A9F4F0E94C2A1FA82E9821B8282
:10E170001C821D821E8280E591E00E94D5A744E0AA
:10E1800050E0BE016D5F7F4F81E090E00E940694F9
:10E190008B819C81AD81BE816F968CAF9DAFAEAF00
:10E1A000BFAF6F97CE01875A9F4F0E9417A2FA8286
:10E1B000E9821B821C821D821E8280E591E00E9402
:10E1C000D5A744E050E0BE016D5F7F4F85E090E051
:10E1D0000E9406948B819C81AD81BE81A5968CAFF7
:10E1E0009DAFAEAFBFAFA597CE01815A9F4F0E94A2
:10E1F0006DA181E00E9403A310922B089CC165E1F0
:10E200007FE084E19CE00E94D48A84E694E09A83D3
:10E21000898363968CAD9DADAEADBFAD63978B83A7
:10E220009C83AD83BE83C8010E940D298091F00BB1
:10E230009091F10B892B09F4D6C10E940DA088237F
:10E2400009F4D1C182E70E94F89F8091F00B909170
:10E25000F10BDC01ED91FC910088F189E02D64E186
:10E2600070E0199544E050E0B8018091F00B909176
:10E27000F10B0E94C08889819A81AB81BC8169962B
:10E280008CAF9DAFAEAFBFAF69978091F00B90910F
:10E29000F10BDC01ED91FC910488F589E02D1995D5
:10E2A00066968FAD6697882309F49DC18F3F81F4F0
:10E2B00067968FAD67978F3F59F468968FAD6897D3
:10E2C0008F3F31F469968FAD69978F3F09F48BC109
:10E2D0006FE07FE084E19CE00E94D48A84E694E0D1
:10E2E0009A83898369968CAD9DADAEADBFAD6997BC
:10E2F0008B839C83AD83BE83C8010E940D298091CE
:10E30000F00B9091F10B892B09F44CC10E940DA0E8
:10E31000882309F447C182E70E94F89F8091F00B9F
:10E320009091F10BDC01ED91FC910088F189E02DD9
:10E3300068E170E0199544E050E0B8018091F00B7D
:10E340009091F10B0E94C08889819A81AB81BC8138
:10E350006F968CAF9DAFAEAFBFAF6F978091F00B54
:10E360009091F10BDC01ED91FC910488F589E02D91
:10E3700019956C968FAD6C97882309F413C18F3F64
:10E3800081F46D968FAD6D978F3F59F46E968FAD7A
:10E390006E978F3F31F46F968FAD6F978F3F09F473
:10E3A00001C16AE07FE084E19CE00E94D48A84E6B7
:10E3B00094E09A8389836F968CAD9DADAEADBFAD71
:10E3C0006F978B839C83AD83BE83C8010E940D2908
:10E3D0008091F00B9091F10B892B09F4AFC00E9452
:10E3E0000DA0882309F4AAC082E70E94F89F8091BB
:10E3F000F00B9091F10BDC01ED91FC910088F1891B
:10E40000E02D6CE170E0199544E050E0B801809196
:10E41000F00B9091F10B0E94C08889819A81AB81A9
:10E42000BC81A5968CAF9DAFAEAFBFAFA5978091D5
:10E43000F00B9091F10BDC01ED91FC910488F589D2
:10E44000E02D1995A2968FADA297882309F476C086
:10E450008F3F81F4A3968FADA3978F3F59F4A49675
:10E460008FADA4978F3F31F4A5968FADA5978F3FC1
:10E4700009F464C063E07FE084E19CE00E94D48AF8
:10E4800034E6E32E34E0F32EFA82E982A5968CADD1
:10E490009DADAEADBFADA5978B839C83AD83BE8391
:10E4A000C8010E940D292996FFAEEEAE2997A596C8
:10E4B0008CAD9DADAEADBFADA5972D968CAF9DAF8C
:10E4C000AEAFBFAF2D972396FFAEEEAE23976F96FC
:10E4D0008CAD9DADAEADBFAD6F9727968CAF9DAFA8
:10E4E000AEAFBFAF2797FAA2E9A269968CAD9DADFA
:10E4F000AEADBFAD69978BA39CA3ADA3BEA3FA82BB
:10E50000E98263968CAD9DADAEADBFAD63978B8355
:10E510009C83AD83BE839E01295B3F4FAE014F5B61
:10E520005F4FBE016F5D7F4FC8010E94AEA884E1BE
:10E530009CE00E943E8982E090E07AC084E694E00C
:10E5400023969FAF8EAF23976F964CAD5DAD6EADAA
:10E550007FAD6F9727964CAF5DAF6EAF7FAF2797BC
:10E560009AA389A369964CAD5DAD6EAD7FAD6997F9
:10E570004BA35CA36DA37EA39A83898363968CAD22
:10E580009DADAEADBFAD63978B839C83AD83BE83E2
:10E59000AE014F5B5F4FBE016F5D7F4FC8010E94B0
:10E5A000EDA8C5CF84E694E09AA389A369964CAD03
:10E5B0005DAD6EAD7FAD69974BA35CA36DA37EA3EC
:10E5C0009A83898363968CAD9DADAEADBFAD6397E5
:10E5D0008B839C83AD83BE83BE016F5D7F4FC8017B
:10E5E0000E943FA9A4CF84E694E09A83898363962E
:10E5F0008CAD9DADAEADBFAD63978B839C83AD837A
:10E60000BE83C8010E948AA992CF61EC7EE08EE1B0
:10E610009CE00E94D48A62E97EE08EE19CE00E9448
:10E62000D48A80912B088F5F80932B0886EF9FEF11
:10E63000909335088093340889E0EBE3F2E0D80149
:10E6400001900D928A95E1F7FE013A9687E1DF018C
:10E650001D928A95E9F78CEF9BE0009731F0AE01AF
:10E66000475F5F4F62E00E94EB11CE018F5B9F4FCF
:10E670000E944E250E940DAD683B7B4081059105AF
:10E6800038F464E670E080E090E00E94DBACF2CF0A
:10E6900027968CAD9DADAEADBFAD27978093660B31
:10E6A0009093670BA093680BB093690BC8010E940D
:10E6B00073A8892BC9F0E090620BF090630BD7012F
:10E6C000ED91FC91C088D1886DE272E0CE01819617
:10E6D0000E94198B49EE54E1BE016F5D7F4FC70167
:10E6E000F6011995811110C161E67EE08EE19CE092
:10E6F0000E94D48A8EE19CE00E943E8996E7C92E52
:10E700009BE0D92E7601B12CA12CD7018D919C9143
:10E71000892B49F1950143E050E060E070E0CB01C6
:10E720000E9430B6D701ED91FC91808591850097CC
:10E7300011F00E94EFDAD701ED91FC91868197816B
:10E74000009711F00E94EFDAD701ED91FC918481DE
:10E7500095810E94EFDAF701808191810E94EFDAC2
:10E76000D7011D921C92BFEFAB1ABB0AE2E0EE0E7E
:10E77000F11CF8E0AF16B10441F686E0EBE5F2E0FB
:10E78000DE01919601900D928A95E1F7FE01B79610
:10E790008AE1DF011D928A95E9F788EF9BE00097F7
:10E7A00031F0AE014A5D5F4F66E00E94EB116EED05
:10E7B00075E0C8010E948DE8B12CA12CF601819171
:10E7C00091916F01892B09F0A8C08AE090E00E9426
:10E7D00053DA7C01009709F4A0C0DC0119961C9261
:10E7E0001E92189715961C921E921497F80101908C
:10E7F0000020E9F7CF010197801B910B0E9453DAAB
:10E800006C01D70115969C938E931497892B09F46C
:10E81000A4C04E01B1E28B0E911CF40101900020C6
:10E82000E9F7CF010197881999090E9453DAD701B6
:10E8300019969C938E931897009709F48BC0B40196
:10E840000E94ACE880E590E0F70191838083138219
:10E850001282B801C6010E94ACE8F60101900020C6
:10E86000E9F73197CE16DF0620F4319781818E3299
:10E87000C9F76F0122E0C20ED11CD6010D90002015
:10E88000E9F7CD018C199D090B960E9453DA4C01D2
:10E89000F70197838683009741F0B6010E94ACE8A8
:10E8A00065EE75E0C4010E948DE8F501EE0FFF1FD3
:10E8B000EA58F44FF182E082950142E050E060E0D6
:10E8C00070E0CB010E9430B6019781F161EF75E0F5
:10E8D0008EE19CE00E946E8A8EE19CE00E943E895F
:10E8E000CC59DF4F0FB6F894DEBF0FBECDBFDF911E
:10E8F000CF911F910F91FF90EF90DF90CF90BF903D
:10E90000AF909F908F90089569E47EE084E19CE051
:10E910000E94D48A84E19CE0EFCEFFEFAF1ABF0AD9
:10E9200028E0A216B10409F049CFD0CF68E37EE019
:10E9300084E19CE00E94D48AB80184E19CE00E94BA
:10E940006E8A61E37EE084E19CE00E94D48A84E1E7
:10E950009CE0C4CFC6010E94EFDAD70116968D91D4
:10E960009C91009711F00E94EFDAF7018085918564
:10E97000009711F00E94EFDAC7010E94EFDAA6CFEC
:10E98000CF93DF93CDB7DEB72E970FB6F894DEBFE7
:10E990000FBECDBF809130088F5F809330086AEF43
:10E9A00076E184E19CE00E94D48A84E19CE00E94AC
:10E9B0003E891092100C10920F0C80E090E1909321
:10E9C0000B0C80930A0C84E890E09093120C8093D7
:10E9D000110C81E080930C0C80E090E290930E0C7F
:10E9E00080930D0C82E78093130C8EEF9BE00E94C6
:10E9F00022228B37910509F0BEC06CEE76E185ECE2
:10EA00009CE00E94D48A85EC9CE00E943E891C8296
:10EA10001B8281E393E09A8389838EEF9BE09E8340
:10EA20008D838FEF9FEF98878F8380E00E946D6AC0
:10EA3000CE0101960E94B7A7909384078093830725
:10EA40008EEF9BE00E94721880918307909184075B
:10EA5000892B01F560EE76E18EE19CE00E94D48A7C
:10EA60008EE19CE00E943E896FE576E0CE0109963A
:10EA70000E941388CE0109960E944AB5CE010996DC
:10EA80000E94D4878091300881508093300890E0B4
:10EA900080E019C06DEC76E184E19CE00E94D48AAC
:10EAA00084E19CE00E943E898091300881508093EF
:10EAB00030080E94A56B8091F00B9091F10B892B8F
:10EAC00059F481E090E02E960FB6F894DEBF0FBEA9
:10EAD000CDBFDF91CF9108950E940DA0882389F3C7
:10EAE00082E70E94F89F8091F00B9091F10BDC017E
:10EAF000ED91FC910088F189E02D60E670E01995B8
:10EB00006091F00B7091F10B40E0CE0109960E94EC
:10EB10009888BE01675F7F4F82EF9BE00E94DA8694
:10EB2000CE0109960E94D4878091F00B9091F10B51
:10EB3000DC01ED91FC910488F589E02D19956FEACF
:10EB400076E185EC9CE00E94D48A62EF7BE0CE0106
:10EB500009960E940A88BE01675F7F4F85EC9CE0A2
:10EB60000E94C68A85EC9CE00E943E89CE010996EF
:10EB70000E94D487A6CF8EEF9BE00E948214892B3F
:10EB8000A1F08EEF9BE00E94AC146FE576E0CE0121
:10EB900001960E941388CE0101960E944AB5CE01CB
:10EBA00001960E94D4870E94B9B58EEF9BE00E9427
:10EBB00072186CEB76E184E19CE00E94D48A84E1D7
:10EBC0009CE00E943E895ECFEF92FF920F931F93CD
:10EBD000CF93DF9300D000D0CDB7DEB78091F00B9C
:10EBE0009091F10B892B09F46CC087E70E94F89F84
:10EBF0008091F00B9091F10BDC01ED91FC9100887C
:10EC0000F189E02D70E060E0199510E000E080915E
:10EC1000F00B9091F10BDC01ED91FC9111971C969A
:10EC20002D913C910217130740F40190F081E02DE3
:10EC300060E019950F5F1F4FEACF0088F189E02D42
:10EC400070E060E0199503E813E087E8E82E83E0C0
:10EC5000F82E8091F00B9091F10BF80161918F01EA
:10EC6000DC01ED91FC910190F081E02D1995E01609
:10EC7000F10679F78091F00B9091F10BDC01ED91A9
:10EC8000FC910488F589E02D19956FE576E0CE01B9
:10EC900001960E941388CE0101960E944AB5CE01CA
:10ECA00001960E94D48787E090E00E9416A387E037
:10ECB00090E00E9420A369E772E184E19CE00E9459
:10ECC000D48A1092100C10920F0C80E090E1909377
:10ECD0000B0C80930A0C84E890E09093120C8093C4
:10ECE000110C81E080930C0C80E090E290930E0C6C
:10ECF00080930D0C82E78093130C8EEF9BE00E94B3
:10ED0000AC148EEF9BE00E94721888EC90E026967F
:10ED10000FB6F894DEBF0FBECDBFDF91CF911F912C
:10ED20000F91FF90EF900895FF920F931F93CF9351
:10ED3000DF9300D000D0CDB7DEB78C01BC01CE018F
:10ED400001960E940A88BE016F5F7F4F85EC9CE0B0
:10ED50000E94C68A85EC9CE00E943E89CE01019605
:10ED60000E94D4876BE273E1CE0101960E94DC879A
:10ED7000BE016F5F7F4FC8010E943A86F82ECE0118
:10ED800001960E94D487FF2069F0B801CE01019658
:10ED90000E940A88CE0101960E944AB5CE010196D2
:10EDA0000E94D48726960FB6F894DEBF0FBECDBF63
:10EDB000DF91CF911F910F91FF9008954F925F9235
:10EDC0006F927F928F929F92AF92BF92CF92DF927B
:10EDD000EF92FF920F931F93CF93DF93CDB7DEB7E0
:10EDE000C859D1090FB6F894DEBF0FBECDBF8E0152
:10EDF0000F5B1F4FD8011D921C92FE01ED5BFF4F70
:10EE00008EE1DF011D928A95E9F78091F00B9091D8
:10EE1000F10B892B09F4CFC10E940DA0882309F4BE
:10EE2000CAC182E70E94F89F8091F00B9091F10B8C
:10EE3000DC01ED91FC910088F189E02D60E270E049
:10EE400019954FE150E0B8018091F00B9091F10BD2
:10EE50000E9452A07C018091F00B9091F10BDC019B
:10EE6000ED91FC910488F589E02D1995E114F104E8
:10EE700009F4A1C1F801EE0DFF1D10828091FD0B78
:10EE80001F928F938091FC0B1F928F938091FB0BAD
:10EE90001F928F938091FA0B1F928F938091F90BA1
:10EEA0001F928F938091F80B1F928F9382E196E0CF
:10EEB0009F938F931F9280E48F93FE0131966F0191
:10EEC000FF93EF930E94EBE86EE074E184E19CE035
:10EED0000E94D48AB80184E19CE00E946E8AB60147
:10EEE00084E19CE00E946E8A84E19CE00E943E895D
:10EEF0007E01F1E6EF0EF11CD70113961C921E92D3
:10EF0000129788EE93E0A0E0B0E0F7018483958348
:10EF1000A683B78388E0848788EE93E09687858709
:10EF200082EE93E091838083108A1786128B018B87
:10EF3000148A138A80E590E0968B858B118E62E3AC
:10EF400073E185EC9CE00E94D48A62EF7BE0CE0105
:10EF500085589F4F0E940A88BE0165587F4F85ECF7
:10EF60009CE00E94C68A85EC9CE00E943E89CE010E
:10EF700085589F4F0E94D48761E476E0CE01835785
:10EF80009F4F0E94138861E476E0CE0185589F4F21
:10EF90000E941388BE0165587F4FCE018B579F4F4B
:10EFA0000E940A8862EF7BE0CE018B579F4F0E9440
:10EFB0007087BE0163577F4F0E947087BC01CE01EE
:10EFC0008D569F4F0E940A88CE018B579F4F0E94FB
:10EFD000D487CE0185589F4F0E94D487CE01835796
:10EFE0009F4F0E94D48783E496E0CB57DF4F9983ED
:10EFF0008883C558D040C757DF4F19821882C95837
:10F00000D040C557DF4F19821882CB58D040CD561B
:10F01000DF4F88819981C359D040C957DF4F998309
:10F020008883C758D04068E074E185EC9CE00E947A
:10F03000D48A0E944129AB01BC012AE085EC9CE006
:10F040000E94F28885EC9CE00E943E8964E670E0B4
:10F0500080E090E00E94DBAC84E996E7D70150960F
:10F060009C938E931F9769E479E88CEB91E90E9459
:10F0700096DD8C010FB6F894DEBF0FBECDBF892B95
:10F0800009F4F4C083E090E00E9453DAD8011D96A1
:10F090009C938E931C97FC01F182E0821282C7013F
:10F0A0000E946917882319F0C7010E94B469D7012B
:10F0B00053966D917C9154975596AD90BC90611587
:10F0C000710509F48FC0CE0185589F4F0E94198B9E
:10F0D000A501BE0165587F4FC7010E94EF69181650
:10F0E00019060CF0C0C0D7015196BC9051975296AA
:10F0F000AC90DF92CF928DE893E19F938F931F9313
:10F100000F930E941DDEDF92CF9288E893E19F93D8
:10F110008F931F930F930E941DDED8011C96ED91D3
:10F12000FC9181E08283DF92CF9285E893E19F9307
:10F130008F931F930F930E941DDED8011C96ED91B3
:10F14000FC911282AF92BF928FE493E19F938F93D1
:10F150001F930F930E941DDE0FB6F894DEBF0FBE03
:10F16000CDBFB12C86E4C82E83E1D82E8B2D94E040
:10F170008902F0011124A5E8B0E0AC0FBD1FEA0F31
:10F18000FB1F808191810097A9F122813381211594
:10F190003105C9F33F932F939F938F93DF92CF92C3
:10F1A0001F930F930E941DDEB3940FB6F894DEBF39
:10F1B0000FBECDBFDBCF40E250E060E474E1C80198
:10F1C0000E94C3DC62E274E184E19CE00E94D48A84
:10F1D000B80184E19CE00E946E8A84E19CE00E9478
:10F1E0003E894CCEF70161897289A501C7010E9451
:10F1F0008B1775CF8AE893E19F938F931F930F939B
:10F200000E941DDED70158961C921E925797D80176
:10F210001C96ED91FC91C080D1800F900F900F90C3
:10F220000F9033E3A32EB12CD601ED91FC91008415
:10F23000F185E02DC601199541975CF4B1E0AB1A58
:10F24000B10839F064E170E080E090E00E94DBAC4E
:10F25000EBCFD601ED91FC910084F185E02DC60144
:10F260001995419734F4C8010E94959110E000E08F
:10F270005AC06FE576E0CE0183579F4F0E941388F6
:10F28000912CA12CD601ED91FC910688F789E02DF7
:10F29000C60119958823E1F1BDE0AB1201C0A92C8C
:10F2A000D601ED91FC910688F789E02DC6011995EC
:10F2B0008111D4C0D601ED91FC910084F185E02D3F
:10F2C000C6011995892B09F4DBC0D601ED91FC919B
:10F2D0000284F385E02DC6011995B82EBAE08B178C
:10F2E00009F4D0C0EDE08E1709F4CCC0FFEF8F1702
:10F2F00009F4C6C0682FCE0183579F4F0E94C6866F
:10F300009A2CAB2CBFCFBAE0BB12FACFAB12F8CF1E
:10F31000CC24C394D12CCE0183579F4F0E94D48715
:10F32000CD2809F4A3CFD7015796ED90FC906AEF52
:10F3300073E185EC9CE00E94D48AB70185EC9CE0E7
:10F340000E94B49F85EC9CE00E943E8964E670E0D8
:10F3500080E090E00E94DBAC0115110509F451C179
:10F36000B8ECEB16F10409F02AC16EEE73E184E10A
:10F370009CE00E94D48A64EF71E080E090E00E94FB
:10F38000DBACEF961FAE1EAEEF97C158DF4F198270
:10F390001882CF57D0408FEF9FEFCF57DF4F998321
:10F3A0008883C158D0408BE193E0ED969FAF8EAF3C
:10F3B000ED97CD57DF4F19830883C358D040F89499
:10F3C00081E00E946D6ACE0185589F4F0E94B7A7C9
:10F3D00090938407809383077894C8010E94959145
:10F3E0008091830790918407892B09F0D6C06FE53F
:10F3F00076E0CE0183579F4F0E941388CE0183573A
:10F400009F4F0E944AB5CE0183579F4F0E94D487D9
:10F4100067ED73E18EE19CE00E94D48AF12CE12C2F
:10F42000CE018D569F4F0E94D487C701C856DF4F2B
:10F430000FB6F894DEBF0FBECDBFDF91CF911F9105
:10F440000F91FF90EF90DF90CF90BF90AF909F9083
:10F450008F907F906F905F904F900895D601ED91BF
:10F46000FC910084F185E02DC6011995892B09F0E6
:10F4700021CF64E670E080E090E00E94DBAC10CF2A
:10F48000BB24BA9461E576E088E29CE00E946E8A33
:10F49000BE0163577F4F88E29CE00E94C68A88E2E3
:10F4A0009CE00E943E896DE373E1CE0185589F4F39
:10F4B0000E94DC87BE0165587F4FCE0183579F4F66
:10F4C0000E943A86982ECE0185589F4F0E94D4877D
:10F4D000992099F1CF56DF4F28813981C159D04009
:10F4E00049E050E0BE0163577F4FCE0185589F4FE2
:10F4F0000E942488ED968EAD9FADED97412C512C46
:10F500003201009719F00E943EDC2B014201CE012E
:10F5100085589F4F0E94D4874114510429F0D70188
:10F5200058965C924E925797B40188E29CE00E94F4
:10F53000B49F88E29CE00E943E89F701878490880E
:10F5400081149104D1F0CF56DF4F88819981C15940
:10F55000D040892B91F0BE0163577F4FCE01855873
:10F560009F4F0E940A88CE0185589F4FF40119953C
:10F57000CE0185589F4F0E94D4876FE576E0CE017B
:10F5800083579F4F0E94A487FFEFBF12BCCEC801D4
:10F590000E949591D12CC12CBECE0E94A56B80916A
:10F5A0002F08882329F00E946CA267FF0E944D1D3E
:10F5B00060ED73E184E19CE00E94D48A31CFE0E306
:10F5C000EE16E1E0FE0651F46CEB73E184E19CE0A1
:10F5D0000E94D48AC8010E94959122CF64EA73E107
:10F5E0008EE19CE00E94D48AC8010E949591B701E7
:10F5F0008EE19CE00E94B49F8EE19CE00E943E89D7
:10F600000FCF61E973E185EC9CE00E94D48AEE247F
:10F61000EA94FE2C05CF0F931F93CF93DF93EB015A
:10F6200002970CF485C00A811B8164E273E1C80172
:10F630000E946EDC892B51F481E00E940CA388ECBF
:10F6400090E0DF91CF911F910F91089560E273E1F7
:10F65000C8010E946EDC892B11F480E0EECF60E0DF
:10F6600073E184E19CE00E94D48A0E946CA263FB57
:10F67000662760F981E0682770E084E19CE00E94E1
:10F68000B49F84E19CE00E943E898091F00B9091B0
:10F69000F10B892BE9F10A811B810E940DA08823BF
:10F6A000B9F1F80101900020E9F73197E01BF10B67
:10F6B000B09770F582E70E94F89F8091F00B9091CF
:10F6C000F10BDC01ED91FC910088F189E02D60E205
:10F6D00070E01995B8018091F00B9091F10B0E94A8
:10F6E0006E8A8091F00B9091F10BDC01ED91FC9111
:10F6F0000190F081E02D60E019958091F00B9091E0
:10F70000F10BDC01ED91FC910488F589E02D199550
:10F710006A817B8184E19CE00E946E8A69EF72E1DC
:10F7200084E19CE00E94D48A84E19CE00E943E89AE
:10F73000809134089091350802977CF10E94DE7622
:10F74000883C910539F424E030E03093350820936B
:10F75000340877CF8F3F9807C9F46EED72E185ECDE
:10F760009CE00E94D48A85EC9CE00E943E89109225
:10F770002E0883E090E0909335088093340881EE62
:10F780009BE00E94B46989EC90E05BCF20912F0848
:10F790002111D9CF2FE030E0D8CF61ED72E18EE1B9
:10F7A0009CE00E94D48A8EE19CE00E943E8984EF16
:10F7B00091E047CF5F926F927F928F929F92AF922C
:10F7C000BF92CF92DF92EF92FF920F931F93CF934E
:10F7D000DF93CDB7DEB7CF56D1090FB6F894DEBFB1
:10F7E0000FBECDBF4C018B01F42E4AE050E06F2DCF
:10F7F00085EC9CE00E94428966E97DE085EC9CE016
:10F800000E94D48AB801CE0101965C010E940A8848
:10F81000B50185EC9CE00E94C68A85EC9CE00E94C4
:10F820003E89C5010E94D48792E0F9126BC264E957
:10F830007DE0C5010E94DC87B501C8010E946A868F
:10F84000F82EC5010E94D487FF2009F4D0C220E021
:10F850004DE251E0B4018FEB9BE00E94168EE090E8
:10F860002708F09028086DE87DE0CE0186599F4F6B
:10F870000E94DC8766E87DE0CE018C599F4F0E9494
:10F88000DC87CE01885A9F4F0E944E256E961FAD91
:10F890006E976D960FAD6D976C96DFAC6C976B960F
:10F8A000CFAC6B976FE576E0CE0181960E9413880E
:10F8B000BE016F5D7F4FC5010E940A886C2DC50196
:10F8C0000E94258764E576E00E9456876D2D0E9490
:10F8D000258764E576E00E945687602F0E94258781
:10F8E00064E576E00E945687612F0E942587BC015F
:10F8F000CE01825A9F4F0E940A88C5010E94D48778
:10F90000CE0181960E94D48761E87DE0CE018E5AB7
:10F910009F4F0E94DC876FE576E0CE01845B9F4FAE
:10F920000E94138800EF1BE0D80118966C9170E0DC
:10F9300084E0759567958A95E1F7C5010E94CC9F93
:10F940004D815E8169817A81CE01845B9F4F0E94E7
:10F950009A86C5010E94D487F80160856F7070E0B7
:10F96000C5010E94CC9F4D815E8169817A81CE0163
:10F97000845B9F4F0E949A86C5010E94D4870F5FC7
:10F980001F4FFBE0063F1F0779F66BE77DE0CE01D6
:10F990008A5B9F4F0E94DC876AE57DE0CE018196FD
:10F9A0000E94DC87BE016F5D7F4FCE01CE960E9424
:10F9B0000A88BE016A5B7F4FCE01CE960E94708797
:10F9C000BE01645B7F4F0E947087BE016E5A7F4FFD
:10F9D0000E947087BE01625A7F4F0E947087BE01ED
:10F9E0006C597F4F0E9470878C014AE0B50180E519
:10F9F00090E00E9408DDF50101900020E9F73197C1
:10FA0000AF014A195B09B501C8010E949A868111AC
:10FA100003C0C8010E941387BE0166597F4FC80109
:10FA20000E947087B7010E945687BC01C4010E94E2
:10FA3000C68AC4010E943E89CE01CE960E94D48718
:10FA4000CE0181960E94D487CE018A5B9F4F0E948F
:10FA5000D487CE01845B9F4F0E94D487CE018E5AFB
:10FA60009F4F0E94D487CE01825A9F4F0E94D48715
:10FA7000CE018C599F4F0E94D487CE0186599F4F4B
:10FA80000E94D487C4010E943E8964E670E080E051
:10FA900090E00E94DBACD401ED91FC910488F589E3
:10FAA000E02DC401199501E010E088C028966EADE4
:10FAB0007FAD2897CE0181960E94ECA3892B09F493
:10FAC00050C122961CAE1DAE1EAE1FAE22972696CA
:10FAD0001CAE1DAE1EAE1FAE26978FAD8F708FAFC2
:10FAE00040E053E0BE016F5D7F4FCE01CE960E9495
:10FAF000CB3000E020E033E040E250E0B501CE0141
:10FB0000CE960E94A02DBC01C6010E94AE8708ECD3
:10FB100010E129C1EE2009F4F3C046E050E070E0A6
:10FB200060E0C8010E94D785D8016D917C91CE011B
:10FB300081960E94513BCE0181960E94291400E9D2
:10FB400011E08823B9F189A5873061F4CE0181964F
:10FB50000E94985C61E0892B09F462E0CE018196F5
:10FB60000E94011B22961CAE1DAE1EAE1FAE229738
:10FB700026961CAE1DAE1EAE1FAE26978FAD8F70A3
:10FB80008FAF40E053E0BE016F5D7F4FCE01CE9658
:10FB90000E94CB3000E020E033E040E250E0B501CD
:10FBA000CE01CE960E94A02DBC01C6010E94AE8758
:10FBB00008EC10E1CE0181960E945F14C801C15982
:10FBC000DF4F0FB6F894DEBF0FBECDBFDF91CF91F0
:10FBD0001F910F91FF90EF90DF90CF90BF90AF906B
:10FBE0009F908F907F906F905F900895F801608153
:10FBF00071810E942D9F7C01892B09F040C104E98D
:10FC000011E0DCCFEE2009F47BC049E050E070E069
:10FC100060E0C8010E94D7854AE0B401C5010E9496
:10FC2000988841E050E067E974E0C8010E949A8634
:10FC30004D815E8169817A81C8010E949A8666E35E
:10FC40007DE085EC9CE00E94D48AB801CE018196CB
:10FC50000E940A88BE016F5D7F4F85EC9CE00E9488
:10FC6000C68A85EC9CE00E943E89CE0181960E9466
:10FC7000D4876EE27DE0CE0181960E94DC87F80198
:10FC8000848195812DA13EA182179307E1F4892BF0
:10FC9000A1F1E080F18069A07AA0D7018D917D016A
:10FCA000882359F1082E000C990B0E9428E86C015A
:10FCB000F30181913F01082E000C990B0E9428E866
:10FCC000C816D90651F3CE0181960E94D4875520DB
:10FCD00041F021E048EC50E0B4018FEB9BE00E9442
:10FCE000168ED8018D919C910E94448E009711F43C
:10FCF00084E991E08C01C5013DC055245394E3CFC4
:10FD000001E97ECFB1E0FB1270C063E57DE0C50183
:10FD10000E94DC87B501C8010E943A86582EC501B1
:10FD20000E94D487552049F1EE2051F346E050E07F
:10FD300070E060E0C8010E94D7854AE0B401CE01BE
:10FD40008A5B9F4F0E949888F80160817181CE0183
:10FD500081960E94513BCE0181960E942914811107
:10FD6000A5CE00E911E0CE0181960E945F14CE017C
:10FD70008A5B9F4F0E94D48721CF6CE37DE0C50151
:10FD80000E94DC87B501C8010E943A86F82EC501A1
:10FD90000E94D487F11036CF61E27DE0C5010E9458
:10FDA000DC87B501C8010E943A86182FC5010E9460
:10FDB000D48700E0112309F401CF80E00E940CA356
:10FDC00069EF7CE084E19CE00E94D48A84E19CE0BD
:10FDD0000E943E896FE576E0C5010E941388C50147
:10FDE0000E944AB5C5010E94D48700E05DCE6CE454
:10FDF0007DE0C5010E94DC87B501C8010E943A86FA
:10FE0000F82EC5010E94D487F11084CE66E47DE00F
:10FE1000C5010E94DC87B501C8010E943A86F82E10
:10FE2000C5010E94D487FF2001F3EE2009F468CFBA
:10FE300045E050E070E060E0C8010E94D78564E5CD
:10FE400076E0C8010E945586882339F0E090360894
:10FE5000F0903708E114F10491F46FE576E0C80101
:10FE60000E945586811107C080913608909137080D
:10FE7000009709F0BBCEE0908307F090840720E064
:10FE800048EC50E2B4018FEB9BE00E94168EC40157
:10FE90000E943E891C821B8281E393E09A838983BE
:10FEA0009E828D828FEF9FEF98878F83B701C50168
:10FEB0000E947A8FEACD0895FC0124813581621772
:10FEC000730748F480819181009729F0860F971F6E
:10FED000FC018081089580E008950895AF92BF925B
:10FEE000CF92DF92EF92FF920F931F93CF93DF9306
:10FEF0006C017B018B01040F151FEB015E01AE1835
:10FF0000BF08C017D10759F06991D601ED91FC9156
:10FF10000190F081E02DC6011995892B79F7C50173
:10FF2000DF91CF911F910F91FF90EF90DF90CF90D5
:10FF3000BF90AF900895FC01A089B1898C91A689EA
:10FF4000B78982FD0FC09C91818D8F5F8F73228D49
:10FF5000821749F0A18DAE0FBF2FB11D5D969C9306
:10FF6000818F08958C910895FC01538D448D252F28
:10FF700030E0842F90E0821B930B541710F0CF9643
:10FF8000089501970895FC01918D828D981761F075
:10FF9000A28DAE0FBF2FB11D5D968C91928D9F5F8C
:10FFA0009F73928F90E008958FEF9FEF0895FC016B
:10FFB000918D828D981731F0828DE80FF11D858D1E
:10FFC00090E008958FEF9FEF0895FC01918D228DB1
:10FFD000892F90E0805C9F4F821B91098F73992736
:10FFE000089582E399E00E94E57F21E0892B09F4DE
:10FFF00020E0822F08958FEC99E00E94E57F21E0B8
:020000021000EC
:10000000892B09F420E0822F08958CE69AE00E9463
:10001000E57F21E0892B09F420E0822F089588E212
:100020009CE00E94E57F21E0892B09F420E0822FEB
:100030000895FC01A48DA80FB92FB11DA35ABF4F7D
:100040002C91848D90E001968F739927848FA689D7
:10005000B7892C93A089B1898C91837080648C932B
:10006000938D848D981306C00288F389E02D8081DA
:100070008F7D80830895EF92FF920F931F93CF930C
:10008000DF93EC0181E0888F9B8D8C8D98131AC0D3
:10009000E889F989808185FF15C09FB7F894EE89BA
:1000A000FF896083E889F989808183708064808317
:1000B0009FBF81E090E0DF91CF911F910F91FF9062
:1000C000EF900895F62E0B8D10E00F5F1F4F0F730A
:1000D0001127E02E8C8D8E110CC00FB607FCFACFC5
:1000E000E889F989808185FFF5CFCE010E941980CA
:1000F000F1CFEB8DEC0FFD2FF11DE35AFF4FF08296
:100100009FB7F8940B8FEA89FB8980818062CFCFFB
:10011000CF93DF93EC01888D8823B9F0AA89BB893E
:10012000E889F9898C9185FD03C0808186FD0DC029
:100130000FB607FCF7CF8C9185FFF2CF808185FF4A
:10014000EDCFCE010E941980E9CFDF91CF910895C4
:1001500080E090E0892B29F00E940F8081110E949D
:10016000000080E090E0892B29F00E940580811139
:100170000E94000080E090E0892B29F00E94FB7F24
:1001800081110E94000080E090E0892B29F00E94FC
:10019000F17F81110C94000008950F931F93FC01CF
:1001A00062857385848595850281138124813581DB
:1001B000601B710B820B930B068517852089318993
:1001C000601B710B820B930B1F910F910895DC0143
:1001D000ED91FC910190F081E02D19948FEF9FEF4C
:1001E0000895FC0162897389848995890895EF9245
:1001F0000F931F93CF93DF93FC01248D222341F0B3
:10020000213051F1DF91CF911F910F91EF9008951F
:10021000228933894489558986899789A08DB18D32
:10022000821B930BA40BB50B892F9A2FAB2FBB27E7
:100230008C010F5F1F4F6281738184819581CFB7DD
:10024000F894DCB7E1E0ECBFEE24E394E2E0FEEFEB
:100250001995DCBFCFBFD6CFF0E0E0E0DF91CF91C2
:100260001F910F91EF901994FC01138E128E411182
:100270000CC082899389A489B589868B978BA08FBE
:10028000B18F148E81E090E0089590E080E00895B1
:10029000CF92DF92EF92FF92CF93DF93DC01CB01FD
:1002A000642FCFB7F8946D01EE24FF24CBBEDCB7EA
:1002B00041E04CBFA901E1E0FEEF1995DCBFCFBFE3
:1002C000DF91CF91FF90EF90DF90CF900895CF9383
:1002D000DF93FC01248D211110C0EC01828D938DE0
:1002E000892B49F066897789808D918D30E020E0F7
:1002F00045E00E9448811B8E1A8EDF91CF910895B0
:100300001F93CF93DF93FC01248D211145C0162F3D
:10031000EC01828D938D892B49F466897789808DD4
:10032000918D30E020E043E00E9448814A8D5B8D52
:10033000CA0181709927FE01E80FF91F158F892BDB
:1003400069F02D8D3E8D6E897F89888D998D640F22
:10035000751F811D911D41E00E9448818A8D9B8DF2
:1003600001969B8F8A8F81159140B1F46E897F89A8
:10037000888D998D30E020E045E00E9448811B8EF9
:100380001A8E8E899F89A88DB98D9F5FAF4FBF4F01
:100390008E8B9F8BA88FB98F81E090E0DF91CF91FA
:1003A0001F910895DC01ED91FC910280F381E02D15
:1003B00040E01994FB014481558122813381215011
:1003C00031094217530750F4A081B181A40FB51F22
:1003D0008C938481958101969583848380E0089530
:1003E000CF93DF93EC01E881F9810284F385E02D5E
:1003F000CE0119950196B9F7DF91CF910895CF926B
:10040000DF92EF92FF920F931F93CF93DF937C01C4
:100410006A018B01D0E0C0E0CC15DD0581F0D70189
:10042000ED91FC910284F385E02DC70119958F3F72
:10043000980729F0F80181938F012196EDCFCE0125
:10044000DF91CF911F910F91FF90EF90DF90CF90B0
:100450000895CF93C62FDC01ED91FC910088F189BE
:10046000E02D1995DC01ED91FC910190F081E02DDA
:100470006C2FCF911994062E000C770BFC0177831B
:1004800066830895CF93DF93EC018E819F8101965F
:1004900011F5E881F9810088F189E02DCE011995E7
:1004A000DC01ED91FC910084F185E02D1995892BFB
:1004B000B1F0E881F9810284F385E02DCE01199530
:1004C0008132910534F3E881F9810684F785E02DC6
:1004D000682FCE01199581E0DF91CF91089580E0DA
:1004E000FBCFFC0120812EBD9B012150310941F041
:1004F00051810DB407FEFDCF4EB55EBD4193F5CFE2
:1005000061507109860F971F0DB407FEFDCF2EB500
:10051000FC0120830895E0913908F0913A08808128
:1005200090913808892B80830895E0913908F091E3
:100530003A089081809138088095892380830895B6
:100540008EBD00000DB407FEFDCF8EB5089590E07E
:1005500020911E09233339F40C96982F990F990F87
:10056000990F80E008954896F8CFEF92FF920F938D
:100570001F93CF93DF93EC018B017A010E940DADA5
:10058000688B798B8A8B9B8B8C819D81DC01ED91B3
:10059000FC910280F381E02DA701B801DF91CF919A
:1005A0001F910F91FF90EF9019941F93CF93DF93BA
:1005B000EC01162F0E940DAD688B798B8A8B9B8B7B
:1005C0008C819D81DC01ED91FC910190F081E02D09
:1005D000612FDF91CF911F911994CF92DF92EF920B
:1005E000FF92CF93DF93EC018E819F818F3F98071D
:1005F00059F02FEF3FEF3F832E83DF91CF91FF9094
:10060000EF90DF90CF9008950E940DAD6B017C01BB
:10061000A4EFCA0EA1E0DA1EE11CF11CE881F98109
:100620000088F189E02DCE011995DC01ED91FC9156
:100630000084F185E02D1995892B39F40E940DADC8
:100640006C157D058E059F0548F3E881F9810088CA
:10065000F189E02DCE011995DC01ED91FC91028428
:10066000F385E02DDF91CF91FF90EF90DF90CF9059
:1006700019940E9423E80F931F93CF93DF93D0E048
:10068000C0E0009791F08C01CDE7D8E068817981D6
:100690006115710529F0C8010E94A3E8892B29F092
:1006A0000B80DC81C02D209789F7CE01DF91CF919F
:1006B0001F910F910895CF92DF92EF92FF920F93C7
:1006C0001F93CF93DF936C018B0186E090E00E9433
:1006D00053DAEC019093BF088093BE08F6010190B5
:1006E0000020E9F7CF018C199D090E9453DA7C01A3
:1006F000B6010E94ACE8F60101900020E9F73197BD
:10070000EC19FD09EE0DFF1D1082F982E8821B83B2
:100710000A838091C0089091C1089D838C83D093F7
:10072000C108C093C008DF91CF911F910F91FF9036
:10073000EF90DF90CF9008950F931F93CF93DF93A7
:10074000EC0188819981009759F02A813B81261715
:10075000370730F081E0DF91CF911F910F9108951D
:100760008B016F5F7F4F0E9442E7009759F099839A
:1007700088831B830A832C813D81232B59F7FC013D
:100780001082E8CF80E0E7CFFC01868197818F3F20
:10079000980729F02FEF3FEF378326830895808550
:1007A00091850C94E1DD7F928F929F92AF92BF92E0
:1007B000CF92DF92EF92FF920F931F93CF93DF932D
:1007C000CDB7DEB7A6970FB6F894DEBF0FBECDBF8C
:1007D0008C01762E942E852E20E2A22ECE0101963B
:1007E0007C01DC01EA2D1D92EA95E9F76801F3E44A
:1007F000CF0ED11C84E694E09AA389A38FEF8BA33C
:100800008CA38DA38EA343E450E0BE016F5D7F4FA8
:10081000C6010E949124019609F4BFC081E089833A
:100820008A8386E0B82EBB821C82D80114966D9113
:100830007D918D919C9117970E944AE46D837E83F0
:100840008F83988789869A8680E890E09C878B873B
:100850004CE150E0B701C6010E942624FE01379604
:100860008AE1DF011D928A95E9F74801B8E08B0E15
:10087000911CF401D70101900D92BA94E1F740E187
:1008800050E0B701C6010E942624F7011192AA94F4
:10089000E9F796E0A92EB12C40E250E0B701C6017D
:1008A0000E942624F1E0AF1AB108B1F783E68983EC
:1008B00092E89A8393E59B838C8385E38D8381E023
:1008C0008E837F829DE3988797E099878A8786E069
:1008D000F401DE011B9601900D928A95E1F78CE000
:1008E000898B8A8B66E576E0CE0143960E94ACE860
:1008F000D8011B966C91CE0149960E9461A8F8011F
:100900006485CE014B960E9461A8D8011D966C911A
:10091000CE014D960E9461A84EE150E0B701C6019C
:100920000E942624B3E07B121EC082E3898384E008
:100930008A83F80196859B8397859C8390899D8304
:1009400091899E8396E39F838887828D8987838D93
:100950008A87848D8B87858D8C874CE050E0B7012A
:10096000C6010E94262487E3898386E08A8391E07A
:100970009B8393E09C838D838FE08E838AE38F83B8
:100980008BE388878FEF898749E050E0B701C60184
:100990000E942624C6010E946024A6960FB6F894F1
:1009A000DEBF0FBECDBFDF91CF911F910F91FF90A2
:1009B000EF90DF90CF90BF90AF909F908F907F90FF
:1009C000089590E080E00C94FE22CF93DF93C4E181
:1009D000D0E00E94E184882361F061E070E080E073
:1009E00090E00E94DBAC2197A1F780E0DF91CF91EE
:1009F000089581E0FBCFFF920F931F93CF93DF9376
:100A00001F921F92CDB7DEB7F82E22E030E0AE0184
:100A10004F5F5F4F66E270E00E94FF2309811A81F9
:100A200010270127102722E030E0AE014F5F5F4F13
:100A300066E270E08F2D0E94FF2389819A819827BA
:100A4000892798270817190749F4C8010F900F90B4
:100A5000DF91CF911F910F91FF9008958C01E3CF0B
:100A60001F920F920FB60F9211242F933F938F93E3
:100A70009F93AF93BF938091CE089091CF08A091A0
:100A8000D008B091D1083091CD0823E0230F2D3745
:100A900068F126E8230F0296A11DB11D2093CD0811
:100AA0008093CE089093CF08A093D008B093D1083C
:100AB0008091D2089091D308A091D408B091D50824
:100AC0000196A11DB11D8093D2089093D308A093E5
:100AD000D408B093D508BF91AF919F918F913F916A
:100AE0002F910F900FBE0F901F9018950196A11D8A
:100AF000B11DD4CFAF92BF92CF92DF92EF92FF920F
:100B00000F931F93CF93DF93DC01CD90DC9011976F
:100B1000C114D10439F01496CD91DC918C01760189
:100B2000209761F4DF91CF911F910F91FF90EF908B
:100B3000DF90CF90BF90AF90089575015701BFEF40
:100B4000AB1ABB0AF7018081082E000C990B0E949A
:100B500065DC892B91F72197CC0DDD1D8881082E4E
:100B6000000C990B0E9465DC892B29F0CE15DF055E
:100B700010F02197F3CFAE014F5F5F4F4E195F0921
:100B8000D80115965C934E931497CE14DF0420F48D
:100B9000B701C6010E945FE8D801ED91FC91119761
:100BA00014968D919C91E80FF91F1082BBCFCF93C3
:100BB000DF93DC011496ED91FC916E177F0728F509
:100BC0004115510511F19F01261B370B42175307A1
:100BD00008F49A01DB01EC0188819981E21BF30B97
:100BE000FD83EC83AF01461B570B260F371FBC015B
:100BF000620F731F8A0F9B1F0E94D1E8E881F98161
:100C00008C819D81E80FF91F1082DF91CF910895AB
:100C1000DF92EF92FF920F931F93CF93DF93FC012C
:100C2000E480F580E114F10451F48FEF9FEFDF9140
:100C3000CF911F910F91FF90EF90DF900895EC01FD
:100C40000190F081E02DEE0DFF1DD0801082088113
:100C50001981062E000C770BC8010E94E0E80E0DEA
:100C60001F1DF801D082009701F328813981821B72
:100C7000930BDDCFFB0144815581FC01248135813B
:100C80002417350778F080819181009759F0FB0196
:100C9000608171816115710529F00E94C3E821E02E
:100CA000892B09F020E0822F0895FC0124813581F1
:100CB000232B39F421E0FB018081882349F020E0D7
:100CC00007C0808191810E94A3E821E0892BB9F7B8
:100CD000822F0895FC0124813581FB0144815581D7
:100CE00024173507E1F4FC0180819181FB016081CB
:100CF00071810097D1F061157105A1F4232BC1F02A
:100D0000FC01808190E008C0232B91F0FB018081E1
:100D100090E091958195910921E0892B09F020E0DF
:100D2000822F08950E94A3E8F7CF6115710561F73E
:100D300021E0F6CFEF92FF920F931F93CF93DF93B3
:100D40006115710541F480E0DF91CF911F910F9102
:100D5000FF90EF90089541155105B1F07B01EC0132
:100D60000C811D81040F151FB8010E949C838823EC
:100D700051F3288139818C819D81B701820F931FA6
:100D80000E94ACE81D830C8381E0DECFCF93DF931C
:100D90001F921F92CDB7DEB769831A8241E050E0FF
:100DA000BE016F5F7F4F0E949A860F900F90DF9178
:100DB000CF9108950F931F93CF93DF938C01EB0195
:100DC000FC01808191810097E1F068817981611552
:100DD0007105A9F0428153812C813D81421753074F
:100DE00070F00E94ACE88C819D81F801958384832A
:100DF0001D821C82DF91CF911F910F9108950E9457
:100E0000EFDA88819981F801918380838A819B81BF
:100E1000938382838C819D81958384831982188238
:100E20001B821A82E5CFCF93DF93EC0188819981F1
:100E3000009711F00E94EFDA198218821D821C823D
:100E40001B821A82DF91CF910895EF92FF920F9348
:100E50001F93CF93DF9300D01F92CDB7DEB77C01F5
:100E6000862F4AE08E010F5F1F4FB80190E00E946D
:100E700008DDF80101900020E9F73197AF01401B30
:100E8000510BB801C7010E949A86811103C0C701A6
:100E90000E941387C7010F900F900F900F90DF9162
:100EA000CF911F910F91FF90EF900895CF93DF9313
:100EB000EC016115710539F4CE010E941387CE0152
:100EC000DF91CF910895FB0101900020E9F7319760
:100ED000AF01461B570B0E949A86882369F3EFCF18
:100EE000CF93DF93EC01FB014481558160817181D7
:100EF0000E949A86811103C0CE010E941387CE0101
:100F0000DF91CF910895EF92FF920F931F93CF93AC
:100F1000DF93EC017B018A01BA010E949C8381115D
:100F20000BC0CE010E941387CE01DF91CF911F919C
:100F30000F91FF90EF9008951D830C83B701888176
:100F400099810E94ACE8F0CFFB0101900020E9F705
:100F50003197AF01461B570B0C948387CF93DF93D8
:100F6000EC016115710531F00E94A487CE01DF917B
:100F7000CF9108950E941387F9CFCF93DF93EC01AF
:100F8000FB018617970749F0608171816115710532
:100F900041F0448155810E948387CE01DF91CF913A
:100FA00008950E941387F9CFFC01808191810097F9
:100FB00011F00C94EFDA0895EF92FF920F931F93C4
:100FC000CF93DF93EC018B01198218821B821A8266
:100FD0001D821C82CB010E949CDC7C01BC01CE01E5
:100FE0000E949C83811109C0CE01DF91CF911F9196
:100FF0000F91FF90EF900C941387FD82EC82B80163
:1010000088819981DF91CF911F910F91FF90EF908F
:101010000C9495DCFC0111821082138212821582DD
:1010200014820C94BD87FC011182108213821282FB
:1010300015821482FB0101900020E9F73197AF017E
:10104000461B570B0C948387AF92BF92CF92DF92CF
:10105000EF92FF920F931F93CF93DF935C016B018D
:101060007A0189012417350720F48F2D7901042F87
:10107000182F6FE576E0C5010E941388D6011496FB
:10108000CD91DC91EC16FD06C8F40C171D0708F491
:10109000E801D601ED91FC911197EC0FFD1F108135
:1010A00010826D917C916E0D7F1DC5010E94AE87EF
:1010B000F60180819181C80FD91F1883C501DF9186
:1010C000CF911F910F91FF90EF90DF90CF90BF9045
:1010D000AF9008950F931F93CF93DF93EC010E947D
:1010E0000DAD688779878A879B87E881F9810284BB
:1010F000F385E02DCE01199597FF15C00E940DAD27
:10110000088519852A853B85601B710B820B930B23
:101110000C811D812E813F81601771078207930723
:1011200020F38FEF9FEFDF91CF911F910F910895E3
:10113000EF92FF920F931F93CF93DF93EC017B010C
:10114000042F6FE576E00E941388C7010E946A8829
:10115000002E000C110B97FD0BC00817190741F06A
:10116000682FCE010E94C686C7010E946A88F3CF0D
:10117000CE01DF91CF911F910F91FF90EF900895D5
:10118000CF92DF92EF92FF920F931F93CF93DF9353
:101190006C017A018B01D0E0C0E0C6010E946A8830
:1011A00097FD07C0F80181938F012196EC16FD068B
:1011B000A1F7CE01DF91CF911F910F91FF90EF909A
:1011C000DF90CF900895FB0101900020E9F731975F
:1011D000AF01461B570BDC01ED91FC910280F381BE
:1011E000E02D19948F929F92AF92BF92EF92FF924F
:1011F0000F931F93CF93DF93CDB7DEB7A1970FB6B1
:10120000F894DEBF0FBECDBF7C01FA01CB0119A25D
:10121000223008F42AE08E010F5D1F4F822E912CA0
:10122000B12CA12CBF01A50194010E94CBE3F901CF
:10123000CA016A300CF5605DD8016E938D01232BD5
:10124000242B252B79F790E080E0109721F0BD0149
:10125000C7010E94E388A1960FB6F894DEBF0FBEC7
:10126000CDBFDF91CF911F910F91FF90EF90BF9075
:10127000AF909F908F900895695CDECF6DE576E02A
:101280000C94E388242F462F50E070E060E00C942B
:10129000F288EF92FF920F931F93CF93DF93009703
:1012A00051F4CFEFDFEFCE01DF91CF911F910F917E
:1012B000FF90EF900895DC011C96ED90FC90F701F3
:1012C00000811181D801ED91FC910688F789E02D0C
:1012D000C8011995882329F3D801ED91FC91008468
:1012E000F185E02DC8011995D801ED91FC91892B6C
:1012F00061F30284F385E02DC8011995EC01019694
:1013000081F2F801818D882339F04AE050E06C2F9A
:1013100088E29CE00E944289D70112968C91882332
:1013200011F2C532D10509F0BECFD801ED91FC9183
:101330000084F185E02DC801199502975CF0D80171
:10134000ED91FC910688F789E02DC801199581116E
:10135000ECCFA7CFD1E0C0E0D801ED91FC910284A1
:10136000F385E02DC80119958F3F980709F499CFAF
:101370009C01215431092A31310570F48D2F829559
:10138000807F829FC00D1124D11104C00C2E000C4F
:10139000DD0B89CFD0E0E0CF9C01215631092A3105
:1013A000310560F3C0978A30910570F79D2F9295B3
:1013B000907F989FC00D1124E7CFDC01ED91FC9147
:1013C0000190F081E02D1994CF92DF92EF92FF927D
:1013D0000F931F93CF93DF932115310581F4DC0127
:1013E000ED91FC910190F081E02D642FDF91CF9180
:1013F0001F910F91FF90EF90DF90CF9019942A30BA
:10140000310501F52AE077FF1DC06A017B01EC017F
:101410006DE20E94DD898C0144275527BA014C19E1
:101420005D096E097F092AE0CE010E94F288800FD3
:10143000911FDF91CF911F910F91FF90EF90DF905F
:10144000CF900895DF91CF911F910F91FF90EF9072
:10145000DF90CF900C94F2888F929F92AF92BF92C0
:10146000CF92DF92EF92FF920F931F93CF93DF9370
:101470007C018B014C0182E0880E911C5701E5E054
:10148000AE0EB11CD0E0C0E0F40161914F014AE022
:1014900050E0C8010E9442896C016EE2C8010E94BE
:1014A000DD898C0D9D1DC80FD91F8A149B0461F71F
:1014B0004AE050E0F7016581C8010E9442898C0F23
:1014C0009D1FDF91CF911F910F91FF90EF90DF90C3
:1014D000CF90BF90AF909F908F9008956115710548
:1014E00011F00C94E38890E080E008950F931F932F
:1014F000CF93DF93EC018B0161E476E00E946E8A6A
:1015000001151105C1F1F80161918F01662399F16F
:10151000603240F0623231F06C3521F0CE010E9431
:10152000DD89F1CF6CE5CE010E94DD89F8013197AC
:1015300080818C30D1F044F48930D9F08A30B9F010
:10154000883009F762E6EACF823259F024F462E784
:101550008D3021F3D8CF8F3231F06CE58C35F1F23C
:10156000D2CF62E2DBCF6FE2D9CF66E6D7CF6EE6AD
:10157000D5CF64E7D3CF62E2CE010E94DD8990E04F
:1015800080E0DF91CF911F910F910895DB011496B8
:101590004D915C9115976D917C91DC01ED91FC91E1
:1015A0000280F381E02D1994EF92FF920F931F9325
:1015B000CF93DF938C017B01D0E0C0E0F701EC0F0B
:1015C000FD1F6491662361F0D801ED91FC910190BB
:1015D000F081E02DC8011995892B11F02196EECFED
:1015E000CE01DF91CF911F910F91FF90EF90089561
:1015F0000F931F93CF93DF93EC010E94D48A8C0149
:10160000CE010E943E89800F911FDF91CF911F91E3
:101610000F9108958091260881110AC088E29CE00C
:101620000E943E8962E179E188E29CE00C94D48AD0
:101630000895DC0184E694E08D939D9384E0FB01A2
:1016400001900D928A95E1F708953F924F925F9233
:101650006F927F928F929F92AF92BF92CF92DF92C2
:10166000EF92FF920F931F93CF93DF93CDB7DEB727
:10167000EA970FB6F894DEBF0FBECDBF7C012A01FA
:101680003B0169010E940DAD4B015C0187010D5BBF
:101690001F4FC8010E94351618161906ACF00E949B
:1016A0000DAD681979098A099B094616570668061F
:1016B000790608F468C10E94A26961E070E080E0E8
:1016C00090E00E94DBACE5CF42E250E0BE016F5FEC
:1016D0007F4FC8010E94C01589818230D1F0312C22
:1016E000832DEA960FB6F894DEBF0FBECDBFDF9113
:1016F000CF911F910F91FF90EF90DF90CF90BF900F
:10170000AF909F908F907F906F905F904F903F90A1
:101710000895F801848995898334910501F76D81D5
:101720007E818F8198850E944AE44B015C01F6011D
:1017300080829182A282B38246E050E0B701685F66
:101740007F4FCE014D960E9452E8892B41F6F7015A
:1017500080819181A281B38188169906AA06BB0671
:1017600008F4BDCF84819581A681B781881599053C
:10177000AA05BB0508F4B3CF89899A89AB89BC89CE
:1017800086879787A08BB18B4EEC50E070E060E0CD
:10179000C8010E94C015312CC701829698AB8FA753
:1017A000F701B696FAABE9AB08969CAB8BAB670139
:1017B0009AE1C90ED11CBD96FEABEDABC7014296B6
:1017C00098AF8FABFD97FAAFE9AF4701FEE18F0EFF
:1017D000911CF801818D928D181619060CF080CF9E
:1017E000C8010E94DF158333910509F4B2C014F5D6
:1017F0008130910509F464C044F4892B51F3C80188
:101800000E94DF15AC01552775C08330910509F49E
:1018100062C00697A1F7C8010E94DF15B82E44E008
:1018200050E0B401C8010E94C015EB2DE450FF0B3D
:10183000AF0160C08A33910509F45FC084F5853338
:101840009105B1F1C697D9F6C8010E94DF155C0178
:10185000B601CE0189960E94198B8BA59CA5ADA5DA
:10186000BEA5892B8A2B8B2BB1F0EDA9FEA9408058
:10187000518062807380B601CE0183960E94198BDD
:101880008DA19EA1AFA1B8A5A501481659066A066B
:101890007B0609F0B8CF44E050E0B60118C08B33A6
:1018A000910509F440C08F3F910509F492CFA7CF6D
:1018B000C8010E94DF15C8010E94DF15382E89CFAC
:1018C000C8010E94DF1544E050E06FA978ADC8015F
:1018D0000E94C0157ECFC8010E94DF15B82E44E0DB
:1018E00050E069AD7AADC8010E94C0158B2D8450BF
:1018F000990BAC0170E060E0EACFC8010E94DF15EF
:1019000044E050E069A97AA9C8010E94C015F70116
:1019100066A177A180A591A50E944AE466A377A35A
:1019200080A791A756CFC8010E94DF1544E050E080
:101930006BA97CA9C8010E94C015F70162A573A517
:1019400084A595A50E944AE462A773A784A795A7DA
:1019500040CFC8010E94DF1544E050E06FA578A990
:10196000C8010E94C015F70162A173A184A195A1CD
:101970000E944AE462A373A384A395A366A777A7F2
:1019800080AB91AB26CF33243A94AACE1F920F920C
:101990000FB60F9211240BB60F922F933F934F93D4
:1019A0005F936F937F938F939F93AF93BF93EF93C7
:1019B000FF9382E399E00E941980FF91EF91BF911C
:1019C000AF919F918F917F916F915F914F913F91D7
:1019D0002F910F900BBE0F900FBE0F901F90189578
:1019E0001F920F920FB60F9211240BB60F922F93E6
:1019F0003F934F935F936F937F938F939F93AF9397
:101A0000BF93EF93FF9382E399E00E949B7FFF9146
:101A1000EF91BF91AF919F918F917F916F915F9166
:101A20004F913F912F910F900BBE0F900FBE0F90D3
:101A30001F9018951F920F920FB60F9211240BB69C
:101A40000F922F933F934F935F936F937F938F9357
:101A50009F93AF93BF93EF93FF938FEC99E00E9416
:101A60001980FF91EF91BF91AF919F918F917F91DD
:101A70006F915F914F913F912F910F900BBE0F90FF
:101A80000FBE0F901F9018951F920F920FB60F92D6
:101A900011240BB60F922F933F934F935F936F9345
:101AA0007F938F939F93AF93BF93EF93FF938FECAD
:101AB00099E00E949B7FFF91EF91BF91AF919F9121
:101AC0008F917F916F915F914F913F912F910F90E7
:101AD0000BBE0F900FBE0F901F9018951F920F9284
:101AE0000FB60F9211240BB60F922F933F934F9383
:101AF0005F936F937F938F939F93AF93BF93EF9376
:101B0000FF938CE69AE00E941980FF91EF91BF91BC
:101B1000AF919F918F917F916F915F914F913F9185
:101B20002F910F900BBE0F900FBE0F901F90189526
:101B30001F920F920FB60F9211240BB60F922F9394
:101B40003F934F935F936F937F938F939F93AF9345
:101B5000BF93EF93FF938CE69AE00E949B7FFF91E7
:101B6000EF91BF91AF919F918F917F916F915F9115
:101B70004F913F912F910F900BBE0F900FBE0F9082
:101B80001F9018951F920F920FB60F9211240BB64B
:101B90000F922F933F934F935F936F937F938F9306
:101BA0009F93AF93BF93EF93FF9388E29CE00E94D3
:101BB0001980FF91EF91BF91AF919F918F917F918C
:101BC0006F915F914F913F912F910F900BBE0F90AE
:101BD0000FBE0F901F9018951F920F920FB60F9285
:101BE00011240BB60F922F933F934F935F936F93F4
:101BF0007F938F939F93AF93BF93EF93FF9388E26D
:101C00009CE00E949B7FFF91EF91BF91AF919F91CC
